:020000024000BC
:10E000006FF0617C00000000001801180028012852
:10E0100002280328002901290229032904290529A6
:10E02000062907290829002A012A022A032A042A84
:10E03000052AA62A88DF0600D4090500420400202C
:10E04000BC040020CA0300209C03002032030020EF
:10E05000760B0500B60B0500540D0500D40F050026
:10E06000B810050034080500E60705008C02002002
:10E070003602002072150500D00700204C0B050069
:10E080007A12050088980600689A0600D29A06005F
:10E09000DC5C0600145D060072160600A80B060084
:10E0A0000A930600AA1205000A63060064AE050082
:10E0B000F4AE05004EAF05009A1D0500D81D050001
:10E0C000581C0500CE700500F26B0500480A0020C0
:10E0D000047D05006A800500205F0500C45E050020
:10E0E000826205006C5F0500A45E05001A5F0500F2
:10E0F0005A5E0500E45F05003C600500EC5F05002A
:10E10000F05F05008660050044600500746005004E
:10E110002E65050032650500E05F0500E85F05003B
:10E120008460050030650500326105008A660500DF
:10E13000C48D0500388E0500728E05001A73050027
:10E140002E730500627305004C54050072560500DD
:10E150004E570500863A05001C3505005A4B050050
:10E1600098350500D84605006EC1060012BA0600B3
:10E17000D4BE0600E0D30600CCD206003AD6060094
:10E180002AD6060032D6060074D606006AAC06000F
:10E19000000000000000000000000000000000007F
:10E1A000E4D60600D2D0060070D0060000000000C1
:10E1B000000000000000000000000000000000005F
:10E1C000E87B06000E6B0600646E06004C6C0600D1
:10E1D0002676060062930600000000009EAC060052
:10E1E000F6160500245D0600EA620600E2630600FA
:10E1F000000000000000000000000000DE760500C6
:10E20000267B060000000000000000000000000067
:10E21000BE6A0600BA090020905D060060D60600BE
:10E2200000000000000000002ED606005E0F050072
:10E230005274050068D60600D47D0600387F0600BB
:10E24000A47F06001ABF060064D606006CD606003E
:10E25000340B060070D60600801B002088240020A6
:10E2600000000000000000000000000000000000AE
:10E27000000000000000000000000000000000009E
:10E280006373B60082801C419105110523AEF5FE33
:10E29000C5BFB727002037370020938707551307DE
:10E2A000C7C16373F700828023A007009107D5BF21
:10E2B000411122C4B747024006C603A4C72023A6C3
:10E2C00007200F10000011C199E5B747024023A6AF
:10E2D0008720014545A093073500C207C183F19B04
:10E2E000C207C183130740036366F7023727002084
:10E2F0000325077D372700208326877C6391A602AC
:10E30000373700200327C78569D3C207DD8D054550
:10E31000029765BF372700200325C77CE1BF7A211C
:10E3200031EF5A21636CF704B72600203306F7401B
:10E3300021489386867D6375C8028328050003D82B
:10E340006600138687001D8F2A9661175AA2232024
:10E3500016012313060010C15EA1130788FFFAA25D
:10E360006EA1EE222105B387F540FEA2B747024019
:10E3700023A68720B2402244410182800841BDBFCC
:10E38000B747024003A8C72023A607200F100000AC
:10E3900001E523A607218280B727002003AE077D71
:10E3A000B727002003A3877C8146F28763FE6708B6
:10E3B00083A80700636DF50863EBA808138787003F
:10E3C0006364E508F223216705076319E600372631
:10E3D00000200347065F05072308E65E3726002076
:10E3E0001305867DCE237A21239307001306867DAD
:10E3F0002E97420741837AA16383C7033725002004
:10E400000325C57C630DF500EA2211E9DE2223A075
:10E4100016012107BE95A105CEA27AA2B687984320
:10E4200063046702B726002083A6C67C630ED7006C
:10E43000762399EAD6234E231843A106AE96D6A397
:10E4400098C37E22A1077EA2B747024099B7BE8635
:10E45000C687A9BFB7270020B726002083A7077D5E
:10E4600003A6867C2A87B305B5406314F6003A8577
:10E4700029A8938687009C43E369D7FEE377F7FEDC
:10E480002E85E3E4D5FEE3F2F5FE828023AC05FEA3
:10E490001C4181E70CC18280BA8703A787FF6DFF0B
:10E4A00023ACB7FE8280411126C24AC0B744024065
:10E4B00006C622C403A9C42023A604200F1000000E
:10E4C00009E923A62421B240224492440249410191
:10E4D00082802A842105BD654205C18D4181C93BE9
:10E4E00011C9FD572320050042A17CA123A62421A8
:10E4F0002105D1BF23A624210145F1B701114AC846
:10E500004EC6B747024006CE22CC26CA83A9C720F2
:10E510002A8923A607200F10000037250020032496
:10E52000457D8144014609E889ECA1654A8597103B
:10E5300005E0E78060D125A08347E4FF639D2703C2
:10E54000A1C0A6851305457D970005E0E780004F33
:10E5500069DCA1654A85971005E0E7800089F240F3
:10E560006244B747024023A6372126854249D24458
:10E57000B2490561828091E02286032484FF65B759
:10E58000A284E5BFB737002083A7478299E33E8581
:10E590008280BA236315B7009823E30AA7FEDC47FD
:10E5A000F5B7B747024003A7C72023A607200F10DF
:10E5B000000001C599C1814711E6B747024023A673
:10E5C000E7208280B386F50003C80600B306F50095
:10E5D000850723800601E317F6FEC5B737470240DB
:10E5E0008327C720232607200F10000019C191C1DF
:10E5F00011E6374702402326F7208280910503A7C2
:10E60000C5FF11057D16232EE5FEDDB73747024015
:10E610008327C720232607200F10000001C53307DA
:10E62000C50011E6374702402326F7208280050502
:10E63000A30FB5FEE31DE5FEF5B7B747024083A67D
:10E64000C72023A607200F10000081473307F500DD
:10E650000307070019E7374702402326D7203E85E6
:10E6600082808507E5B7011126CA4AC8B74702402C
:10E6700006CE22CC83A4C7202A892E8623A6072073
:10E680000F100000131506019305F004418132C6F6
:10E6900005312A8401C53246CA8521372285F240D8
:10E6A0006244B747024023A697204249D2440561FD
:10E6B0008280B747024003A7C72023A607200F1078
:10E6C000000001C599C1814711EAB747024023A65E
:10E6D000E720054582808507E309F6FE3308F5004B
:10E6E000B386F500034808009422E306D8FEB74736
:10E6F000024023A6E72001458280B747024003A7D6
:10E70000C72023A607200F1000009307F6FFBE9531
:10E710002A966317C500B747024023A6E7208280E8
:10E72000FD159C310505A30FF5FEE5B737470240FF
:10E730008327C720232607200F10000001C53307B9
:10E74000C50019E6374702402326F720014582809D
:10E7500005058346F5FFE397B6FEE31BE5FE374765
:10E7600002402326F72005458280797126D2B734EE
:10E77000002022D403A4448206D64AD04ECE52CCE6
:10E7800056CA5AC85EC662C455C4373A00203729F3
:10E790000020B7390020814BB73A002037CBC901A0
:10E7A000130A8A821309897D938909873E2099EF8C
:10E7B0005C44639A0B0023A2F482032CC4002285DC
:10E7C000C1366284A9A823A6FB00C5BF83A7CA815E
:10E7D00082971C443307F5406376F50003A7490090
:10E7E0001D8F2A979306FB3763EAE6062328090064
:10E7F0002E200820970005E0E780205F5C40584409
:10E80000B1C70C4403A64900AE97BE8663E4B700C7
:10E8100063E4C700B386C74014C4A28B3A8459F49A
:10E82000B72700209387877D984B854663FCE604D5
:10E830007D1798CBB250225492540259F249624A41
:10E84000D24A424BB24B224C4561828063950B0009
:10E8500023A2E4829DB723A6EB0085B703278A0293
:10E8600019CB63EDA7003385A740832709016374A3
:10E87000F5002328A900A28B404455B703A74900FF
:10E88000BA97D5B723A8070075B701114EC6B74789
:10E89000024006CE22CC26CA4AC852C483A9C72049
:10E8A00023A607200F1000003734002093070487A9
:10E8B000C843DC2713040487B9CFB73700209387F8
:10E8C000879D03D7870A21CB83A4470A6385A404C5
:10E8D000B72700201387877D184B138A877D630F26
:10E8E000A70E373900208327C981829763E5A40EDC
:10E8F0008327C981898C829703270A0163F3E40087
:10E900002687B307A7003E85544063E4E70063E42D
:10E91000D7003385D740B747024023A637215C4054
:10E92000639DA702B72400209384847D9848B7375D
:10E93000002083A7C7816315A70A82975440B74771
:10E9400036FE938707C8B6973387A7003A85636476
:10E95000F7006364D7003305D740B73400209387AE
:10E96000C4B1DC539384C4B199CBB737002083A6DC
:10E9700087B93707CDFF7D179C46F98F9CC611E1FB
:10E9800048408547DCC4B737002083A707858297B6
:10E9900005E1DC5089CFDC4499CB976006E0E78045
:10E9A00060E1975006E0E780406023A60400753BD5
:10E9B000DC5091CBB737002003A787B9B7063300E7
:10E9C0001C47D58F1CC7F2406244D2444249B24929
:10E9D000224A056182805C40BE9419BF268525BF0E
:10E9E000829794485840B387A6003E8563E4D700D9
:10E9F000E3E5E7F63385E7408DB7B727002023A886
:10EA0000A75411C5B72700200547238AE754828001
:10EA1000B727002003A70755411122C406C6138457
:10EA2000075511C30297B727002083C7475593F7AF
:10EA3000F70F99E323200400B24022444101828071
:10EA4000011126CAB734002022CC4AC89387048714
:10EA500006CE4EC652C456C2DC27373900209384F6
:10EA600004871304498095E3B73700209387C7B123
:10EA7000D833058B19CBF8339946639BE60AA382FA
:10EA80000700EF1020465C4482971C4491C3829794
:10EA900037240020B73900209307847D03A709821B
:10EAA0009033130A847D8347847D93961700BA962A
:10EAB0009622C9CA8347847D63EEC708230C047C71
:10EAC000373400209307C4B19C371304C4B1639159
:10EAD0000710B737002083A7C781F5C3DC40232880
:10EAE000FA006131B737002083A70785E9CB7C3076
:10EAF00011476366F70CB7370020938787B6DC278A
:10EB0000918BD5EFB727002083C7475593F7F70FB1
:10EB1000DDE783461A0003A6098263C7D70C624467
:10EB2000F240D2444249B249224A924A0561B1BBFD
:10EB3000F8339D46E39BE6F4A3820700EF10803A8A
:10EB40001C4899B7850793F7F70F230CF47CE3EC87
:10EB5000C7F48DB786073E970E23231007000345A1
:10EB6000847DB737002083A7078013172500B73AA5
:10EB70000020BA979C43239C0A80829783D78A817E
:10EB80000347847D93C7F7FF7D8D9317170003A775
:10EB900009823E971E235D8D0AA38347847D81C72A
:10EBA0008507230CF47C8327498081C78297232221
:10EBB00009800347847D83471A00E371F7F0F24030
:10EBC0006244D2444249B249224A924A0561828053
:10EBD0007C3093F7F70FE39E07EEA30404009750F1
:10EBE00006E0E780806CF5B51397170032971A237B
:10EBF00079F785071DB7374702408326C720F1778D
:10EC0000FD17F58F2326F72001000100B72700200C
:10EC10009387877DC84F832787262326D7206A05B9
:10EC200093C7F7FF99835D8D8280B727002083C744
:10EC3000B77D89CFB737002083C7C78791CBB73758
:10EC4000002003A307886307030002830545828031
:10EC5000094582801305F00F8280B737002003C674
:10EC6000479DB727002003A7075C81476315F6007F
:10EC7000814636858280BA8613078702835587FDD1
:10EC8000E389A5FE850793F7F70FCDB7B7370020C7
:10EC900003C7579DB727002083A7C75D2A860507AE
:10ECA00081463E859E236388C700850693076500DD
:10ECB000E3E9E6FE01458280B727002003A7475D10
:10ECC00019E3014615A81C4703D8A700636B05018B
:10ECD00083584700B38608016355D5008146639485
:10ECE00016011843F1BF3E86C10703D3A7FF631780
:10ECF000A30099C123900501328582808506C20652
:10ED0000C182F1BFB737002003C6479DB737002047
:10ED100003A7479781476315F600814636858280B1
:10ED2000BA861307C703835567FCE389A5FE8507E9
:10ED300093F7F70FCDB7032785116DCB411122C48F
:10ED400006C65C258345E5042A8493F7C70F5CA5B6
:10ED50001437522713958601618563F7C506635101
:10ED60000506082793F6F60714B7054693E627002D
:10ED70006314C50093E6170054A45C4389075CC381
:10ED80004CB8032504112E864C430905EFF07F8112
:10ED9000832784115038D443DA27B296118FD4C315
:10EDA000DAA789473CBCB73700200347640383C711
:10EDB000A7836371F7045C2493E707015CA41DA893
:10EDC00093E717005CA46DBF9376F60F63590502B5
:10EDD0000827854513E627006314B50013E61700DE
:10EDE00050A454B8A304070085473CBC8327841172
:10EDF0009C43D5FBB240224401454101828093E708
:10EE000017005CA454B8A3040700032504114C4365
:10EE10000905EFF00FF9832784115038D443DA271E
:10EE2000B296118FD4C3DAA78D47C1B7054582804A
:10EE3000B737002083A7C7AF411122C406C6858B10
:10EE40002A84D5E34165130525F5971006E0E78090
:10EE5000604E51C93C253EA583270412ADE3232013
:10EE6000A4122322A41285472311F40423200500B1
:10EE70007C2854415EA5583418A5054718B5373786
:10EE80000020032707B41385170215811C437D1545
:10EE90001375F50F9CC25C43DCC21C479CC65C47E3
:10EEA000DCC61C4B9CCA5C4BDCCA1C4F9CCE5C4F26
:10EEB000DCCE19CD9386060213070702C1BF832754
:10EEC000441288C3835724042322A412850769BFF0
:10EED000B73700209387879D9A2705079AA7B240E6
:10EEE0002244410182805C2423090400054593C724
:10EEF00047005CA4EDB71C2D93F7E70FC5EB1C3D55
:10EF0000D5E73029542509CA3737002083456503E2
:10EF10000347B78363E7E50013F7060149CB0147D1
:10EF200009C6C18A0357E51B81C68356251C36973F
:10EF30003DCFB737002003D587871307C712374661
:10EF40000F00B335A702411113060624814622C4DF
:10EF500026C206C67D543305A70297D006E0E78097
:10EF6000C0B4B737002083C7F783B384A700B7378F
:10EF7000002003A787A68327070963F387003E8441
:10EF8000184375FBB737002083A7C7818297814755
:10EF90006364A400B307A440B2402244B3B797000F
:10EFA00093C7170092443E854101828081473E8588
:10EFB0008280B737002003A747B47C53FDFF8280CF
:10EFC00001114EC6B73900209387899D22CC03A436
:10EFD000870926CAB7340020938704879E274AC82A
:10EFE000035964080325040906CE3309F902B7471B
:10EFF0000F001387F7239387072452C456C25AC0C1
:10F000009389899D938404873A993359F902636DF2
:10F010002503373A00208327CA8133092541829787
:10F020006367A9023309A9406346090283570404B0
:10F03000A30F040085072310F4048347041463948A
:10F0400007102285CD2511A2DC403E95D9B7DC40C2
:10F050003E99C9BF8327CA81829703278408636FBB
:10F06000E508198D7E3C9A248E07B387E7021307C3
:10F07000003293870719B3D7E70263E5A708B74AB9
:10F080000F00138BFA23938A0A24835704048507FD
:10F090002310F4048347041499E32285692522850B
:10F0A000971006E0E780008E631D0524832604097F
:10F0B0008327C408D840B6973E8563E4D70063E44D
:10F0C000E7003385E7407C3C035964082328A40803
:10F0D00085077CBC9E243309F9025A993359590398
:10F0E000636C2505330925418327CA8182976369AB
:10F0F000A9043305A940E34A05F80DBFDC40998F08
:10F100003E958DB7A1452285970006E0E780C07F38
:10F11000A305A402B737002003A3C7856303031E1A
:10F120006244F240D2444249B249224A924A024BD6
:10F130008945154505610283330927412A996DB731
:10F14000DC403E997DB7228551252285971006E047
:10F15000E78040836317051A8A2483576408B746FB
:10F160000F001386F623B387A7029386062403278E
:10F170000409230B040283AA4400B297B3D7D70231
:10F18000636BF718B307F7408326C4082324F408F9
:10F19000014BB387E6003E8963E4D70063E457017F
:10F1A000338957411E3023282409A1CB83560404F8
:10F1B0005A3037460F0056B03387E640B387E70230
:10F1C0003A301306062481468145BA97C207C183A7
:10F1D0003385A7023EB097D006E0E780008D11CDC1
:10F1E0004A95333925012E99AA8763142B0163644C
:10F1F0005501B30755412328F4088327CA81829714
:10F200002A898327CA818297E30D25FF8327CA8134
:10F210000329840882976365A9103305A940630A0E
:10F22000051083DA84008357640837490F001307F9
:10F23000F923B387570313090924BA97B3D72703D0
:10F24000373700200347F783BA9763E4A70EB33537
:10F250002503035A2402568681463305250397D099
:10F2600006E0E7808084330BAA0033055A03374653
:10F270000F00130606248146814597D006E0E780FB
:10F28000C0820DC1B337250356868146B305B90246
:10F290003305A902BE9597D006E0E78000813305CB
:10F2A000AA402AB03545975006E0E780600D23ACB0
:10F2B000890838348547631DF700930700FD7CA457
:10F2C000B737002003A587B0DC24B1CFEFF0EFF211
:10F2D000B736002003A646B4B73700209387C7B1DE
:10F2E0001547F8B35846F977FD17F98F5CC60F102C
:10F2F000000083A746B48966060B94C723A267075C
:10F30000D8C7F2406244D2444249B249224A924AA2
:10F31000024B05618280B3065701B387F640ADB555
:10F32000DC403E99DDBD8145970005E0E780C009DE
:10F3300045B7DC2423AC090885C3B737002003A5F3
:10F3400047B0970005E0E780C042B7E700E0370725
:10F35000000223A2E72075B78347940285456244E3
:10F36000F240D2444249B249224A924A024BB395F2
:10F37000F500C205C18101450561170305E067007D
:10F38000C3A6011122CC4AC84EC606CE26CA52C414
:10F3900056C25AC0383585472A842E8983290509E3
:10F3A0006315F71E83570508035BC503373A002032
:10F3B00093060A8783DA8600130A0A8763FF6719B0
:10F3C0001429639CE618032785116318071803277F
:10F3D000450A6314071874351D476390E6182A3DE3
:10F3E000330BFB409307204E330565038324440908
:10F3F00037460F001306062481463305F502B7375A
:10F40000002083C7E783B3549502B3B5AA02BE9424
:10F41000C204C180231394083385AA0297C006E072
:10F42000E780A068AA9933B5A9002E954E87832757
:10F430004A0019E163E4F9003387F940B3845403C7
:10F44000B7460F009387F623938606242320E9000E
:10F45000BE94B3D4D40293171B00A6976369F70E2A
:10F460001D8F2320E900B739002083A7C981832499
:10F470000900829763EEA4103385A440635D050AFA
:10F4800083A7C981373B0020130B0B878297032783
:10F4900009006365E510198D7E3C03578B008E07CC
:10F4A000B387E7021307003293870719B3D7E70240
:10F4B00063EBA70E374A0F00930AFA23130A0A24B4
:10F4C0008357040485072310F4048347041499E345
:10F4D0002285912C2285970006E0E780A04A6DE105
:10F4E000832604098327C40803274B00B6973E856B
:10F4F00063E4D70063E4E7003385E7407C3C835452
:10F5000064082328A40885077CBC83578B00B38438
:10F51000F402D694B3D444036363950CB3049540CA
:10F5200083A7C98123209900829763EEA40A3385BB
:10F53000A440E34705F8B737002083C7F78363E2A9
:10F54000A708B737002023A887A601459DA88326D2
:10F550004A00B387F6403E9729B783576408374778
:10F560000F00B38457039307F723A6979304072448
:10F57000B3D4970263E79900B3849940232099009C
:10F58000DDB583274A00BE99C5BF23A03501E1BD83
:10F59000B737002083A74787BE94F9BD83274B0068
:10F5A000998F3E95D5BDA1452285970006E0E7805D
:10F5B000A035A305A402B737002083A7C78581EF34
:10F5C0007D55F2406244D2444249B249224A924AAD
:10F5D000024B05618280894515458297D5B7B304F2
:10F5E0009740AA9435BF83274B00BE9489B721CD9D
:10F5F00001116C0022CC06CE2A84613339C1FD573B
:10F600006307F502B736002093868682FC3A94564B
:10F61000324791C285836360F702B307F7403EC665
:10F62000B24503459402970005E0E780E091F2407F
:10F63000624405618280B736002083A646873697EC
:10F64000E9BFBD3AEDB78280B737002079711387E3
:10F65000879D4AD00329070906D622D426D24ECE4A
:10F6600052CC56CA094763000906B7340020938A72
:10F67000879D9387C4B1FC3395469384C4B10D47ED
:10F680006383F604DC442A8A99CB975006E0E7802E
:10F690006012975006E0E780409123A60400FD59D0
:10F6A0006C004A85F93915E937150020130505D591
:10F6B000EFF0AFB4A147DCA0B737002083A747B471
:10F6C0000947F8D30D47B250225492540259F249D7
:10F6D000624AD24A3A854561828063743501324478
:10F6E000AA8903290900E31D09FAFD571307F00F42
:10F6F000E38BF9FC914763F187029307B4FF232062
:10F70000FA0023A2FA0A0147DDFFB737002083A7DA
:10F7100047872320FA0045BFB737002083A74787D4
:10F72000ED17A297E9BF797126D206D622D44AD026
:10F730004ECE52CC56CA5AC85EC6834755030344C0
:10F740007513AA843E941374F40F9307400263F672
:10F7500087001304B4FD1374F40F03AA841383AA5F
:10F76000C413A38B841222865285D68597C006E0E7
:10F77000E780E030058915E503CBD41201498149C2
:10F78000337B6403930B50024A865285D68597C01B
:10F7900006E0E780C02E058915C5639169031374DF
:10F7A000F90F238B8412B250225492540259F24919
:10F7B000624AD24A424BB24B456182808509E209D6
:10F7C00093D989410509E31179FDE1BF83278509B3
:10F7D00003560504797193D60701BD8EC206C18216
:10F7E000358E1357764093575640898B058B5D8F26
:10F7F00093573640918B5D8F93571640A18B5D8F49
:10F8000093171600C18B5D8F9317360093F707028D
:10F810005D8F931756009355860093F707041E06D5
:10F820005D8F1376F60F518F93D7554013D6354021
:10F83000118A898BD18F13D67540D18F13D615407D
:10F84000218AD18F13961500418AD18F13963500E6
:10F8500013760602D18F13965500137606049E0583
:10F86000D18F93F5F50FCD8FA20745465D8F3307F6
:10F87000C70222D42A8426D252CC56CA032A841321
:10F88000832AC4135AC806D6369742074183935732
:10F890007740135557400989858BC98F13553740D9
:10F8A0001189C98F135517402189C98F1315170066
:10F8B0004189C98F1315370013750502C98F1315B8
:10F8C000570093558700137505041E07C98F1377DA
:10F8D000F70FD98F13D5354013D755401189098BB0
:10F8E000498F13D57540498F13D515402189498F0C
:10F8F000139515004189498F13953500137505023D
:10F90000498F13955500137505049E05498F93F58E
:10F91000F50F4D8F2207D98FB387C7024AD04ECE3D
:10F920005EC662C4B697C207C18313D7774013D5AA
:10F9300057400989058B498F13D537401189498F65
:10F9400013D517402189498F139517004189498F95
:10F950001395370013750502498F1395570093D5FA
:10F960008700137505049E07498F93F7F70FD98F0A
:10F9700013D5354013D755401189098B498F13D5BD
:10F980007540498F13D515402189498F139515006E
:10F990004189498F1395350013750502498F1395D9
:10F9A0005500137505049E05498F93F5F50F4D8F8E
:10F9B0002207D98FB387C702130650025285D68516
:10F9C000B697BD8E93940601C18033F6C402137BB3
:10F9D000F60F97C006E0E780800A05890DED8347A2
:10F9E000D41201498149B3849702130C5002C1809B
:10F9F0004A865285D68597C006E0E780400805898B
:10FA0000937BF90F11C563863403850993F9F90FC8
:10FA10000509E31F89FD230B6413B250225492544D
:10FA20000259F249624AD24A424BB24B224C4561DA
:10FA300082805E8BCDB7797122D406D6BC312E84FC
:10FA400023160100DC87DC21100802C05C87DC3152
:10FA50008A8502C2DC8602C402C802CA02CC02CE77
:10FA60000D2A0347F1011C200145631EF7000347DF
:10FA7000E1011C3001456318F7000345D1013C202A
:10FA80001D8D13351500B25022544561828001113D
:10FA9000B737002022CC03A487A926CA4AC84EC67D
:10FAA00006CEAA8413092500854905C09C3038304C
:10FAB000858B6304F700405CCDBF19469305440075
:10FAC0004A85EFE01FBFE31835FF2285F24062440C
:10FAD000D2444249B249056182804111B7370020C2
:10FAE00022C403A487A926C24AC006C693042500DF
:10FAF000054901E82285B24022449244024941016D
:10FB00008280A6851305A4023D37E30525FF405CEE
:10FB1000CDB74111B737002022C403A487A926C25C
:10FB20004AC006C693042500054901E82285B24073
:10FB300022449244024941018280A6851305A40112
:10FB4000DD3DE30525FF405CCDB70111B73700204F
:10FB500022CC03A407A926CA06CE2AC42EC68544F1
:10FB600019E40145F2406244D244056182809C84DC
:10FB70001830858B6304F7000044DDB71946930500
:10FB8000A10013052400EFE0DFB2E31795FE054561
:10FB9000D1BFB736002083A7C6B01307001098C3A3
:10FBA00023A0070018310348250022074208429786
:10FBB000034805004297034835006208429798D7EA
:10FBC0005831034865002207420842970348450020
:10FBD00042970348750062084297D8D71835034802
:10FBE000A500220742084297034885004297034830
:10FBF000B5006208429798DB58350348E5002207B4
:10FC0000420842970348C5006835429762052A9723
:10FC1000D8DB9831A821220742052A9788212A9704
:10FC2000A83162052A9798CFD831E82122074205EA
:10FC30002A97C8212A97E83162052A97D8CF9835A4
:10FC4000A825220742052A9788252A97A835620504
:10FC50002A9798D3D835E825220742052A97C82540
:10FC6000EC352A97E2052E97D8D3D843759BD8C395
:10FC7000D84313671700D8C398431367170098C376
:10FC800003A7C6B05C43858BBDE71C4F01451CA292
:10FC900083A7C6B09C4FA1831CB283A7C6B09C4F5C
:10FCA000C1833CA283A7C6B09C4FE1833CB283A72B
:10FCB000C6B0D84F58A2D84F218358B2D84F4183ED
:10FCC00078A2D84F618378B2985318A698532183AD
:10FCD00018B69853418338A69853618338B6D853E1
:10FCE00058A6D853218358B6D853418378A6DC53FD
:10FCF000E1837CB68280010061B7B737002003A79B
:10FD000047B41605136505083C4B93E707083CCB41
:10FD1000B737002083A7C7B003A7450E88C398CB89
:10FD200003A7850E0145D8CB03A7C50B98CF03A722
:10FD3000050CD8CF03A7450C98D303A7850CD8D3BF
:10FD400003A7C50C98D703A7050DD8D703A7450D62
:10FD500098DB03A7850DD8DB03A7C50D98C703A7BC
:10FD6000050ED8C798431367070498C38280B73736
:10FD7000002003A747B41605136505083C4B93E71D
:10FD800007083CCBB737002083A7C7B003A7C50E31
:10FD900088C398CB03A7050F0145D8CB03A7C50B94
:10FDA00098CF03A7050CD8CF03A7450C98D303A77A
:10FDB000850CD8D303A7C50C98D703A7050DD8D7B2
:10FDC00003A7450D98DB03A7850DD8DB03A7C50D59
:10FDD00098C703A7050ED8C798431367070498C3AD
:10FDE000B73700209387C7B1130700F8F8A38280C4
:10FDF000B736002003A706B141114AC01C5F06C6F2
:10FE000022C4998326C2858B3689B5CF9307000615
:10FE1000373400201CDF8347C4B19304C4B193F787
:10FE2000070489CFB737002083A7C7818297C8CC42
:10FE30008347C4B193F7F70B230EF4B08347C4B1E3
:10FE400093F7070285C38347C4B1373700200327E0
:10FE500047B493F7F70D230EF4B0DC48A16614C73E
:10FE600086077CD7DC2093F7070491EF8547DCB049
:10FE7000B737002083A747B4096798C7130700FC6A
:10FE8000D8A09848F8D3032709B11C5F9183858BCC
:10FE900089CBC1471CDFB73700209387C7B18546A0
:10FEA000D4A31C5F9D83858B91CB930700081CDF37
:10FEB000B73700209387C7B10547D8A3B7370020CD
:10FEC00083A7C7B0D8430583058B19C7D843759B53
:10FED000D8C3D843799BD8C3B24022449244024944
:10FEE00041018280B7370020B736002003A647B40F
:10FEF0009387C6B103C7C6B1058B19E79833058B45
:10FF000001E7785265FBD833A38207008280373837
:10FF10000020032708B11C5F9583858BBDE701C6D0
:10FF20001C5BBD831CA29DC6832708B1985B460756
:10FF3000935767016356070093E707C0C207C18361
:10FF400003970600C207C18709C7BA970947B3C715
:10FF5000E7029EA285C11C3191CF3E951C35054715
:10FF6000194593F6F7066393E602E207E187394500
:10FF700063CE0700832708B13737002001459C5F17
:10FF8000ED838D8BA303F7B28280054582804111FA
:10FF900022C406C63734002026C2032744B43DE5F8
:10FFA000AE877453FDFEB73400209384C4B13E8500
:10FFB000B28523810400974006E0E7802013B7371D
:10FFC000002083A707B1B70680009843558F98C3D8
:10FFD000D857719BD8D7832744B4A3820400A38049
:10FFE0000400094798C3832644B4B7370020938799
:10FFF000C7B1B823058B11E7B833058B19E3F85265
:020000025000AC
:100000006DFBB24022449244410182808D47631FC0
:10001000F500B737002083A707B1B70680009843E3
:10002000558F98C3D857719BD8D775BF8547E31CA8
:10003000F5FA5447F977FD17F58F5CC70F100000EC
:10004000032744B48967130600F81CC7B73700209C
:100050009387C7B1D0A3B737002083A707B19C43CC
:10006000B1838D8B91E7930760197CD354C7A5BFEB
:100070009307E01BDDBF5D7152DC373A0020032798
:100080000AB186C6A2C4A6C2CAC04EDE1C43B73996
:1000900000203739002093F7F7E793E707081CC3E0
:1000A00083A689B93707CEFF7D179C4613068002C9
:1000B0002A84F98F9CC6832749B42800AE8423A8DC
:1000C000070493051008EFE06FD43545974006E02C
:1000D000E780002B83270AB19376F41F370633009D
:1000E00023A40700984B370FFCFF4E881367F703D4
:1000F00098CBF84FCA88130510F8137707E0558F8F
:10010000F8CF9843F576FD16758F98C337370020E2
:10011000832649B41307C7B1A3020700A300070051
:10012000054798C29843D285B70204001377F7E7D2
:1001300098C398439303802511491377F7E7136712
:10014000071098C303A789B97D1F85491C47930FE2
:100150008002D18F1CC793079005BCCA01473400A9
:100160001353370026938347030013767700B3D7E2
:10017000C740858BE1C383A705B1832E88B9239C33
:1001800007042390070603AECE02137EDEFF23A6EC
:10019000CE0383AE0700137EF70793FE0EF833EE0F
:1001A000CE0123A0C70103AE4702336E5E0023A237
:1001B000C70383AE48B4014E23A27E0603DA0706C6
:1001C00063074E0303AE0703038A0600135EFE00B7
:1001D000620E135E8E416358CA0103AE0703135EBD
:1001E000FE002380C60103DE0706137EFE0F03AA6E
:1001F0004E0663060A0003DA8705E37F49FB03AE78
:100200004702337EEE0123A2C70383870600635CA7
:10021000F400034E03003396C9001346F6FF33760D
:10022000C6012300C3003E8663D3A7002A861315A8
:100230008601618505071377F70F8506E312F7F34B
:10024000B640264496440649F259625A616182805A
:10025000B737002083A747B4D8479316170163D256
:10026000060298479316170163DD06007D57B8D73D
:10027000372700201307877D544F850654CF116719
:1002800098C798470D83058B11CF37370020130788
:10029000C7B1342393E6160034A3930600F854A3A1
:1002A000214798C79847058B19CB3737002013078C
:1002B000C7B1143393E6160014B3054798C798479F
:1002C0000983058B09E798470583058B31CB3737C1
:1002D00000201306C7B1A30206009447B7350020DB
:1002E00083A505B18982858AE5C69441B1828D8A4C
:1002F000E9EEA84B54521376050294324DC2F9E24E
:100300009306D005D4CF8346C7B193E61600230EDB
:10031000D7B0114798C7D855719B13671700D8D528
:1003200098479316370163D40602373700209306A7
:10033000879D03C606071307879D418A45C203C7E9
:100340000607136707022388E606056798C79847DC
:100350009316270163DF0600373700201307C7B164
:100360005423E206E18663D40600854654A3096758
:1003700098C798479316070163D2060237370020C3
:100380001307879D83461707858AADCA83461707DB
:1003900093E62600A308D706216798C78280ADD2CE
:1003A00005466395C60093061006A9BF09466395E6
:1003B000C60093065006B9B70D466395C60093066E
:1003C000900689B79306B00635BF9306C0061DBFD9
:1003D00038321367170038B209472DBF8346070725
:1003E0000946BD8A6388C600834607070D46BD8A55
:1003F000E39DC6F491462308D70681BF83461707BD
:10040000918AD9DA8346170793E6860061B7B73732
:10041000002083A747B4B73600201387C6B19047A2
:1004200010CF90470D82058A11CA3023136616003B
:1004300030A3130600F850A3214690C79047058AC1
:1004400019C610331366160010B3054690C79047BF
:100450000982058A09E690470582058A31C6A3020A
:1004600007009047B735002083A505B10982058AAA
:1004700059CA904131820D8A41E6A84B50531375F9
:100480000502103221C935EA1306D005D0CF03C6C4
:10049000C6B113661600238EC6B0914694C7D455D4
:1004A000F19A93E61600D4D5944713962601635B20
:1004B00006005423E206E18663D40600854654A371
:1004C000096798C798479316070163D40600216708
:1004D00098C7828055DA05456315A60013061006F5
:1004E00075B709456315A6001306500645B70D45B7
:1004F0006315A6001306900651BF1306B00679B720
:100500001306C00661B7343393E6160034B3894648
:1005100071B737370020B7360020138686B413072B
:1005200087B65C372C3E484AAE97FD8BB355F50035
:100530001CB25CB785898DE9183B8146130800021F
:10054000B3F7E7020147B355E50085899378F70FC4
:1005500089C96395D700A30016018280850693F6AA
:10056000F60F0507E31107FF8280B7370020938756
:10057000C7B1DC3393F7F70FD1EBB737002083A770
:10058000C781411122C44AC006C626C282973739A4
:100590000020930789B68047130989B66302A40631
:1005A00063688504018DB7340020938784B4BC2F21
:1005B00013545500938484B46364F40485676371B1
:1005C000F404813FBC2C032789009396570036978B
:1005D0001D8C2324E900E376F4FE22448830B240E7
:1005E0009244024981454101174306E067004320D8
:1005F000B737002083A7478733848740229565B7A4
:10060000B240224492440249410182808280B7373D
:10061000002083A7C781011122CC26CA52C406CE6E
:100620004AC84EC68297B7340020938784B6804765
:10063000014A6300A406938484B663658506018D30
:1006400037370020930787B4BC2F13545500137A13
:10065000F501130987B4636BF402B739002093895D
:100660000987453D8346A90103A8840083A5490065
:10067000139756004297158C3A86636407016364AA
:10068000B7003306B74090C4E37DD4FC1604336A48
:100690004401F24062445285D2444249B249224A5E
:1006A00005618280B737002083A74787338487405E
:1006B000229579B7B737002003A747B4856793879A
:1006C00007777CD3B737002083A787B983A60709AC
:1006D000139656006358060083A607091396660012
:1006E000634406007453FDF282800000EFE04FB2D5
:1006F0007300000000000000970200009382C20C0B
:100700000383020023800200630F0300F3251034EB
:100710002EC0970500009385A5FD73901534EFF06A
:100720001FCF7300203086DCEFF09FB2E65082804E
:0407300000000000C5
:10073400B72700203727002083A7077D0327877C5E
:1007440001456313F7008280F62399E2D623369598
:100754009C43C5BFB737002083A587823727002075
:1007640093878782138605222328C77CDA239387FD
:1007740085FFB72600204111BA97056523A4F67CAE
:1007840006C61D05935637006374E50093060020E2
:100794003307D600372500202326E57C23A0E52255
:1007A400E11656A2231306001CC3998FE1175EA31A
:1007B40023130700B53FB240B7270020239FA77C2F
:1007C40041018280184183A785FF6319B7001CC1CA
:1007D400FD5723AC05FE238FF5FE8280232CF6FE05
:1007E400C5BF411122C426C23744024006C6832431
:1007F400C420232604200F10000009E92326942096
:100804001545B24022449244410182800347E5FFEA
:100814009307F00F6306F700232694201145D5B7FC
:100824009700FB1FE780C08E014523269420D1BF8B
:10083400411126C24AC0B744024006C622C403A9D5
:10084400C42023A604200F10000089E523A6242138
:10085400154515A0B727002083C7977D2A842E85C8
:100864006375F400894763EE8700A53FB7470240EC
:1008740023A627210D45B240224492440249410156
:10088400828083A785FF99E703C7E5FF9307F00FED
:100894006308F700B937B747024023A627214DBFA5
:1008A40037250020238F85FE1305457D9700FB1F08
:1008B400E780C096A16522856D2C014523A62421DD
:1008C4005DBFB727002023AA077C8280BDCD797144
:1008D40022D406D626D24AD04ECE01444147B3D7BD
:1008E4008540858BB1CF1205314722953305E5024A
:1008F400B737002003A987868544B3948400C204D3
:10090400C180BE892A990327090011C7032549001C
:100914002EC60297B24531473304E40283A7898681
:100924003E941C4489E72320090023220900B25085
:100934002254A58D02599254F2492E854561828034
:100944000504E31EE4F88144DDB72E85828041115D
:100954001397050122C406C626C24AC041872E84C5
:10096400635107029700FB1FE780409211C1953D38
:10097400A1673D8C2285B240224492440249410140
:100984008280EDD9AA8701474146B356E440858A5F
:100994009DCA9207BA97B146B387D702B7360020EB
:1009A40003A986868544B394E400C204C1803E99B9
:1009B4008327090003254900829723200900232265
:1009C4000900258C45BF0507E311C7FC8144D5BF49
:1009D400411126C2B747024006C622C483A4C720D9
:1009E40023A607200F100000B737002083A7C78471
:1009F400372400201304045291C782971C403E956B
:100A040008C031A0B737002083A7C781FDF71C4079
:100A1400374703001307D73FB387E70237A72600FA
:100A2400130737ECB240BA971CC0B747024023A65D
:100A3400972008402244924441018280797126D251
:100A4400B747024006D622D44AD04ECE52CC56CA1C
:100A54005AC85EC662C483A4C72023A607200F1009
:100A6400000005E123A697200945B2502254925470
:100A74000259F249624AD24A424BB24B224C456176
:100A84008280B737002083A7C781BA8A368AB28B9F
:100A94002E8BAA898297B737002003A787863E89C1
:100AA4000144B146C147330CD402330687011042D6
:100AB40059E2C165938505F0414597F0FA1FE78037
:100AC400205819EDB737002083A7C78581C7814512
:100AD40011458297B747024023A697202D4571B749
:100AE400B737002003A7478239E323A2A782230054
:100AF40005008327898605473317870023260500C9
:100B0400232475013AA123225501E29723A037013A
:100B140023A2670123A4570163040A0023008A0067
:100B2400B747024023A69720014581B73E875C471B
:100B3400F5FF48C76DBF0504E317F4F6B747024055
:100B440023A69720214515B7B737002083A7C7866A
:100B5400411122C406C6372400201304847D89C7AA
:100B640082975C483E9548C84848B24022444101B7
:100B74008280B747024083A6C72023A607200F1010
:100B84000000372700200347977D6370E50237365E
:100B9400002013171500032506823A951A21D98DD2
:100BA4000EA123A6D7200145828023A6D7200D4578
:100BB4008280B747024083A6C72023A607200F10D0
:100BC4000000372700200347977D6372E50237361C
:100BD4000020131715000325068293C5F5FF3A95E7
:100BE4001A21F98D0EA123A6D7200145828023A6C0
:100BF400D7200D45828001114AC83747024006CEEE
:100C040022CC26CA4EC652C40329C7202326072055
:100C14000F100000130705FF1377F70FFD4763E379
:100C2400E70AB146B306D502B737002003A7878683
:100C340036971C43C1CB9354450005443D89331575
:100C4400A400131405014180AE892685A28597F07E
:100C5400FA1FE780206C2A8A29C9A2852685913F3C
:100C6400B737002083A7C781B73400209384048753
:100C740082979E242A848146B38537031306006431
:100C8400B3B7370313850532B335B500BE95EFC04E
:100C9400513AB30785003E87D44063E4A70063E478
:100CA400D7003387D7402324EA00B747024023A65E
:100CB40027210145F2406244D2444249B249224AC2
:100CC40005618280B747024023A627210945DDB785
:100CD40001114AC8B747024006CE22CC26CA4EC6E6
:100CE40003A9C72023A607200F100000BD4763EB0C
:100CF400A70431473307E502B737002083A7878667
:100D0400BA979C43A1C305443314A4004204418010
:100D1400AE840145A28597F0FA1FE780A05FAA89F7
:100D240011C5A2850145713523A49900B747024036
:100D340023A627210145F2406244D2444249B249E4
:100D440005618280B747024023A627210945E5B7FC
:100D5400797126D252CCB744024006D622D44AD066
:100D64004ECE56CA5AC85EC603AAC42023A604207F
:100D74000F100000B727002083C7977D6378F50024
:100D8400B737002083ABC78163970B00B747024096
:100D940023A6472199A03739002013090987AE8A71
:100DA400032B490083558900B74736FE938707C84C
:100DB4003E9BB387C5022A84B2898146B3B5C50276
:100DC40013850732B337F50013060064BE95EFC0F0
:100DD40051266370AB0223A644210145B25022542C
:100DE40092540259F249624AD24A424BB24B45618B
:100DF4008280829B83558900AA8413060064B3878A
:100E040035038146B3B5350313850732B337F5008F
:100E1400BE95EFC01122B3079500BE840327490095
:100E240063E4A70063E4E700B384E740D685228542
:100E340097F0FA1FE780004E01C904C5B747024086
:100E440023A64721054559BF936504F0C205C18116
:100E5400414597F0FA1FE780A01E11E9B73700203B
:100E640083A7C78585D7A2851145829705B73737EC
:100E740000208327478299EF2322A78285472326D0
:100E8400050004C52311550100A11CB1232205004E
:100E940075B7BA87D84775FFC8C7CDB779714ECE35
:100EA400B747024006D622D426D24AD052CC56CADC
:100EB4005AC85EC662C466C26AC083A9C72023A694
:100EC40007200F10000025C141443689B28A2E8ABA
:100ED400AA84B14C373B0020054D130C0003B30B1F
:100EE400940303278B865E971C43B9EF9375F40034
:100EF400B315BD0013554440C2055686C181137510
:100F0400F50FB93531C183278B86DE9784C323A2BD
:100F140047016304090023008900B747024023A660
:100F24003721014521A023A637210945B250225477
:100F340092540259F249624AD24A424BB24B224C71
:100F4400924C024D456182800504E31A84F9B74747
:100F5400024023A637212145D1BF011122CC26CA44
:100F64004AC84EC6B747024006CE03A9C7202A8402
:100F7400AE89B28423A607200F100000D13B22853E
:100F8400CE8597F0FA1FE780E0382A8405C5B73785
:100F9400002083D58787130600648146B3879502B2
:100FA400B3B5950213850732B337F500BE95EFC08C
:100FB400510848C013351400F2406244B747024058
:100FC40023A62721D2444249B2490E0505618280F5
:100FD400011122CC4AC84EC6B747024006CE26CAE3
:100FE40083A9C7202A892E8423A607200F10000076
:100FF40097F0FA1FE7800032AA8419C12311050073
:10100400A2854A857D36B727002083C7877D6399EB
:101014002701B737002003D78781598C239C878009
:10102400B747024023A63721014591E01945F24014
:101034006244D2444249B24905618280011126CA00
:101044004AC8B744024006CE22CC4EC603A9C420E7
:1010540023A604200F1000009307F00263E6A70400
:10106400B1473304F502B739002083A78986A297D4
:101074009C439DCB9377F5008545B395F500C20558
:10108400C1811181B13783A789860145A29723A025
:10109400070023A2070023A62421F2406244D2447D
:1010A4004249B24905618280B747024023A62721FD
:1010B4000945E5B7411126C206C622C4B747024016
:1010C40083A4C72023A607200F10000097F0FA1F5F
:1010D400E780402419E90145B2402244B747024061
:1010E40023A69720924441018280B737002083A72A
:1010F400C78100458297B7370020938707876367C6
:10110400A402D843B74636FE938606C83305A440E6
:101114003697E372E5FC13070064B335E5029227C2
:1011240081463305E502EFC0C1707DB7D8433A94D8
:10113400C9BF4111B737002006C623A6A78602956A
:10114400B240B727002023A8A77E01454101828031
:10115400914763E9B700B73700208A059387478032
:10116400BE9588C18280B737002023A20782373515
:101174000020B7370020411123A607865146B73710
:10118400002081451305458006C623AE078022C48E
:1011940026C23724002097F0FA1FE7802020130589
:1011A400847D13068002814597F0FA1FE780001FB3
:1011B400EFF04FDAB737002083C7D7831304847D59
:1011C400854513D527008D8B3E958D473305F50254
:1011D4009947B734002039051375F50F28A0330556
:1011E400F5021305052497F0FA1FE78060E523A4B0
:1011F400A4862DCD3020994781453306F602130687
:10120400062497F0FA1FE780601983A784863820A4
:10121400B7340020938707240A0723A0F480BA97E1
:10122400373700202320F782EFF0AFE91D211C306F
:1012340083A60480371605001397270036971306F4
:10124400068D10C3138717001377F70F0A07371695
:10125400050036971306269510C3138737008907B0
:1012640093F7F70F8A0718B0B69790C3B240224499
:10127400924441018280372700201307877D1C3365
:10128400342363FFD700B736002083A60680138675
:10129400170010B313972700369708C33E85828042
:1012A4009307F00FE5BF1C41F1CF41777D8FB7065F
:1012B400002089476319D70C5A2171C7411126C2EE
:1012C4001946AA849305F00F610506C622C497F057
:1012D400FA1FE780A01E05478D47630FE5089C446D
:1012E40091C7985C994749CBD85C59C737340020DB
:1012F4001306000481451305848297F0FA1FE780E2
:10130400E00913060004A6851305848297F0FA1FEA
:10131400E780200293078482DA2701E7130700108D
:10132400DAA7F82719E30547F8A79A2B19E36D47BD
:101334009AABF83719E31547F8B7B82B19E3054703
:10134400B8ABB83B19E3F837B8BBD82B19E325473A
:10135400D8ABF82801E71307C003F8ABDC5791C7F3
:101364008297B72700202390A77EB73700207D57A8
:10137400A38EE7BECD3B8147B240224492443E85D2
:101384004101828089473E85828001114AC83739EC
:1013940000208327098706CE22CC26CA52C456C20F
:1013A4004EC68297130A0064B335450313090987AF
:1013B400835A89008146568633054503EFC0614749
:1013C400B72700201387877D004FAA840145630651
:1013D40094029389877D33858440636E940003254A
:1013E400490056868146B335AA023305AA02EFC0E6
:1013F4004144018D269523AC9900F2406244D244C5
:101404004249B249224A924A05618280011122CCA2
:101414002E84B7E506000A8541469385C5C706CEE6
:10142400EFC0417A180806043A94B73700200355F0
:1014340004FF83D7A787F2406244AA9737450F0079
:10144400130505243355F50205618280B737002062
:1014540083D7A78751471D45637CF7027947194510
:101464006378F7021307200315456373F702130724
:10147400B0041145637EF700130740060D456379F8
:10148400F7001307600909456374F70013B5B70F34
:101494008280011122CC06CE2A842EC6EFF04FD3CF
:1014A400B245F240818D33A5A5022295624413759D
:1014B400F50F05618280011122CC06CE2A842EC646
:1014C400EFF00FD1B245F240818D33A5A5022295EC
:1014D40062444205418105618280011122CC06CE1D
:1014E4002A842EC6EFF0CFCEB245F240818D33B5BB
:1014F400A5022295624405618280B737002023A0AB
:10150400A7888280B737002013878782585739CF3E
:10151400411122C426C24AC006C613898782029793
:10152400B72700201387877D1A272A849384877D11
:1015340005CBBA876373A700AA87C207C183BA869B
:101544006373E400A286C206C182958F5147635932
:10155400F7008327090391C38297EF40516882A45F
:10156400B2402244924402494101828082800111A6
:10157400B737002022CC3734002023A007889307F4
:1015840084829C5B06CEAA851304848281C72AC602
:101594008297B245C9C19C410545B5CBDC41A5CB79
:1015A4009E25B5C7BE25A5C7DC2589CB5C3813F7B6
:1015B40037008983BA970947634BF704373500200E
:1015C40041461305058797F0FA1FE78080D6B737A1
:1015D400002083A6078737370020232ED78078384A
:1015E4000DE3938707878A279307805737460F00B1
:1015F4003305F5021306062481468145EFC06123B5
:1016040068B8371505001305E53825360145F2405D
:10161400624405618280B72700209387877D37174E
:10162400002023AE070013076798B737002023A8CC
:10163400E7863787320093870787FD56130727A16C
:10164400D4C398C723860700B747024023A4D726EC
:10165400BDBF011122CC3734002093078482884710
:1016640006CE26CA4AC801E90545F2406244D2447E
:10167400424905618280130484821C5CF5D7585C5E
:1016840065D77000854582971844B247E30EF7FC8E
:101694004A249305E004B724002097F0FA1FE7805A
:1016A400209A1387847D08D39384847D55DD522446
:1016B4009305F00F014997F0FA1FE78020CE7C24B0
:1016C4009050634DF900328597F0FA1FE78040A4EB
:1016D400014523A0040223A2040241BF4E2408446E
:1016E400585CB3872503898105093E9508C2029792
:1016F400F9B701114EC6B7390020938789829C47F8
:1017040026CA4AC852C406CE22CC56C25AC02A8A15
:10171400AE8432896388071E9389898203A789036B
:10172400630207121307F01F6360A7123724002017
:101734001307847D832A07021304847D63980A08AF
:1017440003D5C9009565938515E097F0FA1FE780E6
:10175400208F08D02A867DC583D5C90083A7890335
:1017640003A589008981829783A78900832A0402BB
:101774005CD089476314FA08C1476395F40C83D598
:10178400C9009147938505FCB3C5F5028A05D69532
:10179400B8219307A0056313F70A9E216390470BB2
:1017A4004A852686910597F0FA1FE78080B81C5079
:1017B4005685639157130145F2406244D24442492D
:1017C400B249224A924A024B056182805850E38210
:1017D400E7FA03D5C9009565938525E097F0FA1FCC
:1017E400E7800086AA8A39CD83D5C9002A8683A7D3
:1017F400890303A5890089818297A5BF8D47631B4F
:10180400FA00C1476390F40483D5C900938545FD6C
:10181400F199B5BF91476318FA006395440383D5E2
:10182400C900A115F5B793070010631DFA00A1477D
:1018340063EA970083D5C900C115D9BF1C505685EA
:10184400639D570B29458DBF9D6A637A5509930A99
:1018540005E01947B3CAEA0203D7C900372B0020B1
:10186400B38AEA02BE9A93078B7DDC53130B8B7DFC
:101874006395570103240B021DE003D5C9009305AA
:10188400E00497E0FA1FE780A07B2A8445DD83D536
:10189400C90083A789032A86898156858297914541
:1018A4001307A005898193972500A297B423639118
:1018B400E6049623639C460385058A052686A2953D
:1018C4004A8597F0FA1FE780C0A683270B02E384BA
:1018D40087EE228597F0FA1FE7808083E9BD2167B0
:1018E4007917E361A7F6B30A5541BDB7AC335DBFC1
:1018F40083270B02E38887F4228597F0FA1FE78099
:10190400208189B7B727002083A5877F85DD91478C
:101914009306A0058983139727002E973023E3139A
:10192400D6F21223631C460185078A072686BE95D4
:101934004A8597F0FA1FE780C09FB5BD3C33D9BFF5
:10194400B737002093878782984721C3D85F15CF84
:101954008546631CD502411122C437240020130498
:10196400847D105006C611CECE2748508981029737
:10197400085097E0FA1FE780A0792320040223226D
:101984000402B2402244410182808280011122CCAF
:10199400373400209307848256C283AA870026CA5C
:1019A4004AC84EC606CE52C42A89AE84B2891304EC
:1019B4008482638D0A1A5C5C99EB2945F240624487
:1019C400D2444249B249224A924A056182801C5C4F
:1019D400EDD79307F01F63E1A70C372A0020930784
:1019E4008A7D9C53130A8A7DA9C7084483274A0227
:1019F400639CA70489476313F906C147E39FF4FA7C
:101A04004A249147130505FC3345F5029317250035
:101A140003250A022686CE853E959307A0053CA1A0
:101A240023102501110597F0FA1FE78080900145E6
:101A340071B74A249305E00497E0FA1FE7804060F9
:101A44002320AA025DF195BF4E241C5C03260A02E2
:101A5400898182971C442322FA0269BF8D47631B44
:101A6400F900C147E39BF4F44A24130545FD937739
:101A7400C5FF79BF91476317F900E39024F54A2421
:101A84002115F5B793070010E319F9F2A147E3E62E
:101A940097F24A244115E1BF9D676375F5069307E4
:101AA40005E01947B3C7E7025A24372A0020B38751
:101AB400E702BE9A93078A7D9C53130A8A7DB1CBB1
:101AC40083274A026392570703250A0291461308A3
:101AD400A0059305F00F93D72600139727002A97A4
:101AE40030236312060783580700303363992805AF
:101AF400B306D64063C4960485078A072686CE8536
:101B04003E9515B721677917E369A7EAB307F5404E
:101B140061BF4A249305E00497E0FA1FE78040522E
:101B24002320AA0251FD51BD4E241C5C03260A0247
:101B340089815685829723225A0379B70EA3931677
:101B44000601C18249BF5224B3859600910513064C
:101B540006FCE3F4C5E613863400719A1106B296C6
:101B6400230107012310270134B379B7372A002052
:101B740093078A7D9C53130A8A7D95CF03250A0215
:101B840091461308A0059305F00F93D726001397E9
:101B940027002A9730236310060583580700303343
:101BA40063972801B306D640E3D896F40EA39316A0
:101BB4000601C182D9BF68245E249305E00433057D
:101BC400F5024205418197E0FA1FE7806047232030
:101BD400AA024DF5DDB352246C24B385C5023386C5
:101BE40096001106E3EBC5DCBDB7014582809C215C
:101BF4001CA1BE211CB1BE21A1833CA1DC213CB1AE
:101C040011458280B727002023AE0754B727002050
:101C140023AC075482800DCD411126C206C622C4CE
:101C2400AA8401458DC12E84B7E50600228541466C
:101C34009385C5C897E0FA1FE780A06F9C200545EF
:101C44005CA49C305CB4B240224492444101828042
:101C540001458280011122CC26CA06CE0947AA84F6
:101C640032846381E50441468147639BC500638FE9
:101C7400E6006397B6000DA841478147638EE600EE
:101C8400F2406244D2443E85056182808A85228581
:101C9400593741468A8519A88A85B53F41468A85C0
:101CA400228531A0E39AB6FC2E86A285268597E08C
:101CB400FA1FE7800079AA87E1B7B727002023AC91
:101CC400A7548280B727002023AEA7548280011135
:101CD40022CC622106CE26CA4AC84EC62DCC832900
:101CE4008500AE842A8803C9090081471317890136
:101CF400618763550702B147054563F787045114AB
:101D0400420403552800418033878900A2864E8609
:101D14008545EFA02021B337A00085077D14135516
:101D24006900420405891379F90341809CA088B0B5
:101D340023812401C2A0014719C01387190098C444
:101D440009476383E7000145F2406244D2444249B3
:101D5400B249056182800545C5BFC167F917630AA9
:101D6400F502D94763F7B702011122CC2EC606CE7D
:101D74002A84EF705028B2456368B5002285624416
:101D8400F24005616F90E019F24062440545056137
:101D9400828005458280C167F9176314F5006F706E
:101DA4009025411106C6EF90400611E15D45B24011
:101DB400410182809147639DF5001C211CA23C21B6
:101DC4001831A207D98F3EA23C3101455CA2828022
:101DD400114582804111814522C426C206C6AA84C7
:101DE400BD232A8409E9B727002083A7875581C723
:101DF400F945268582972285B240224492444101C6
:101E0400828039714ED656D25AD006DE22DC26DACA
:101E14004AD852D4AA8A2E8BB28951EB36C6A53F32
:101E24009145EF70F02BAA844D493DC5B246054A51
:101E3400238034010544630A0B00B685138514001E
:101E4400029B0505131405014180E20993D98941D8
:101E540063D30902C1455685EF908009654915E5AC
:101E640033868400A2852685EF90905D2A8911ED42
:101E740031044204418091472C085685FC8426CEC7
:101E8400E085EF8050222A8901C963070A0026856C
:101E940097E0FA1FE780C027F25062544A85D25473
:101EA4004259B259225A925A025B21618280BA8401
:101EB400014ABDBF011122CC26CA4AC84EC606CE6D
:101EC4002A893284B689353FAA840DE1B7270020D8
:101ED40083A7C75581CF05476317E40003C40900EE
:101EE40005041374F40FA2854A858297F240624474
:101EF40026854249D244B24905618280AE86B7251F
:101F0400050001470546938525BF6DB79E211CA199
:101F14009E21A1831CB1094582809E211CA19E2182
:101F2400A1831CB1BE213CA1BE21A1833CB11145BA
:101F340082809E211CA19E21A1831CB1BE213CA1B3
:101F4400BE21A1833CB1DC315CA1FC215CB18A25BA
:101F540019054205418182809E211CA19E21A183F5
:101F64001CB1094582809E211CA19E21A1831CB124
:101F7400BE213CA1BE21A1833CB111458280CA216E
:101F840006054205418182809E211CA19E21A183D8
:101F94001CB1AA2109054205418182809E211CA110
:101FA4009E21A1831CB1BE213CA1BE21A1833CB1D1
:101FB400CA2111054205418182809C211CA105454D
:101FC40082809E21411122C406C61CA19E212E841A
:101FD4001105A183A30EF5FEBE219505230FF5FE81
:101FE40083D7D5FFA183A30FF5FE03C6F5FF97E0C2
:101FF400FA1FE78000344820B24022441105410111
:10200400828089476399F5001C3118210145A20794
:10201400D98F1EA28280114582809A21D94763FDFF
:10202400E702011122CC06CE2EC62A84EF70A07CD2
:10203400B2469E22636DF50022856244F240B725C4
:10204400050001470946938505F105615DBBF24032
:10205400624409450561828009458280914785C5AE
:102064001421FD15C2058547C1816390F60213D77B
:1020740025008D89914781E9914711C7050534A24F
:102084001AA248C281473E85828009479147E39C52
:10209400E6FEC94733D7F502B3F5F502E1BFAE86D4
:1020A400B7250500014711469385E5F199BB93F7E0
:1020B400350089EB8981914781C50EA248C28147C9
:1020C4003E8582809147EDBFD8218947631CF70282
:1020D400011122CC2A84C84506CEAE86014709C91F
:1020E4002EC69D4597E0FA1FE780C00FB2462A87A7
:1020F40022856244F240B72505001946938565F3AD
:10210400056101B30945828099E1114582801C2152
:1021140005473EA2E37BF7FEFD1593F5F50F33D794
:10212400F502B387E702E392F5FE050548C21AA259
:1021340001458280DC210947AE866385E70041477B
:102144006399E700B725050001472146938565FC9F
:102154004DB9094582800EA291E1014548C201456D
:102164008280AE86B7250500014729469385C5F5CB
:1021740049B90EA291E1014548C201458280AE866B
:10218400B7250500014731469385A5F69DB90EA2F2
:1021940091E1014548C201458280DA21854763FF08
:1021A400E702011122CC2A84884106CE1DC12EC625
:1021B400854597E0FA1FE780E0022A87228562447A
:1021C400B246F240B72505003946938525F80561E6
:1021D4000DB9F24062440945056182800945828057
:1021E400914785C518218D46914763F0E602FD1598
:1021F400C205C181B3C6E5023308D702639705015E
:10220400050516A23AA248C281473E858280DC2198
:102214000947AE866385E70041476399E700B72520
:10222400050001474146938565FCE1BE094582806E
:10223400B335B000139525008280011122CC26CA43
:1022440006CE98258547AA842E844946631FF70045
:1022540099363E2049151306200963C8A700F240A9
:102264006244D24409450561828018348547631469
:10227400F70013660604484001C98D4532C697E04D
:10228400FA1FE78020F63246A2866244F2402A878B
:102294002685D244B72505009385C5F8056195B612
:1022A4008D4763F8B7021C311821F115A207D98FA5
:1022B4001EA23C313821C205A207C181D98F3EA29A
:1022C4004EA289C5110508C6014582802324060053
:1022D400E5BF11458280011122CC2A84884506CEAF
:1022E400AE8601C92EC6954597E0FA1FE78080EFB8
:1022F400B2462A8722856244F240B7250500594632
:10230400938505FA0561F5BCB335B0001395250036
:102314008280AE86B7250500014761469385E5FBBB
:10232400CDB48547114563F0D7021C320C22A207B5
:10233400CD8F1EA39387E6FF3EA389476386F600ED
:10234400090650C30145828023220700E5BF0147E7
:1023540081467946814575B49E211CA19E21A183A5
:102364001CB109458280BC2105471CA18A216397C1
:10237400E7000A050505420541818280C947330506
:10238400F502CDBF8A210A05420541818280BE2122
:102394001CA18A21BE213305F502050542054181B0
:1023A40082808A2182808A2182808A218280BE2141
:1023B4001CA18A21BE213305F50205054205418190
:1023C40082809E211CA19E21A1831CB1BE213CA11F
:1023D400BE21A1833CB1CA211105420541818280FD
:1023E4009E211CA19E21A1831CB1AA21090542059D
:1023F40041818280894711456398F6001C3214227A
:102404000145A207D58F1EA382809A21D947AE86A3
:1024140063F9E700B725050001470D469385C535E7
:1024240051BC094582801145639DA6001C321422CB
:102434000145A207D58F1EA33C323422A207D58FB3
:102444003EA38280BC210547FD1793F7F70F636114
:10245400F7049E2195CF011122CC2A84C84106CECF
:102464001DC12EC6894597E0FA1FE780A0D72A87A9
:1024740022856244B246F240B7250500154693858D
:10248400A536056105BCF2406244094505618280B8
:10249400094582809547114563F1D706411122C44D
:1024A40026C24AC006C61C32BA841822A207328445
:1024B400D98F9EA03C32382293054400A207D98FBD
:1024C400BEA08947DCA0094613855400368997E0ED
:1024D400FA1FE78000E69307A9FF9EA49947631BB0
:1024E400F90023A60400B240224492440249014563
:1024F400410182801904C0C4FDB782809E2195CF1A
:10250400011122CC2A84C84106CE1DC12EC68545A0
:1025140097E0FA1FE78000CD2A8722856244B246FD
:10252400F240B72505001D4693858538056159B2EB
:10253400F2406244094505618280094582809947D9
:10254400639DF6028947411106C65CA31C3214221E
:10255400B285A207D58F1EA33C3234225023A20792
:10256400D58F130557003EA3910597E0FA1FE78026
:1025740040DCB240014541018280D147114563945A
:10258400F600C147C9B782809E219DCF011122CC9C
:102594002A84C84106CE05C52EC6894597E0FA1F90
:1025A400E78040C42A8722856244B246F240B725B8
:1025B400050025469385253905616FF0BF8FF240EC
:1025C4006244094505618280094582808947114535
:1025D4006398F6001C3214220145A207D58F1EA36E
:1025E4008280011122CC2A84C84106CEAE860147DE
:1025F40009C92EC6854597E0FA1FE780A0BEB246FA
:102604002A8722856244F240B72505002D4693852A
:10261400653A05616FF01F8A1145639DA6001C325F
:1026240014220145A207D58F1EA33C323422A207EF
:10263400D58F3EA38280011122CC2A84C84106CEC4
:10264400AE8601C92EC6854597E0FA1FE78080B99A
:10265400B2462A8722856244F240B72505003546F2
:102664009385A53A05616FF0FF8493F71600114531
:1026740081EB89476386F600858256A310C3014522
:102684008280011122CC2A84C84106CE05C52EC6FB
:10269400854597E0FA1FE780E0B42A8722856244E3
:1026A400B246F240B72505003D469385E53A0561FB
:1026B4006FF05F80F24062440945056182809E218B
:1026C4009DCF011122CC2A84C84106CE05C52EC651
:1026D400894597E0FA1FE780E0B02A8722856244A3
:1026E400B246F240B725050045469385253B056172
:1026F4006FF04FFCF2406244094505618280094550
:102704008280854763F6D70208A70CB71C320C22D7
:10271400A207CD8F1EA39387E6FF3EA38947638656
:10272400F600090650C30145828023220700E5BF55
:1027340011458280014781464D4681456FF08FF7F0
:102744008D47114563F4D7021C320C22A207CD8FAA
:102754001EA33C322C22A207CD8F3EA39387C6FF33
:102764005EA36386A600110610C701458280232458
:102774000700E5BF011122CC2A84884506CEAE8627
:1027840001C92EC6954597E0FA1FE780A0A5B24679
:102794002A8722856244F240B72505005D46938569
:1027A400653C05616FF00FF1854711456395F600AF
:1027B4001C2201451CA38280014781466546814550
:1027C4006FF04FEF011122CC2A84C84106CEAE86A9
:1027D400014709C92EC68D4597E0FA1FE78080A0FE
:1027E400B2462A8722856244F240B72505006D4629
:1027F4009385453E05616FF0CFE0011122CC2A8418
:10280400C84106CEAE86014709C92EC68D4597E05C
:10281400FA1FE780209DB2462A8722856244F2404F
:10282400B725050075469385453E05616FF06FDD5C
:10283400011106CE2EC6EF80605919C5B245F2408B
:102844002A2105616FC0E02EF2404945056182806E
:10285400B7270020A3840758B727002023840758EC
:10286400B727002023A80756B727002023AA075616
:10287400B727002023AC0756B727002023AE0756FE
:10288400B727002023A60756B727002023A40756FE
:10289400B73700202392078A130640389387478A64
:1028A400B2B371761307400B130606B8BAA3D2B3BA
:1028B40011671D46930600059305000A1305007D64
:1028C400DAA3F2B341470546130810F8BAA7DAA70A
:1028D400BAABDAABFAAB9AAF9AB7EEA38EA7F6A768
:1028E40096ABAAAF239E0700239F070023900702FD
:1028F400B2B723960703239707029308F007239898
:1029040007022392E7042393E704239FE704239019
:10291400E7062391E7062392E70623991703130793
:10292400C01CD2BBF2BB239C0702239D0702239E3B
:102934000702239F0702239007042391C7042394CB
:102944000704239507042396C7042397D7042398E1
:10295400D7042399A704239A0704239B0704239CE1
:102964000704239DD704239ED7042393A706239407
:10297400070623950706239607062397B706239889
:10298400B70623990706239AE7067D57239B070674
:102994002390070823910708239207092393E70844
:1029A4008280011126CAAA84214522CC06CE2E8417
:1029B40032C636C43AC297E0FA1FE780C0870DC515
:1029C400A24612473246930700FD1CA1994704B161
:1029D4003CA174A178B152A1AA8522856244F24037
:1029E400D24405616FD0DFE4F2406244D244056111
:1029F4008280B727002023ACA7568280B727002007
:102A040023AEA7568280011122CC4AC806CE26CA1C
:102A14002A890144B30489006368B400F240624423
:102A2400D2444249056182802EC6EFD07FFA9317C3
:102A34000501C183A183B2459CA09307140093F7B9
:102A4400F70F850463F8B700CA97090488A31374C1
:102A5400F40FC9B73E84C9B7411122C437340020EA
:102A6400130444886A20C16706C6FD17630EF50087
:102A7400B737002003C6C79CB725002093850558A7
:102A8400EF800018FD577EA0B240224441018280AD
:102A940009C925151375F50F1335850E1345150052
:102AA40082800145828023900500C1C6797122D4B9
:102AB40026D24ECE52CC5AC806D64AD056CA5EC684
:102AC4003684328AAE892A8B814463F24407B30781
:102AD40094009C23138914004209939A070193DA02
:102AE4000A011359090163840A04CA976341FA0469
:102AF400B307240183CB07005E85593F0DC9938733
:102B0400FAFF2390F90063906B03130519002295D3
:102B1400B250225492540259F249624AD24A424B68
:102B2400B24B45618280D694C204C18079BF01450D
:102B3400C5B701458280011122CC3734002026CA52
:102B44004AC84EC69307448806CE2E89D0CB8CCB78
:102B5400C8C7AA8441469305F00F4A8597E0FA1F37
:102B6400E780C095854913044488631935030848F0
:102B7400C145513D41469305F00F268597E0FA1F64
:102B8400E780C09305496315250348446244F24035
:102B9400D2444249B249C1450561B5B54146814572
:102BA4004A8597E0FA1FE7806091E31535FDC1B7C8
:102BB40041468145268597E0FA1FE7802090E30689
:102BC40025FDF2406244D2444249B2490561828003
:102BD400411122C43734002026C24AC0AE842A8957
:102BE4001306000281451305448806C697D0FA1FD0
:102BF400E780C07A93074488A3812701B737002070
:102C04002388979CEFB03075854719C181474945A2
:102C14002302F488B2402244924402494101828052
:102C2400814791C909C985476319F500DC3193E7E8
:102C340007FCDCB185473E85828089476316F50031
:102C4400DC3193F7F703F5B70D478547E315E5FE48
:102C5400D8311377F70313670704D8B1E9BF814765
:102C640085C119CDD8319306000C85471377070C1D
:102C74006308D700930600048D476303D700894790
:102C84003E858280411122C4005D06C626C21DC84D
:102C9400AA84085009C597D0FA1FE78060474850B6
:102CA40009C597D0FA1FE780A046085409C597D0F4
:102CB400FA1FE780E045228597D0FA1FE780404558
:102CC40023AC0402B240224492444101828019E9B7
:102CD400B737002083C7678891C7372500201305BD
:102CE40005568280373500201305C5898280B737A1
:102CF400002003C567888280B737002003A50789B1
:102D04008280B737002003A547898280B737002027
:102D140083A7878988438280B737002093874788B1
:102D2400D44B9842050798C2A8339307F00F630564
:102D3400F50091656FD0FFE38280011122CC06CEAD
:102D44002E8432C6EF8020199147B2456310F502F4
:102D5400B727002083A7C75795C303A30700630FB2
:102D6400030022856244F24005610283B7270020F4
:102D740083A7475781C703A34700D5B7F2406244EE
:102D8400054505618280011122CC2A844A2106CEA0
:102D940026CA4AC84EC697E0FA1FE780A0CF2DC5C1
:102DA4002A8904218349C500F13D4A85EF80E0501A
:102DB4004A20EF80800D3729002013098958834762
:102DC4000900B9C763969704B727002083C59758AD
:102DD4002685B93C19E1230009004A20EF80A00FA1
:102DE4009147631CF500B737002093874788562026
:102DF400FA236394E6007D57FAA3F2406244D24476
:102E04004249B2490561828081499304F00F65B754
:102E14009307F00FE383F4FC7420522028204E879C
:102E2400A68541365DBF79715EC6AA8B2E8552CCCC
:102E340056CA5AC806D622D426D24AD04ECEAE8A14
:102E4400328B368A97E0FA1FE780C0C47DC1045DE7
:102E54002A89E5C09C50614599C3130540039C54DD
:102E640081C751054205418163050A007105420588
:102E74004181DC5081C75D054205418197D0FA1F2D
:102E8400E780603B2A8455C56146814597D0FA1F87
:102E9400E780C050B737002083C9478D6394090089
:102EA40083490900930700FD1CA0A947A3007401EE
:102EB4003CA0230364018C502312540113058401A4
:102EC40091C908C47146930A440397D0FA1FE78056
:102ED400404656858C5491C948C45146930A4501CD
:102EE40097D0FA1FE780E0445685630C0A0008C8AF
:102EF4007146D285930AC50197D0FA1FE7806043D3
:102F04005685CC5099C548C85D4697D0FA1FE780CE
:102F14004042A2854E85EFD0BF912254B2509254C4
:102F2400F249624AD24A424BB24B4A850259456140
:102F340091BBB250225492540259F249624AD24A85
:102F4400424BB24B4561828001114EC6AA892E853F
:102F54004AC806CE22CC26CA2E8997E0FA1FE780FB
:102F640060B339C5B737002083C4478D91E004218D
:102F7400194597D0FA1FE780002C2A8415C981458A
:102F8400194697D0FA1FE7806041930700FD1CA003
:102F9400B947A30034013CA023122401A285624452
:102FA400F2404249B2492685D24405616FD05F8818
:102FB400F2406244D2444249B24905618280397187
:102FC4005ECEAA8B2E8526DA4ED652D456D25AD04D
:102FD40006DE22DC4AD8AE84328BB68A3A8ABE89AF
:102FE40042C697E0FA1FE780E0AA39C92A89414519
:102FF40097D0FA1FE78020242A8439C141468145AD
:1030040097D0FA1FE7808039B737002003C5478D72
:1030140019E103450900930700FD1CA0BD473CA02E
:10302400B247A300740146A023046401A30454011D
:1030340023054401A30534015CC4A285EFD04FFFEE
:10304400F2506254D2544259B259225A925A025BF3
:10305400F24B21618280797126D2AA8439454AD003
:103064004ECE06D622D42EC6B289368997D0FA1F00
:10307400E780601C0DCDB2459307000D1EA1B1473A
:103084002A844EA13CA1CE851905194697D0FA1F72
:10309400E780202A23062401A2852254B250025933
:1030A400F24913F5F40F925445616FD06FF8B250A2
:1030B400225492540259F24945618280411126C238
:1030C400B734002093844488B83006C622C44AC06A
:1030D4009307F00F6308F7042A89394597D0FA1F3C
:1030E400E78060152A841DCD930700FDB7350020C5
:1030F4001CA1A3002501230105009385C5890D05A5
:10310400194697D0FA1FE780C0229E24A285A830D2
:103114003EA49C305CA42244B24092440249410142
:103124006FD00FF1B240224492440249410182809F
:1031340001115AC02A8B314526CA4EC652C456C202
:1031440006CE22CC4AC8AE84B28A368ABA8997D0CF
:10315400FA1FE780400E2DCD2A84268597E0FA1FBA
:10316400E780409309C55825A1476311F704B73791
:10317400002003C97788930700FD1CA09D47A30086
:1031840064013CA046A023135401231444012315D5
:103194003401A2856244F240D244B249224A924A9E
:1031A400024B4A85424905616FD08FE8B73700204A
:1031B40003C9179DE3110BFCB727002083A70763FE
:1031C4009C47D5DBCE865286D6852685829765B701
:1031D400F2406244D2444249B249224A924A024BE2
:1031E40005618280011122CC2A84214506CE2EC697
:1031F40097D0FA1FE780200415C5B245930700FD58
:103204001CA1C5473CA1BC313CB1DE215EA1FC211F
:103214007CA1FC31AA857CB122856244F24005611F
:103224006FD00FE1F24062440561828001114AC807
:103234002A89614526CA4EC606CE22CCAE89B284FE
:1032440097D0FA1FE78020FF25C1930700FD1CA13A
:10325400BC302A84938584001CB195473CA1FC3082
:1032640011051946A30FF5FE97D0FA1FE780600CED
:10327400DE2023063401A2853EA4BE2C4A857EA40A
:10328400DE2C1EA8FE2C3EA883C704025CA883C7BC
:1032940014025CB8BE30F240D2447EA86244424973
:1032A400B24905616FD0CFD8F2406244D24442495A
:1032B400B24905618280411122C4373400201304CD
:1032C40044883C2006C626C285CBB7240020AA85A4
:1032D40019461385045697D0FA1FE78080052820E5
:1032E40093850456EFF0DF932244B24013850456CD
:1032F400924441016FB0F006B24022449244014529
:1033040041018280411126C2B7340020938744884A
:1033140006C622C44AC0B8339307F00F9384448886
:103324006301F7042A89294597D0FA1FE780A0F0A2
:103334002A8405C9930700FD1CA1A147A300250108
:103344003CA1BC20B7250020938505563CB1194605
:10335400110597D0FA1FE780C0FDA830A285EFD0F1
:103364002FCDB8208D476311F702B727002083A71C
:10337400875799CB03A38700630803002244B24014
:103384009244024941010283B240224492440249D8
:1033940041018280797122D406D626D24AD04ECEFB
:1033A40052CC56CA09444DCD2A890A21AE895144CA
:1033B40097D0FA1FE780006EAA845DC137370020DA
:1033C4009307C79CDC238546BA8AFD1793F7F70F4A
:1033D400494463F7F6085825A1476314F70063913D
:1033E40009089C5C4544ADEF9165938545711305CF
:1033F400C00297D0FA1FE780A0C488DC2A8A4D4413
:1034040025C11306C002814597D0FA1FE78000F951
:103414008357090093064A0036852311FA00714642
:103424009305490036C697D0FA1FE78080F0894794
:103434002300FA00C824B2460356090083C5CA9C77
:10344400611513351500EF8090212A8463860900E5
:10345400CE852685EF80401401C42685EFF09F8237
:103464002285B250225492540259F249624AD24AF5
:1034740045618280B737002083C7079D0547FD1744
:1034840093F7F70F6377F708894749C6011122CCF0
:1034940026CA4AC84EC652C406CEAA89368AB284FF
:1034A4002E8997D0FA1FE780E05E2A84D14731C580
:1034B400485509C597D0FA1FE78080C5F145268590
:1034C40097D0FA1FE78020F348D4CD471DC5542474
:1034D40021478147639DE600630B0A00382D1229BA
:1034E40093062501AA854E85EF806011AA8758208E
:1034F400630E09001367670058A0F2406244D24487
:103504004249B249224A3E850561828013674700D9
:10351400E5B7C9473E8582809307200463EAA70084
:10352400B73700209387478A06053E950A21828093
:1035340041657D158280011122CC2A842E8526CAFC
:1035440006CEAE8497D0FA1FE780C0540DCDB7479E
:103554000F009387F723094563E2870281450A85B3
:10356400414697D0FA1FE78060E3A68560800A850C
:1035740041804081A3010100EF80E07AF24062447F
:10358400D244056182804945D5BFB73700202387DF
:10359400A79C82806F801007797152CC2A8A328569
:1035A40022D426D24AD04ECE56CA5AC85EC606D6B1
:1035B40062C4AE8BB28A368BBA843E89C289468491
:1035C40097D0FA1FE780004D0DC92A8C63130A02B5
:1035D40013774B005C2115CF93E727012302FC00EE
:1035E4008DEC631C0902639A090205E8ED9B230232
:1035F400FC00832B8C0363910B08B2502254925429
:103604000259F249624AD24A424BB24B224C4561BA
:103614008280F59B93E70701D1B793E74700230224
:10362400FC0001CC1C484146A2852324FC0213055E
:103634008C0197D0FA1FE780C0CF63930B02D5D8D3
:103644000325CC0209C597D0FA1FE78060ACF14589
:10365400268597D0FA1FE78000DA2326AC0251BFF3
:10366400E30909F80325CC0209C597D0FA1FE780BE
:1036740020AAF1454A85F1BF9DC483A70B0299EBAB
:10368400916593853571714597D0FA1FE780409B0A
:1036940023A0AB0203A50B0219C57146A68597D0DA
:1036A400FA1FE78000C96388090283A74B0299EBDC
:1036B4009165938525715D4597D0FA1FE780409801
:1036C40023A2AB0203A54B0219C55D46CE8597D054
:1036D400FA1FE78000C61DC483A78B0299EB91658E
:1036E40093851571514597D0FA1FE780609523A4FF
:1036F400AB0203A58B0219C55146A28597D0FA1FC8
:10370400E78020C32254B2509254F249B24B224C67
:10371400CA865A860259424BD6855285D24A624A93
:1037240045616FF04FF0011126CA52C406CE22CC77
:103734004AC84EC62A8AAE8497D0FA1FE7808035DD
:1037440035C1AA89394597D0FA1FE780C0AE2A84CB
:1037540031C9B737002003C9478D6314090003C971
:1037640009009307000D1EA0AD473CA09385690096
:1037740013053400194697D0FA1FE78080BB93F7EE
:103784001400858085885CA444B423154401A28573
:103794006244F240D244B249224A4A854249056110
:1037A4006FD00F89F2406244D2444249B249224A5E
:1037B4000561828001114EC652C456C206CE22CC87
:1037C40026CA4AC8AA8A2E8AB28997D0FA1FE780E5
:1037D400602C2DCD2A891305C00297D0FA1FE780EB
:1037E40080A52A8425C5B737002083C4478D99E076
:1037F400834409009307000D1EA0E9473CA09305EC
:10380400690013053400194697D0FA1FE78060B2A7
:10381400D285231554011305C400414697D0FA1FDD
:10382400E78020B1CE851305C401414697D0FA1F25
:10383400E78020B0A2856244F2404249B249224A5C
:10384400924A2685D24405616FC09FFEF2406244CD
:10385400D2444249B249224A924A056182804111C6
:1038640022C43724002013048456084006C619C510
:1038740097D0FA1FE780C08923200400B240224475
:1038840041018280011106CE22CC26CA4AC82EC626
:1038940097D0FA1FE780002031CDB245B73700201A
:1038A40003C9478D0CD5AA84631409000349050094
:1038B400414597D0FA1FE78000982A8405CD9307E5
:1038C400000D1EA1A5473CA1DC30938564001105C1
:1038D400A30FF5FE194697D0FA1FE78080A59C54E4
:1038E400A285F2405CC46244D2444A8542490561DF
:1038F4006FC01FF4F2406244D244424905618280A1
:103904001D71A2CC86CE2A842EC697D0FA1FE780DA
:10391400601815C954251147AA8749456391E602E1
:103924009C5FB24591C3EC2BB7D605002308B100C8
:103934009386C6CF100889452285EF70103DF64066
:103944006644256182805145DDBFB737002083C7B7
:10395400079D0547FD1793F7F70F637AF704894727
:1039640021CA411122C426C24AC006C6B2842E8985
:1039740097D0FA1FE78000122A84D14715C1630645
:1039840009005C2193E727005CA14146A685130545
:10399400840197D0FA1FE780C0999C481CD48147C2
:1039A400B2402244924402493E8541018280C94783
:1039B4003E858280797122D406D62A842EC697D079
:1039C400FA1FE780200D01CDB2452285230EB100F8
:1039D4006C08EF701039B250225445618280514511
:1039E400DDBF6F702044C1671387E7FF6395E5026D
:1039F400B727002083A7475791EB49458280494563
:103A0400B2402244924402494101828003A3070048
:103A1400E30503FE0283411122C426C24AC006C63E
:103A2400FD172A892E84B284639AF502B7270020F1
:103A340083A7475791CF9C4381CF829711E9B7273A
:103A4400002023842759B7270020A38497584DBF0B
:103A5400A6854A85EFE0DFDD45F5D5B72E8597D0FD
:103A6400FA1FE780200341DD1C210D45E39A27F965
:103A740022852244B2400249A685924441016FB096
:103A8400400B9307200463E1A7064111C16722C4D8
:103A940006C626C2FD172A8409456381F502C54777
:103AA400AE846312F4022E85EFB0E00F37350020A8
:103AB4001305458A06042A9406A00145B24022440F
:103AC4009244410182809307A0036316F4002E857B
:103AD400EFB0E006E1BF9307B003E319F4FC13F57C
:103AE400F50FEFB00006D9B709458280011106CE63
:103AF4002AC6EFE0FFD5EF10401BEF900175B737F2
:103B0400002093874788130700F0BAA32382070095
:103B1400B737002032451387C79CFD5634A3F240C3
:103B24002386A79C954505616F5030567571939710
:103B3400050126C306C722C54AC1CEDED2DCD6DAC9
:103B4400DAD8DED6E2D4E6D2EAD0EECEC187AE84AD
:103B540063D00756373400200345C49C373900200E
:103B6400372A002097C0FA1FE7804072AA8C22CC23
:103B7400B72A0020372B0020372D00201304498852
:103B8400372C002063930C022165258DBA402A440A
:103B94009A440A49F659665AD65A465BB65B265C7D
:103BA400965C065DF64D4961828083C70C0013075D
:103BB400200A639CE7008349340003D52C00C165C7
:103BC4006686FD15EFF06F9785A262471307C79CC1
:103BD40083492700130710096394E71683C71C0061
:103BE40015476391E7026685EFF0EF996685EFC0AC
:103BF4005FBFE24703C5C79C97C0FA1FE78000690F
:103C0400AA8C49B739476395E71603D54C008567F5
:103C1400A5076316F50483A58C0083CB0500639D7B
:103C24000B00850591C93735002019461305C58950
:103C340097C0FA1FE780E06F0347498885476311FF
:103C4400F71063880B00230209885E85EFF00FC725
:103C540071BF89472302F988EFA0707041BF89675B
:103C6400138727006318E50483AB8C00638A0B0C6D
:103C740083C70B0099EB83C72B0003C71B00A20764
:103C8400D98F1EA483C73B001CB0034749888947CA
:103C94006318F70A83C70B0091C72302098803C579
:103CA4000B006DB70C300A248D472302F988EF50BE
:103CB4009040F5B795076318F50083A78C00882317
:103CC400EFF04FE425B7F9771387A7FF2A97420748
:103CD4004183914663F1E6049387A7FCAA97C20740
:103CE400C18371476371F70289671387B700631053
:103CF400E50483A70A57E38B07EE9C43E685E38735
:103D040007EE829715A0370700181307F770B3570B
:103D1400F700858BA1CB83278A57E38907EC9C4363
:103D2400E38607EC66858297E31205EC11A81387F6
:103D3400C7006310E50283A78C009C23E38807EA8D
:103D44009307F00FE384F9EAE6854E85EFC05FAE92
:103D54004DB5B9076318F50083274C57E38807E886
:103D6400DC4369BF896793871704E304F5F8C9BF87
:103D74003D476398E70403D54C0089671387D70050
:103D8400E30CE5FC13879701E308E5FCCD07E31991
:103D9400F5FA7A20C167FD17631DF70083274C5796
:103DA400E38607E4DC43E38307E40965E6854D0520
:103DB40089BFB727002083A7C757E38907E29C433D
:103DC400DDB71307E003E39DE7F683C72C0005473F
:103DD400639EE71283C76C0037270020930D875634
:103DE4006398071083A70D006381071083CB070036
:103DF400A14903C57C0013878C00BA853ACEEFE055
:103E04001FE6A383AC00130640028145681097C0E7
:103E1400FA1FE780A05883C73C0072471946A307DE
:103E2400F10283C77C00BA854818A309F10297C040
:103E3400FA1FE780005083D74C007010CE852318FA
:103E4400F10283D7EC005E852313F10483D70C01C0
:103E54002314F10483D72C012315F10483C74C01E7
:103E64002306F104FD57A306F104FD572317F104BB
:103E7400EFF0CFBB83C73C0072478DE7DD4783D8A3
:103E84000C0103D8EC0083C67C0083D54C003EC2F1
:103E940083D72C013EC00546CE875E85EF70801A1D
:103EA400A381AC0083A70D0081C71145EFF03F9BB0
:103EB40003458B58930B8B58E30A05D283459D58D1
:103EC400EFE01F97E30405D283C63C009307100379
:103ED400638AF60003D64C0083C50B004E873685F3
:103EE400EFE03FAC23800B0011B3834B340009B7E0
:103EF40083278A57834B34009149E38C07EEDC43D4
:103F0400E38907EE814501458297E5B513079002E1
:103F14006397E70883C76C0037270020930D875603
:103F2400B9EB83A70D00A9C783CB0700A14903C53B
:103F34007C0093772500A1CF058913874C01A383C7
:103F4400AC006686CE855E853ACEEFF02FAE83C791
:103F54003C007247A1FBDD4783D8CC0103D8AC01F8
:103F640083C67C0083D54C003EC283D7EC011DB7C9
:103F7400834B340065BF83278A57834B34009149B0
:103F8400DDD7DC43CDD78145014582974DB71387F3
:103F94008C00BA853ACEEFE09FCC72474DB7094703
:103FA400639CE70083A70A57E38207C4DC43E38FDB
:103FB40007C2668582971DB92D476398E70083A7DA
:103FC4000A57E38507C29C47DDB70D476397E700AF
:103FD40066868D4503D54C00F5B619476395E7060B
:103FE4009305A10213051031EF90012E6C101305F7
:103FF4002031EF90612D03D66C008357C10203D5A5
:104004004C0063E8C70083D68C000357A10263F712
:10401400E60093050002EFA01038C9BE6374E60001
:104024002393EC0063F4D7002394FC0003D7CC0063
:1040340083D6AC0003D68C0083D56C00014881473D
:10404400EFA0303565B61D47E38CE7CE3147639565
:10405400E7006686B145BDBF35476398E70083A78F
:104064000A57E38507B8DC4799B74947639DE700DA
:1040740083278A57E38607CCDC43E38307CC814557
:104084000545829775B94D47639CE70083278A5796
:10409400E38807CADC43E38507CAE6850945D5B743
:1040A40013076002E39EE7C86686930560021DB7A6
:1040B40093F7150089CFB727002083A7075789C72F
:1040C400DC4399C30145829713C51400C1B493F727
:1040D400250091CFB727002083A7875791C7DC43DA
:1040E40081C781450545829713C5240045B493F7DC
:1040F40045000145E38C07A8B727002083A7C756CE
:10410400373400201304448889CF85475CA0B7273F
:10411400002083A7875791C7DC4381C781450545A4
:10412400829748446C10EF70B02C6810EFF0AF9891
:10413400B737002083D7678C81CF1306006433869A
:10414400C702B737002003C5C79C9145EFC05FC0C5
:1041540013C5440025BC411122C437240020032583
:10416400C45606C619C597C0FA1FE78060FA23260D
:104174000456B240224441018280757122C537241D
:1041840000208327C45606C726C34AC1CEDED2DC2C
:10419400D6DADAD8DED6E2D405456389070E93056C
:1041A400F1051305F041EF7091069305F105130530
:1041B400F041EF70D105B737002093874788BC23BF
:1041C4000347F105B337F00011C389070327C45629
:1041D400BEC6283393054700EFE09FA40327C456C7
:1041E400AAC40D452C23AEC2EFF00FB3AAC01145EB
:1041F400EFF08FB20324C4562ADE65453824034CFD
:10420400B4003ADCEFF04FB1AA846945EFF0CFB0C7
:104214002A897145EFF04FB0AA896D45EFF0CFAF11
:104224002A8A7545EFF04FAFAA8A7945EFF0CFAEF1
:104234002A8B13050004EFF02FAEAA8B130510048C
:10424400EFF08FADE2042648B6476257F2560646B1
:1042540096451375F50F93FBFB0F137BFB0F93FA36
:10426400FA0F137AFA0F93F9F90F1379F90FE1841E
:104274002AD05ECE5ACC56CA52C84EC64AC426C2AA
:1042840062C0930844000545EFA0B012BA402A4426
:104294009A440A49F659665AD65A465BB65B265C76
:1042A40049618280011122CC06CE26CA8D472E8414
:1042B400631AF504B831B7340020E947CA2193845E
:1042C40044886315F700FE206389A70497C0FA1F8A
:1042D400E780407C19C17E207EA53A2416247220F2
:1042E4004E202830EFE0DFE45A20FE206309F70077
:1042F4008547F2406244D2443E8505618280FD5781
:10430400FEA0FDB78967CD07631CF500BC213147CA
:104314006385E7004547E39DE7FCEFE0EFF3C9BFA2
:10432400B1476319F500B737002003C5179DEFE0C7
:104334007FEB7DBF41677D178147E31CE5FAD431EC
:104344004947E398E6FACC212A20300023140100DF
:10435400EF60700771BF411122C4372400208347E6
:10436400A45826C206C64AC01307E00FAE8463826F
:10437400E7041307F00F1304A4586384E7021145FC
:1043840097C0FA1FE78020EB09CD930700FD1CA11D
:1043940089473CA1854704B13CB1AA850820EFC0F8
:1043A4002FC9F9571CA0B24022449244024941014A
:1043B40082802A89114597C0FA1FE780C0E765D536
:1043C400930700FD1CA189473CA104B1A301250169
:1043D4002244B7270020B24092440249AA8503C56B
:1043E400B75841016FC0CFC479714AD03729002032
:1043F4008327C95622D406D626D24ECE52CC56CACC
:104404004544C5EBB73400209387C49CDC2349445E
:10441400958BC5C3B72700202E8A9165A385A7581D
:10442400AA8993857571314597C0FA1FE78040C109
:104434002326A9564D4435CD23003501A30005009C
:104444002946D285090597C0FA1FE78080EE8327A5
:10445400C9569146B82363E9E60835E74D47B8A342
:10446400B82313670701B8A3930571001305F0413E
:10447400EF70E1599C83F1E7B737002003C76788E1
:104484008D476310F70CEFE03F872C00EF70407608
:104494002800EFE05FE24545EFF00F88014411C9C1
:1044A400130600643306C50203C5C49C9145EFC0DE
:1044B4003F8A2285B250225492540259F249624AE8
:1044C400D24A4561828085466314D700754741BF4F
:1044D40089466314D700494759B78D466314D700FA
:1044E4004147B5BF5547A5BF9546CA8A630DD70056
:1044F40099466315D7000947B8A331A01D46631236
:10450400C702238107006545EFF00F819307F00789
:10451400E30CF5F403A7CA563C2393E707043CA332
:10452400A1B721466314C7000547F9B725466314AC
:10453400C700B4A3C9BFA9460544E31CD7F6114775
:1045440065BF25392A8435D53931A5B7011126CA65
:10455400B724002083A7C45622CC06CE4AC84944B7
:10456400B9C39C230D446390A70437390020034545
:10457400C99C8945EFC0DFA50345C99CB727002026
:10458400914523960758EFC0BFA483A7C45601479B
:10459400814680B31306F100854785450145DC87D4
:1045A400EFA000662A842285F2406244D244424944
:1045B40005618280011106CE22CC26CA4AC88547ED
:1045C400631AF506372400201304C4581E20B9C703
:1045D400373700200347878831E31307B003636B41
:1045E400F702B734002003C5C49C8945EFC05F9E21
:1045F40012209307006403C5C49C3306F602894560
:10460400EFC00FF523100400F2406244D244424943
:1046140005618280938747FC1EA0FDB7B727002061
:1046240083A7C756F5D36244F240D2444249882353
:10463400056129BFB724002083A7C456F1D73737B3
:1046440000201309C79C83474900918BD5DF894714
:104654006310F5062D452EC697C0FA1FE780A0BD4E
:104664002A845DD1B245930700FD1CA1E547A30050
:1046740005003CA1BC3115051946230FF5FEDC21CC
:104684009505A30FF5FE97C0FA1FE78080CA03457E
:1046940059009307F00F6315F50083A7C4568823C8
:1046A400A2856244F240D244424905616FC04F98EA
:1046B4000345C79C8945EFC0BF916244F240D24490
:1046C4004249B72700202396075805616FF0BFA819
:1046D40049458280B737002083C7079D958B638C3B
:1046E40007129307C01C63FCC70009458280F2408F
:1046F4006244D2444249B249094505618280B727E0
:10470400002083A7C75663880710B7270020938724
:10471400A75803C807001307E00F631EE80E011132
:1047240022CC4AC806CE26CA4EC688A313058600E4
:104734004205368932844181A5C9916593856571A5
:1047440097C0FA1FE780C08FAA8955D1B7240020EB
:1047540003A544599384445909C597C0FA1FE780B7
:10476400209B1385890023A0A9002286814523A0CC
:10477400340197C0FA1FE78060C29C402286CA8534
:10478400884397C0FA1FE780C0BA9C40A286F240D3
:10479400C2A36244D2444249B249984305468D4576
:1047A400054505616FA0404591659385557197C096
:1047B400FA1FE780E088AA891DD9B724002003A541
:1047C400C4599384C45909C597C0FA1FE78040941B
:1047D4001385890023A0A9002286814523A03401E2
:1047E40097C0FA1FE78080BB9C402286CA85884315
:1047F40097C0FA1FE780E0B39C40A286F240C2A3B0
:104804006244D2444249B249984305468D45054520
:1048140005616FA0A03E494582809307C01C63FCDC
:10482400A700094582800945F2406244D2444249C6
:10483400B2490561828055C9011122CC2A8421051F
:104844004EC64205AE8991659385657141814AC81A
:1048540006CE26CA97B0FA1FE780807E2A8961D5E2
:10486400B724002003A544599384445909C597C02B
:10487400FA1FE780E089130589002320A900228616
:10488400814523A0240197C0FA1FE78020B19C40F2
:104894002286CE85884397C0FA1FE78080A99C4072
:1048A400C2A3B727002083A7C75685CFB7370020F8
:1048B40083C7079D958B85CBB727002083A74759CE
:1048C40091CF9843D6236244F240D2444249B2493C
:1048D40005468D45054505616FA0003201478146B7
:1048E400DDB7014591B7494581B7B727002083A7B4
:1048F400C7568DC7B737002083C7079D958B8DC3D7
:10490400B727002083A7475999C79843D62305465C
:104914008D450545D1B701478146D5BF0145828004
:10492400494582809307C01C63FCA7000945828027
:104934000945F2406244D2444249B2490561828049
:1049440055C9011122CC2A8421054EC64205AE89DF
:1049540091659385557141814AC806CE26CA97B0A0
:10496400FA1FE780E06D2A8961D5B724002003A5EA
:10497400C4599384C45909C597B0FA1FE780407994
:10498400130589002320A9002286814523A0240140
:1049940097C0FA1FE78080A09C402286CE8588437A
:1049A40097C0FA1FE780E0989C40C2A3B727002075
:1049B40083A7C75685CFB737002083C7079D958B3C
:1049C40085CBB727002083A7C75991CF9843D62317
:1049D4006244F240D2444249B24905468D450545F8
:1049E40005616FA0A02101478146DDB7014591B75C
:1049F400494581B7B727002083A7C7568DC7B73766
:104A0400002083C7079D958B8DC3B727002083A7FC
:104A1400C75999C79843D62305468D450545D1B74F
:104A240001478146D5BF014582804945828093076D
:104A3400C01C63F4A70009458280797122D44ECE4C
:104A440006D626D24AD0AE892A8425C1210591658D
:104A5400420593857571418197B0FA1FE780405EE6
:104A64002A89094563040908B724002003A5845949
:104A74009384845909C597B0FA1FE78060691305C8
:104A840089002320A9002286814523A0240197C000
:104A9400FA1FE780A0909C402286CE85884397C069
:104AA400FA1FE78000899C40C2A3B727002083A790
:104AB400C756014585CFB737002083C7079D4945B1
:104AC400958B8DC76C001305D030EF80E17FB24722
:104AD400014593F7070F99CBB727002083A7875980
:104AE4008D4505459443D223EFA0C011B250225402
:104AF40092540259F24945618280B727002083A766
:104B0400475989CFD2238C43411106C697C0FA1F57
:104B1400E7802082B24001454101828009458280BC
:104B2400B727002083A7475985C7B727002003A7C5
:104B3400C759894719CF52230C43411106C697B070
:104B4400FA1FE780007FB24081473E8541018280A1
:104B540089473E858280797106D622D426D24AD0EE
:104B64004ECE52CC8D4763FCA7008944B2502254E8
:104B7400268502599254F249624A45618280373946
:104B8400002003474988C144E312F7FE9307F5FF69
:104B94009309498893F7F70F8546AE842A8403CA9C
:104BA40029001309498863EAF6068DE1994528002E
:104BB400EFD07FE5B739002003C5C99C9145230197
:104BC4008900EFC0EFC035E481444DB719468145F3
:104BD400280097B0FA1FE780607C19462C002685D0
:104BE40097C0FA1FE780E08549F119469305F00F55
:104BF400280097B0FA1FE780607A19462C002685B2
:104C040097C0FA1FE780E0832DF11946A685280096
:104C140097B0FA1FE780E07171BFE31DE5F803A5C3
:104C2400C9002C00EF60D07CAA8449D523814901B6
:104C340035BF2800EFE02FE8AA8405ED9305710045
:104C44001305F041EF60B15C8483BDFC8D47E31D27
:104C5400F4F64545EFE05F8C25D9B77718009387C4
:104C640007A03306F50203C5C99C9145EFC0EFAE1A
:104C7400F5BD23014901DDBDB737002083C7079D7A
:104C8400918B8DC33725002041111305055906C6A4
:104C9400EFD0DFD6B240B73700207D572395E788A1
:104CA4004101828001456FD07FD5B72700207D5711
:104CB400A385E758B727002079572385E758B737E6
:104CC400002023860792B727002023960758B7278A
:104CD400002023AA0758B727002023AE0758B72778
:104CE400002023AC075837570500B72700209387C7
:104CF4008763130767EB98C3374705001307875B80
:104D0400D8C3374705001307E71798C7B747050007
:104D1400372700209387872A2328F7588280411158
:104D240026C2B724002083A7C45606C622C49DCB3E
:104D34002A840D4597B0FA1FE780E04FAA8501CD7C
:104D4400930700FD1CA18D4700B13CA183A7C45665
:104D54008823EFB0FFAD19C42244B240924441010C
:104D64006FF06FBFB2402244924441018280797156
:104D740052CC372A00208327CA564AD006D622D4DA
:104D840026D24ECE56CA0149A1C703C91700B7346B
:104D940000208547AA89938444886305F904DC20AC
:104DA40005499DE70D4597B0FA1FE780C048AA85DD
:104DB40009CD930700FD1CA19147A30035013CA137
:104DC4008327CA568823EFB0BFA6EFF0CFB80549B2
:104DD400B25022544A8592540259F249624AD24A44
:104DE40045618280B727002083A74759D28A85E38B
:104DF4000145EFE06FF22A8601CAB737002003C5E8
:104E0400C79C8945EFB0DFF483A7CA56B1A0944389
:104E1400D2239305E1000545EFD0FFC871D91C21C9
:104E2400858BF9D70545EFE02FEF9307B0032A846C
:104E340063FEA702B737002003C5C79C5D6613064F
:104E440006708945EFC06F91B7270020130444FC16
:104E5400239687588327CA56094798B3DC2081C70D
:104E640023820400B5B74E855D3D9DB713060064EB
:104E74003306C50251B7411122C42A840D4506C622
:104E840097B0FA1FE780203B0DC1930700FD1CA1DA
:104E9400CD473CA100B12244B7270020B240AA85E7
:104EA40003C5B75841016FB0BF98B24022444101D5
:104EB400828056210111896706CE22CC26CA138628
:104EC40067002A876398C6001C4701458C23EFF0CE
:104ED4008FC81DA8138687006396C6001C47054526
:104EE4008C23F5B7138697006392C602B727002078
:104EF40083A7C756014595C31847082371E505479D
:104F040098B30545EF903046054501A81386A700E0
:104F1400639AC6001C478823993DF2406244D244F8
:104F24000561828013866703E380C6FA13867703DC
:104F3400E386C6FA13868703639AC6081C4537249A
:104F440000201307E00F84238347A4581304A458B4
:104F5400638BE7021307F00F6384E702114597B0F0
:104F6400FA1FE780402DAA8501CD930700FD1CA1FF
:104F7400894704B13CA1A30105000820EFB05F8B71
:104F8400F9571CA051B7B727002003A7C7563E8482
:104F9400014541D78DE885447D454485EFE0CFD771
:104FA400688613050002EFE02FD78327C456C8850F
:104FB4001307B10084B374001306A10085450545A9
:104FC400EF90104491B72685993B3DBF1386970314
:104FD400E382C6F41386E7036396C6001C450945BD
:104FE4008C23F5B59387F7030145E398F6F21C4744
:104FF40088231DE56C001305D030EF80E12CB24707
:10500400414793F7070FE381E7F09305B1001305D8
:105014006031EF80612B88858545EF90F03EEDB5DA
:10502400993DDDB5B737002083C7079D411106C6FA
:10503400958B99CB3725002013058563EFD07F9B93
:105044004D45B240410182800145EFD09F9A014510
:10505400CDBF9821937625009377D70F99C2936794
:105064002700131885011358884113F7F707635471
:10507400080013E70708937685009377770F99C2A2
:10508400936787001377050293F6F70D19C393E628
:10509400070294A1634508009377A50291C71C22D7
:1050A40093E7C7001CA282807DFD1C22CD9BDDBF3F
:1050B4002D45631B0710882109476313E51001116F
:1050C4004EC6BE89DC4122CC26CA4AC806CE9833D5
:1050D4009C23B68422075D8F42078D6641879387A0
:1050E40036A032842E89630BF70A63C0E7029387E4
:1050F40016A06307F70863CAE70A938606A0630B42
:10510400D70423900400054559A0938766AA630E2B
:10511400F708938786B86301F70A938646A0E312DB
:10512400D7FEDC45C1C321479AA09A2318A29A232B
:10513400218318B2BA2338A2BA23218338B2DA23DE
:1051440058A2DA23218358B2FA2378A2FE23A1833A
:105154007CB22DA8C84597B0FA1FE7800027420506
:1051640041814E86637335012A8692A042064182AC
:105174008325C900228597B0FA1FE780801B39A0D8
:10518400DC459E238AA01CA2A1831CB20145F240E7
:105194006244D2444249B2490561828099479EA043
:1051A4001946F9B723900400D5B785479EA08327F5
:1051B400C9009C231CA0D9BFE1479EA061464DBFF6
:1051C4002390060005458280828083C805008947B4
:1051D400639BF816DC41797122D406D626D24AD0D4
:1051E4004ECE52CC56CA03C817009C232E842208E4
:1051F4003368F80042088D6713580841138327A0C9
:10520400630F68102A8A3A89B684B285634C030115
:10521400138707A0630BE802938717A06301F80ABA
:10522400854711A8138737A06300E80C138767AA82
:105234008D47E317E8FEB250225492540259F249C2
:10524400624AD24A3E8545618280484432C697B05C
:10525400FA1FE7808017420541819D47E36D25FDD4
:10526400B72A0020938A3A5A83C70A00B3099900DF
:10527400B24563D43701B5477DBF48442686C20989
:105284004A9597B0FA1FE780C00A03C60A0048444B
:1052940093D9090105063306364181454E9597B0E9
:1052A400FA1FE780A00FB727002083A7875A99E346
:1052B400814751B79C438145E5DF528525A0AD4721
:1052C400E31B09F6E39916FB1C3214225844A20787
:1052D400D58F1EA3B727002083A7875AF1DB9C43F1
:1052E400E1DB85458297E9B7B727002003C7C75A92
:1052F4008D4731D3AD47E31009F49947E39DF6F6A2
:105304004844194697B0FA1FE780A002B727002047
:1053140083A7875AD1DF9C43C1DF8D4579BFB72767
:10532400002083C547538D47A18991D5AD4701F727
:105334008547E392F6F4182293070008E3EDE6EEBE
:105344005C4498A3B5B785473E858280B727002083
:10535400411123A4075AB727002022C42383075AE4
:105364000944B7270020A3838752B7270020A381CD
:10537400075AB727002023828752B727002023909B
:10538400075AB7270020238A875237250020B727DA
:10539400002021472386075A1946B7270020814554
:1053A4001305055B06C6A38AE75297B0FA1FE78088
:1053B400E0FEB7270020238587523707A000B727D0
:1053C40000209387C7521307070598C33707E803DC
:1053D400D8C3B7270020238387520547B727002067
:1053E400A382E752B7270020238B8752372500205A
:1053F400B7270020238B075A6146B7270020814531
:10540400130585642384875297B0FA1FE78000F957
:10541400B7270020A3848752B7270020A382075A06
:1054240037570500B72700209387474C1307470BCE
:1054340098C3B2402244375705001307E71CD8C36A
:1054440023A407004101828095476302F51A79710C
:1054540022D426D206D64AD04ECE52CCB2842E8442
:1054640063E4A7048947630DF51463EFA7004DC5F2
:105474000547630FE5120945B2502254925402596C
:10548400F249624A456182808D476304F51491476D
:10549400E313F5FEA1476395F5083725002021465F
:1054A400A6851305C5523DAA930720046305F51686
:1054B40063E1A7029D476306F514A147E31DF5FACE
:1054C4008547639FF5041822B7270020A382E75A73
:1054D400F1A8930710086309F51493072008630DD6
:1054E400F51493070008E318F5F88547639AF50265
:1054F400B727002083C7475A1387F7FFB725002033
:105504009385056612072E97920750478820A107B6
:10551400BE95EFF01FB459A89307800F63F4B7004A
:10552400614599BF372A002083464A5AB72700208D
:105534001387076692063697484793890766130AC6
:105544004A5A09C997B0FA1FE78080BCB7270020E0
:10555400A381075A1306140091659385057132855A
:1055640003490A0032C697B0FA1FE78060AD83474B
:105574000A0012094E9992072326A900CE97C8471C
:1055840045D13246814597B0FA1FE78020E1834731
:105594000A002286A6859207CE97C84797B0FA1FBD
:1055A400E78020D9B7270020A381875A0145E9B5B0
:1055B400E398F5F61A22B72700202390E75AFDB79F
:1055C4008547E39FF5F41822B72700202386E75A7E
:1055D400F1BF9947E396F5F4372500201946A685CF
:1055E4001305055B97B0FA1FE780A0D4C1B78547C0
:1055F400639DF5061822B72700200145A382E752D0
:105604008280E147E39EF5F0372500206146A685B8
:1056140013058564C1BF8547E394F5F01822B727C5
:105624000020238AE75259B78547E39BF5EEB72755
:10563400002083C7275AC9B58547E393F5EE0822AE
:1056440093772500E39E07ECB727002083C7D75A3A
:10565400B7250020938505661387F7FF1207920785
:105664002E97A1075047BE956DB5614582804111C3
:10567400AA8706C611472E856386E70A6361F70287
:105684000547638EE706A9C709476381E7080D4705
:105694006384E7088947B2403E85410182801D4703
:1056A400638AE708636AF7001547E395E7FEB727BF
:1056B400002083C75752B9A821476383E70813071B
:1056C4002004E399E7FCB727002083C7475399A038
:1056D400B727002083C7475A13974700B7270020EE
:1056E40093870766BA97CC478947D5D5B727002053
:1056F40003C6375A97B0FA1FE780A0C331A0B72773
:10570400002083D7075A9EA1814771B7B72700208D
:1057140083C7C75A1CA1CDBFB7250020194693855E
:10572400055BC9BFB725002021469385C552EF808C
:105734006149D9BFB72500206146938585645DBF63
:10574400B727002083C7575AF1B7630F0538B72727
:1057540000209387675A98236318073885463728AB
:10576400002094A309479307086698A337E7060027
:1057740013078733D8C337E7060013074730D8C762
:1057840094A7239507007D57630DE534137715001F
:10579400854539C3B7E6060093864631D4CBB72690
:1057A4000020938676520947D4CFB726002098ABC1
:1057B4002382E65A2380E70237E7060005461307EB
:1057C400C73190AF239D0700D8D32384C702239504
:1057D400070223A607028D45137725002DC31397CF
:1057E4004500B7E606003E979386463154C3B72674
:1057F4000020894805469386465254C72300170162
:1058040010A7231507001387150042074183B72605
:1058140000202381E65A1207B7E606003E979386D6
:10582400C63054C38905B72600209386065AC2059C
:105834002300170110A72315070054C7C18113774C
:1058440045002DC313974500B7E606003E9793869F
:10585400463154C3B72600208948054693864653EB
:1058640054C72300170110A7231507001387150039
:1058740042074183B7260020A386E65A1207B7E6FB
:1058840006003E979386463354C38905B726002005
:105894009386C65AC2052300170110A723150700D3
:1058A40054C7C1811377850021CF13974500B7E60C
:1058B40006003E979386463154C3854614A7B726FF
:1058C400002009469386565354C710A32315070096
:1058D40013871500420741831207B7E606003E9777
:1058E4009386063454C3A14614A78905B72600201D
:1058F4009386065BC20510A32315070054C7C18114
:105904001377050129CF13974500B7E606003E97A4
:105914009386463154C3B7260020894805469386AA
:10592400A65254C72300170110A723150700138795
:105934001500420741831207B7E606003E97938697
:10594400063354C38905B72600209386C652C20580
:105954002300170110A72315070054C7C18113772B
:10596400050229CF13974500B7E606003E979386B4
:10597400463154C3B72600208948054693866652AB
:1059840054C72300170110A7231507001387150018
:10599400420741831207B7E606003E979386063115
:1059A40054C38905B726002093865652C2052300A6
:1059B400170110A72315070054C7C18113770504E5
:1059C40029CF13974500B7E606003E9793864631E4
:1059D40054C3B7260020894805469386665354C7A6
:1059E4002300170110A7231507001387150042078A
:1059F40041831207B7E606003E979386C63354C325
:105A04008905B72600209386665BC205230017012B
:105A140010A72315070054C7C1811377050821CFA8
:105A240013974500B7E606003E979386463154C364
:105A3400D14614A7B726002009469386865254C738
:105A440010A323150700138715004207418312078B
:105A5400B7E606003E979386063254C3854614A7DC
:105A64008905B726002093868664C20510A32315F2
:105A7400070054C7C1811375051039C91397450030
:105A8400B7E606003E979386463154C3B7260020F6
:105A9400094505469386965208A310A723150700C7
:105AA40054C713871500420741831207BA9737E793
:105AB400060013070732D8C38905372700201307C8
:105AC400575AC20588A390A723950700D8C7C18158
:105AD400B72600209386464C4146130508666F306E
:105AE400202E130530037DB101458280011106CEBD
:105AF40022CC0546638CC50211460944639EC50247
:105B04003EC63AC436C2EFD0AF8C2A8492462247AE
:105B1400B2471DE13E86BA853685EFD0CF81EFF0DE
:105B24006FD0EFF06F95EF60006739A0EFD04F8A28
:105B34002A8419E1EFF00FCF2285F2406244056117
:105B4400828079714ECEAE896C0022D426D24AD09E
:105B540006D62A89B284EF0090682A840DE1CE85A6
:105B64004A85EFC00FE02A8419E93245B7260500BB
:105B740026879386A6152D468145EF1020002285A1
:105B8400B250225492540259F2494561828079718B
:105B94004ECEAE896C0022D426D24AD006D62A89AB
:105BA400B284EF00D0632A840DE1CE854A85EFC02C
:105BB400CFE82A8419E93245B7260500268793865B
:105BC40046234D468145EF00707B2285B250225416
:105BD40092540259F24945618280397126DAAE84C1
:105BE4004C0022DC4AD84ED652D406DEAA89328929
:105BF400368AEF00D05E2A8421E9A685630D090068
:105C04009E202C007C84BE207C85930720307C86DB
:105C1400930780025C874E85EFC0CFD12A840DE5BF
:105C24005946A6851305A1002304210197A0FA1F54
:105C3400E78020701245B726050052879386C61068
:105C440025462C00EF0090732285F2506254D25402
:105C54004259B259225A21618280797126D2AE8486
:105C64006C0022D44AD04ECE06D6AA893289EF00DF
:105C740010572A840DE1A6854E85EFC04FD02A84A3
:105C840019E93245B72605004A87938666173546D3
:105C9400A685EF00B06E2285B25022549254025968
:105CA400F24945618280BD47638CF50663E9B7021A
:105CB400A5476387F50663EDB7009947638CF50440
:105CC4009D47638FF5049547638CF50401458280F5
:105CD400B5476387F50463E1B704AD47F5B7DD471E
:105CE400638EF50263EAB700C947638BF502D947AF
:105CF4006386F502C547C9BFF5476383F50263E4CC
:105D0400B700ED47D1B793072005638BF5009307E0
:105D1400200D5DBF4845828008418280084582800D
:105D2400484182809307F00F630FF506011126CADC
:105D3400AA841305000222CC4AC84EC652C456C2D5
:105D440006CE3A89B689B28A2E8A97A0FA1FE780CE
:105D5400804E2A844D450DC8930700FB1CA0A30068
:105D640054012311440123023401130584006146C4
:105D740063050902CA8597A0FA1FE780805BA285A4
:105D84002685EFA0FFAA0145F2406244D24442496D
:105D9400B249224A924A05618280814597A0FA1F3E
:105DA400E780C05FE9BF09458280011122CC06CE9D
:105DB4002A844C86D08697B0FA1FE780A0CD05C10F
:105DC4005425B737002021479387C79C639DE6007D
:105DD400E82378009306E0070146A285A137F24044
:105DE40062440561828078009306E0070146A2853B
:105DF400C833EDB7930700643306F6026FB00F8A19
:105E040015C5182185469307270093F7F70F63FFFD
:105E1400F600411122C42A843A8506C6EFB00FA2C7
:105E2400FD571CA0B24022444101828082801A2185
:105E34009307000B6310F7025C214947639AE7005C
:105E4400183985476398E7002A2185456F30501B30
:105E54006D47CDBF828001116C846C0022CC26CAB0
:105E64004AC806CE2A89B6847085EF0050372A8442
:105E74000DE12C004A85EFC08FA22A8419E932452E
:105E8400B726050026879386060615462C00EF00E4
:105E9400F04E2285F2406244D24442490561828038
:105EA4007971930720306C8470857C862C0093076D
:105EB4008002014606D65C870D33B250456182806C
:105EC400C177797185073EC4894726D27C86AE8422
:105ED400930780024C0022D44AD006D62A895C87D4
:105EE400EF00F02F2A840DE12C004A85EFC02FB279
:105EF4002A8419E91245B726050026879386461E8B
:105F040045462C00EF0090472285B250225492540B
:105F1400025945618280B2860546C1B1797126D2A3
:105F2400AE846C0022D44AD04ECE06D6AA893289D9
:105F3400EF00F02A2A840DE1A6854E85EFC0EF8D8F
:105F44002A8419E93245B72605004A8793866600F4
:105F54000D46A685EF0090422285B25022549254F9
:105F64000259F249456182807971930720206C843B
:105F740070857C862C0093078002014606D65C87D8
:105F8400EFF0BFC5B25045618280011122CC06CE2C
:105F94002A842EC632C436C297B0FA1FE78080AF77
:105FA4000DC94825B7370020A1469387C79C1247DF
:105FB4002246B245631AD500E823B2862E86A2850E
:105FC4006244F2400561B9BBB286C8332E86A2850D
:105FD400C5BFF24062440545056182806FF07FB61B
:105FE4006FF03FB66FF07FC76FF03FC779714ECE49
:105FF400AE896C0022D426D24AD006D62A89B2842D
:10600400EF00F01D2A840DE1CE854A85EFC0EF989C
:106014002A8419E93245B72605002687938626196E
:106024003D468145EF0090352285B250225492546A
:106034000259F24945618280B28601466FF0FFB988
:10604400011122CC2E846C0026CA06CEAA84EF004D
:106054001019DD476309F500930710101EA4A285EB
:106064002685EFC08F9DF2406244D2440561828050
:10607400239405009E2599E36FF07FB10945828042
:10608400C5BFB727002003C7E75E854763F8E7026B
:10609400011122CC2E846C0026CA06CEAA84EF00FD
:1060A400101401E9930700101EA4A2852685EFC0F1
:1060B400CF98F2406244D24405618280594582807F
:1060C400B727002023ACA75A8280B727002023AE2D
:1060D400A75A8280011122CC26CA06CE2A84AE8415
:1060E40097B0FA1FE780009BA6852285EFB0FFC614
:1060F40005E92285648697B0FA1FE780A0990DC14F
:106104005425B737002021479387C79C639FE60037
:10611400E82378009306F0070146A285EFF09FC0BC
:10612400F2406244D24405618280C833DDB7011174
:1061340026CA06CEB68422CCDD4663E3B608D94629
:1061440063FFD50AA5466382D50A63EFB604954674
:10615400638DD50899466388D50A054441687D183E
:10616400631706093AC6EFB01FC3330685403247AA
:1061740042064182420441803305C4004205BA8587
:10618400418132C6EF30C075AA8751C199C03246E9
:1061940092A0B30580406244F240D2443E8505613A
:1061A40017A3FA1F67000304C5466380D504C946D4
:1061B4000D44E394D5FAC167FD17E31DF6FA5DB704
:1061C400F5466380D50463E4B600ED46D5B793067F
:1061D40020056388D5029306200DE390D5F8C167A6
:1061E400FD170D446319F600B5BF094485BF930636
:1061F400200DE391D5F8310642064182A5BF15442E
:106204005DBF0D444DBFC167FD171D447DB7F2400E
:106214006244D24405618280011122CC26CA06CE92
:10622400D0212E841307000281469945AA840137A0
:106234002AC621C51E205020930554007C803E2090
:106244007C8189477C82930780025C8397A0FA1F34
:10625400E780200E5C208A8526857C84EFB0DFE60B
:106264002A8411C5324597A0FA1FE78060EA228587
:10627400F2406244D244056182804D44CDBF5D71D9
:1062840086C6A2C4A6C2CAC04EDE89476306F6000B
:10629400C14709446318F6040144A9C52E894C0872
:1062A40032C6B689AA84252F2A84324605EDC177E1
:1062B4008507CA851305D1013ECC230EC10097A0E2
:1062C400FA1FE78000072C082685B9372A8419E9C4
:1062D4005245B72605004E879386260B1D462C088B
:1062E400EF00D0092285B640264496440649F25967
:1062F40061618280797122D436844AD04ECE52CCE8
:10630400B2892E8A3A898146130710022286D9451A
:1063140026D206D6AA84213D2AC621C12286CA8550
:106324006084231241012313310197A0FA1FE780EF
:1063340040004C002685EFB01FFA2A8411C532456F
:1063440097A0FA1FE780C0DC2285B25022549254F1
:106354000259F249624A456182804D44F5B7011100
:1063640022CC26CA06CE4AC8DD472A84AE84638975
:10637400F50281470A206C005C86EFB09FF9054561
:106384006380A4080824B165938505B8EFA0BF868F
:10639400E5473CA0B72705009387C7305CC085A0BC
:1063A40058393149B2863306270318499C4232973B
:1063B4001043E310F6FCDE225223E31CF6FA8C466B
:1063C400084797A0FA1FE780C00745D55C385828CE
:1063D400850793F7F70F5CB863FAE702B3872703DF
:1063E40018480A20BA979847D623B2238E23193720
:1063F40049F10824B165938505B8EFA0CFFF59454D
:10640400F2406244D2444249056182807C289DB7AF
:10641400011122CC26CA06CEDD472A84AE846393BA
:10642400F5060A21EFB03F97522C36285A286D16EC
:106434002A9642064182B307D640C20752ACC183B2
:1064440063F9E7069305C5FF3308F7406358B802BC
:10645400BA96918EC206184C0E280A20C1823E9725
:10646400513D0DE10824B165938505B8EFA0AFF85F
:106474005945F2406244D244056182806D159316F9
:106484000501D1BF81470A206C005C86EFB07FE82C
:106494000545E380A4FE0824B165938505B8EFA003
:1064A4008FF5E5473CA0B72705009387C7305CC04C
:1064B400C1B78547C9BF397126DAAE842C0022DC06
:1064C4004AD84ED606DE2A89B289112B2A8431E5B0
:1064D4004A85EFB05F8CD6206D1563C5A600931670
:1064E4000501C1829844B2208E204A8521352A8430
:1064F4000DE53146A68508082306010097A0FA1F7A
:10650400E78020E3BE202245B72605004E87938608
:10651400462A5D466C00FC8695252285F25062541D
:10652400D2544259B2592161828071B769B77971E5
:1065340026D206D622D44AD04ECE52CC56CA5AC8F7
:106544008944D1C949CA2E842A89BA8A368B328AA7
:10655400EFB07F8493054400814771159A21635DF0
:10656400A708850793F7F70FB105E319FAFE8A85A3
:106574004A85B521AA8425E131453305AA029165EE
:1065840093851570CD4497A0FA1FE78060ABAA8964
:1065940039C131463306CA02A28597A0FA1FE780A3
:1065A40040D91844562032200E204A85A133AA84AB
:1065B40015ED0245B7260500854756879386462A7A
:1065C4005D464C005C824EC423064101A3060100D3
:1065D400230761016523B25022542685025992543F
:1065E400F249624AD24A424B456182804E8597A065
:1065F400FA1FE780E0B1C5B7ED44F1BF79714ECE23
:1066040037E60600AE89C16526D20147AA848946C9
:1066140013068634FD15054522D406D64AD0EF105C
:10662400A078054429C92A891307300281461146F6
:10663400F5452685EFF0BFAF2AC655440DCD8357E7
:10664400A900CE8601467C8491477C8585471CA1A0
:10665400B2472C002685A38007003247FD573CA390
:1066640032473CB3EF10C0692A8411C5324597A064
:10667400FA1FE780E0A92285B250225492540259AD
:10668400F24945618280411106C6EFF0CFE119C598
:10669400B240410117A3FA1F670083A7B24041012A
:1066A4008280011106CE2AC6EFB0CFD53245B72776
:1066B400002023AC075AB727002023AE075A914580
:1066C400B7370020A386A79CEF30201CF240056159
:1066D4006F2070037971939705014AD006D622D4AE
:1066E40026D2C187014963DB070AB737002003C5F7
:1066F400D79C2E8997A0FA1FE78040B92A8441CD00
:1067040018219307000A6315F70885474C08DC85B0
:10671400EFB0EFDBAA8405ED83476101714763762F
:10672400F708138717FE1377F70F9306000263F534
:10673400E608858BCDC7B727002083A7875B9944DC
:1067440099C72A201306B1004C088297AA849C8515
:1067540099C7084409C597A0FA1FE780609B95E094
:106764005247B7070001938707F07D8FB7071200E0
:1067740093870710630EF70003476101ED47631920
:10678400F7002A208545EF30A007CD476388F40041
:106794002285EFA00F85A1673349F900B250225436
:1067A4004A8592540259456182803707301405079F
:1067B4003357F700058B35DF372700200327C75BE6
:1067C40059D70347510141F75C8699472308F100E3
:1067D4002A206C0023170100EFB04FF28DBFB727BA
:1067E400002083A7C75B8DC32A201306B1004C0881
:1067F400829731DDAA8483475101B1FB834761014C
:10680400230891005C86E9B79944F5B7397122DC15
:1068140026DA06DE4AD84ED652D456D25AD0A547E6
:106824002A84B2846398F50E834745021A22835A58
:10683400260085072302F5029307F7FFB387FA02C0
:106844005442C207C183B69703C917009C23542539
:1068540022093369F90085476390F6023307570329
:10686400231006008149014A130B3501931A0701CD
:1068740093DA0A0163EA5905C167FD176303F90A4C
:106884001E286370F90A05094209542413590901A1
:106894002317240105470A209305E400639CE600BE
:1068A4007C85930720307C86930780022314210182
:1068B4005C872C00EFB01F880824B165938505B868
:1068C400EFA06FB35945B9A8B620DC402C28ED16CB
:1068D40013865900C206C1823E965A85EFB08FB71F
:1068E40005C5630B3A01C840B220B3053501529582
:1068F40097A0FA1FE780E0A3BE203E9A9E20420A9A
:10690400135A0A0185079EA0BE20BE99C20993D9D5
:1069140009018DB75822A9476310F702834745023E
:1069240081CF0145F2506254D2544259B259225A8D
:10693400925A025B2161828034281309340137E5BD
:1069440006004A86894513058533EFB0AFB019C1F7
:106954000545C9BF342837E506004A86894513052D
:106964004534EFB02FAF6DF5342837E506004A867D
:1069740089451305C532EFB0EFAD79F9342837E511
:1069840006004A86894513054531EFB0AFAC69F17D
:10699400D820BD47E3EEE7FAA56793874712B3D73C
:1069A400E700858BD5D78347440285072302F40289
:1069B40003D92400D1B5011106CE2EC697A0FA1F23
:1069C400E780A00211C93C25B245138717006395DF
:1069D400E50093F707F83CA5F240056182800111B8
:1069E40006CE2EC697A0FA1FE78020001DC1B2452F
:1069F40091C188C11C251307E00F5D456388E7003A
:106A04001307F00F01456383E7005945F240056120
:106A140082800945E5BF411122C42A84210506C6A6
:106A240026C24AC0EFF0CFBD3C20A51793F7D70F7D
:106A340089EB58248547631EF7041C488144314977
:106A4400A1E3FD57230104001CB42302040213052F
:106A5400C4002244B2409244024961468145410146
:106A640017A3FA1F67008393B38724033E95084551
:106A740009C59790FA1FE780A069850493F4F40F81
:106A84005C280848E3E2F4FE9790FA1FE780406828
:106A94004DBF084C75F975B7411122C4416406C64F
:106AA40026C29307E4FF6301F502AA849DE197A03F
:106AB400FA1FE78080F309E91305F4FF97A0FA1F92
:106AC400E780A0F211C106A1B240224492444101E0
:106AD400828085476391F50497A0FA1FE780E0F070
:106AE4002A847DD1FD571EA11C241307F00F638156
:106AF400E7021307E00F6389E700342008340147F5
:106B04005146A685EFF00FA222853137FD571CA40C
:106B14002305040055BF8947E398F5FA8545EF40FE
:106B2400203D5DF1268597A0FA1FE78000EC2A84BA
:106B340045FD59BF39C118259307F00F630FF702BC
:106B4400011122CC06CE2A8434210E2108350147B6
:106B54005D46EFF02F9D3820E1476318F7000A20C7
:106B64006C0023060100EFB0CFFAF9571CA422856C
:106B74005D35F24062440561828082809307F00FA4
:106B84006306F706011122CC26CA2A844EC6AE84B7
:106B9400B689AA8593068500377505004AC852C48C
:106BA4003A89328A130585B3794606CEEFF08FA46D
:106BB400A3042401230144012322340185C01305C5
:106BC400C4006244F2404249B249224AA685D244F2
:106BD400614605611793FA1F6700A375F24062448A
:106BE400D2444249B249224A056182808280B72751
:106BF40000202382A75C828095476394F50683472F
:106C04004502854685072302F5021E22584230229A
:106C1400FD17C207C1836312D6048A07BA97983353
:106C24009C232207D98F7A2563F5E704411106C610
:106C340022C485075EA52A849305C5000A21EFB006
:106C44000FC60824B165938505B8EF90DFFAB2400A
:106C54002244D9473E8541018280C946B387D70281
:106C640075BF5422294785476396E60003474502CA
:106C740011C381473E8582809D47639BF50483470A
:106C84004502762585072302F5021E225842FD1788
:106C94008A073E971C331823A207D98F014763F252
:106CA400D704411106C622C485072A845EA593052C
:106CB400C5000A21EFF04FD60824B165938505B8C5
:106CC400EF907FF3B240224459473A8541018280D4
:106CD4005422A94705476396F60003474502133734
:106CE40017003A858280411122C406C626C2B547E0
:106CF4002A846395F50483474502B28485072302F9
:106D0400F5020A21EFB02F899E201307F5FF0145F4
:106D140063C1E7027A240A209305C400BA977EA4CB
:106D2400EFB0EFC50824B165938505B8EF90BFECCB
:106D34005945B240224492444101828058229D47E1
:106D44000545E318F7FE0345440213351500D5B78E
:106D5400C5476396F5061E223A22FD17B387E7025C
:106D64000347450205072302E5025842C207C183CF
:106D74003E973C333823A207D98F41677D1763952B
:106D8400E70081473E858280138717005AA57A253C
:106D9400E3F9E7FE411122C49305C5002A840A21C0
:106DA40006C6EFB0CFC60824B165938505B8EF9049
:106DB4009FE4B2402244D9473E8541018280542257
:106DC40029478547E390E6FC034745025DFB5DBF29
:106DD400011122CC26CA4AC852C406CE4EC6BC21D2
:106DE40015472A8AAE84328436896399E704368645
:106DF400A28526851135AA895DE185476311F40AC8
:106E040003474900A9476300F70288344A87854647
:106E14000146D285EFE01FF119E585454A85EFE08B
:106E24009FE813341500B420883401476946D2859D
:106E3400EFE05FEF2685EFF01FBEB5A81D4763970F
:106E4400E7003686A2852685053D75B725476398F4
:106E5400E7003686A2852685EFF05F9B69BF35473C
:106E64006397E7003686A2852685B53D69B7454711
:106E74006397E7003686A2852685D93DADBF5D4779
:106E8400639EE700D82585473686A2852685631D3F
:106E9400F702EFF0CFCC8547631AF5048549A5477F
:106EA4006317F402835709009DE30544E38D09F653
:106EB400D947E391F9F82285F2406244D244424929
:106EC400B249224A05618280EFF08FD4E9B7883451
:106ED4004A87A2860146D285EFE0DFE479F5A285F0
:106EE4004A85EFE05FDC13341500C9B70544E1B708
:106EF400397122DC06DE26DA4AD84ED652D456D26E
:106F04009E211944B9E783C925002A89328A9387C7
:106F140059FE93F7D70FAE84DDE3B727002083C66D
:106F2400475C1307F00F938A475C19446383E602B6
:106F3400F5476395F90497A0FA1FE78000ABAA8987
:106F44001DCD30250DCE93178601E18763DD070043
:106F540001442285F2506254D2544259B259225A01
:106F6400925A21618280F5454A85EFE01FE483C788
:106F7400A90093E707F82385F900D9BF8149D620F2
:106F840090448C3088203800EFB0AFB92A8471F176
:106F9400B42003C50A0038000146CA85EFE09FD833
:106FA4002A8445F9B24799C323000A00BC207547D7
:106FB400E390E7FAE38E09F82385F90059BF97A017
:106FC400FA1FE78080A2AA8A41D58547639FF90802
:106FD400CE2088443000EFA0FFDD2A843DF903C7AA
:106FE4002A00C54763FFE708DD47630DF70AB73793
:106FF400002003C59A0083C7D79C6398A70A01445D
:1070040003C72A008D47631EF7043C8403D7CA00D4
:1070140063F4E7002396FA0083D5CA004A85EFF0AB
:107024006F8BB737002083D787836D47637BF70265
:1070340083D5CA005D476376B7021387350091058F
:107044006349F7001307B00FBE856374F700930517
:10705400B00F1166C20513060629C1814A85EF7077
:10706400D02D5685EFF03F9BEDB53C211144E392C2
:1070740037EF5C41E38F07ECCE20884430008297E1
:10708400A9BFB72702009387072AB3D7E700858BE8
:10709400B9DFB0203400D6854A85EFF07FD32300D2
:1070A400AA0045BD83A70A01E5B7B420380001460C
:1070B400CA85EFE03FC72A8421F5AC202800EFE021
:1070C4009FBE15DD23000A0025BF011122CC3734F1
:1070D400002006CE26CA4AC84EC652C49309C49C90
:1070E40003C589009307800291653305F5029385F2
:1070F4006570372900209304095C9790FA1FE78094
:1071040020F403C689009307800281453306F60202
:1071140088C09790FA1FE78060289C404D459DCF1A
:107124009304C49C1309095C0144130A8002FD59A9
:107134009C24636DF40237750500130545EFEFE0F9
:107144003FF8377505001305A59BEFA01FB73775EA
:1071540005001305C5A9EF30B0500145F240624463
:10716400D2444249B249224A05618280B3074403AA
:10717400032509006146814505041374F40F3E9507
:1071840023103501230105002314350123050500CF
:107194002302050231059790FA1FE780202049BF9A
:1071A40001458280B737002083C6579D814763E538
:1071B400D70001473A8582802E87910503D6C5FF03
:1071C400E30AA6FE8507E5B70DC93C2105478907F3
:1071D40093F7F70F6373F702411122C406C62A849A
:1071E4000E2128310147F9465D46EFE0BFB3F95758
:1071F4003EA0B2402244410182808280B737002001
:1072040003C7579DFD56814763E3E700828016A1BB
:107214002301050085071105C5BF01458280372676
:10722400002013067654930700021CA2372700207F
:10723400FD572303F75437270020230CF752372731
:107244000020A30BF7528545B72700202392B7549B
:10725400B72700202393075CB727002023A8075CE7
:10726400B727002023A0075EB727002023AA075CC6
:10727400B7260020B7E706009386C6539387873264
:10728400DCC2B72700202384075CB727002093873C
:10729400074D094798A298A398AB2380E702238857
:1072A400E70237E7060013078731D4C7D8DBB7E610
:1072B40006000D47238CE7029386463137270020CA
:1072C400D4CB0327C75C37E50600B7E606001305F1
:1072D400853393868634C8C38CA7239507008CAF67
:1072E400239D0700D0CFD4D323840702239507021C
:1072F40023A60702239D0702D8DFB727002037778C
:107304000500938707511307A73B23A00700D8C3A1
:1073140023A407008280411106C6693509C52821C6
:10732400B240410182800145E5BF411122C426C219
:107334004AC006C6AA842E893284AD3501E9416566
:10734400CA857D158535C54701C506A120A181479C
:10735400B2402244924402493E854101828029E39D
:1073640089483547639F1603011106CE22CC26CAED
:107374001832102293C7F7FF2207598EF18F32C6B5
:107384009DE3C4452A84A685793732460147630EB6
:10739400A60022856244F240A685D244056171B7F5
:1073A4002D473A85828013070008F2406244D24494
:1073B4003A850561828083C80500094863940803FF
:1073C40003A845008347180003480800A207B3E751
:1073D4000701C2070D68C187130828906394070149
:1073E4008947B5BF05458280011122CC372400208E
:1073F40013048453182006CE26CA4AC84EC69307DF
:10740400F00F630FF702AA892945B2842E89979059
:10741400FA1FE78040E20DC59307100B1EA123025B
:107424000500231135012313250106A5AA8508208B
:107434006244F240D2444249B24905616F904FBF61
:10744400F2406244D2444249B2490561828041110A
:10745400B727002026C2AE8483A5C75C22C406C613
:107464002A84553D098909C922852244B240A6854A
:10747400924441016FF08F98B240224492440545F2
:1074840041018280411122C426C24AC006C6AA8490
:10749400130445001309850B1E209DC3084409C528
:1074A4009790FA1FE780C0C62285314681459790A0
:1074B400FA1FE780A0EE3104231A04FEE31E24FD24
:1074C400B2402244FD579EA0024992444101828069
:1074D400B737002003C6579DB727002003A7875D51
:1074E40081476315F600814636858280BA86130784
:1074F400870B835587F4E389A5FE850793F7F70F78
:10750400CDB7B727002083A7075E81CBDA236314A6
:10751400A700884782809C43CDBF014582804111EA
:1075240006C6C53709C50845B240410182800145F8
:10753400E5BF011126CA9384450022CC4EC606CE6F
:107544004AC852C456C25AC026878149014481465A
:1075540081473D45122345CABDEE42233E23B286F0
:10756400A297C207C18385093107E395A9FE35C4F3
:107574002E8991659385457022859790FA1FE7803F
:1075840020AC2A8B39C9814A014A8C4495C1D22046
:1075940033054B019790FA1FE780A0D9DE20884479
:1075A4003E9A420A135A0A019790FA1FE78040B69E
:1075B40063890A003146814526859790FA1FE78042
:1075C400E0DD850AB104E3E23AFD232669012314D0
:1075D4008900054521A0630DD6000145F2406244AF
:1075E400D2444249B249224A924A024B05618280FE
:1075F4003223E314F6FE52233294B2974204C207B4
:107604004180C1838DB70545E37A35FD8DB7B72732
:10761400002083A7475D99E30145828098473A2774
:107624006315A7001385470082809C43EDB7411181
:1076340006C6F13F09C50A21B240410182800145D5
:10764400E5BF411106C6E13709C52821B240410111
:1076540082804145E5BF411122C42A842E8506C695
:10766400CD37AA8505462285EF30806895476305A6
:10767400F500BD476313F5002145B24022444101A2
:1076840082804111B727002022C406C603A4475DA7
:1076940081469387475D21C01844322718406317F9
:1076A400A60285CA98C22E8581C921469305440045
:1076B4009790FA1FE780E0C722859790FA1FE7802A
:1076C40020A50145B240224441018280A2863A8429
:1076D400D9B798C3C9BF0545F5B737270020832715
:1076E400075E01461307075EA1C703D8470094430A
:1076F400631BA802011106CE22CC26CA05CA14C2F5
:10770400AA843E852E849790FA1FE78060A02C00FF
:107714002685853F01E519C0B2471CC0F24062448A
:10772400D244056182803E86B6877DBF14C3C9BF3B
:1077340005458280411122C42A84090506C6EFE06A
:107744002FECFD573CB0B2402244410182804111EC
:1077540022C4416406C626C29307E4FF6301F5020E
:10776400AA849DE19790FA1FE780402B09E913054D
:10777400F4FF9790FA1FE780602A11C106A1B24076
:10778400224492444101828085476391F504979095
:10779400FA1FE780A0282A847DD1FD571EA13C2032
:1077A4001307F00F6381E7021307E00F6389E70013
:1077B40028300147F9465146A685EFE0AFD6228529
:1077C400953FFD573CA02302040055BF8947E39829
:1077D400F5FA8545EF30C0715DF126859790FA1F63
:1077E400E780C0232A8445FD59BF1D71A6CACEC6B1
:1077F40086CEA2CCCAC8D2C4D6C2DAC05EDEAE84FB
:10780400AC21F947AA896396F5049790FA1FE7809B
:10781400E0202A8411ED01442285F6406644D644D2
:107824004649B649264A964A064BF25B2561828050
:107834003C210547890793F7F70FE37EF7FC2831CE
:107844000147F9460146CE85EFE0CFCD2285DD35EF
:10785400D9B703AB0400B7070001938707F03707D4
:107864001200B377FB0013070710B28A0149638B38
:10787400E7022EC69790FA1FE780401A2A89B2457C
:1078840015C1502105C293178601E187E3C507F8A6
:107894004E85EFE08FD18347490093E707F8230231
:1078A400F90095BF372A002003476A549307F00F65
:1078B400130A6A541944E301F7F6E147E3EEB7F417
:1078C40093D71500FD1713973700B7E70600938782
:1078D400C7C9BA9703A80700E30008F483AB4700BD
:1078E400E38C0BF2420B135B0B0163050B00C947DE
:1078F400E394F5F2D62090448C308820380802981E
:107904002A8419F92C084E85829B2A8431C19C3023
:10791400E39407F0BC20230AA10039472308F100AF
:107924006396E70262471C331823A207D98F0C0819
:107934004E85FC81EFA08FDCE30F05EC14080546AF
:10794400D9454E85EFE06FE42A84F9B5BC84C5B708
:10795400B4209147E381F6EC03450A003808014658
:10796400CE85EFE02FBC2A84E31805EAAC20280872
:10797400EFE06FB319C123800A009840B7070001F4
:10798400938707F07D8FB707120093870710E304EE
:10799400F7E8E30209E8BC202302F900B5BD0111B0
:1079A40006CE2EC69790FA1FE780400711C95C21C6
:1079B400B245138717006395E50093F707F85CA1B8
:1079C400F24005618280397152D42E8A4ED69305D5
:1079D400E101AA89528522DC4AD856D206DE26DA8B
:1079E400328936C63AC4BE8A9790FA1FE780C0052A
:1079F400054435C1AA84A8873944EFF09FB021CD4E
:107A040003284500630908042247B246D6874A86FC
:107A1400A6854E8502982A841DED9307E00F638C9A
:107A2400FA02982089476318F702D8401C331823B8
:107A3400A207D98FC2070D67C18713072790639CDC
:107A4400E7008347190003460900D285A2075D8E2B
:107A54004E85EFF07F992285F2506254D2544259F8
:107A6400B259225A925A21618280797122D42221F8
:107A74004ECEAA89228556CA06D626D24AD052CCE0
:107A84005AC85EC662C4AE8AEFF09FA401E922859B
:107A9400EFA09FD2594429E5014499A003C7890066
:107AA4008547AA8401446316F702AA8513858900D1
:107AB400EFF03FA821C9FA209624D044CE2003D564
:107AC4002900E1470937D9472A846318F50223A618
:107AD40004002685EFF01F9B41C0D947E30EF4FA5A
:107AE4002285B250225492540259F249624AD24A2F
:107AF400424BB24B224C4561828061DDDE202390F3
:107B0400FA00C1BF13894400014AB94B594C3D4B9B
:107B140083550900DDDDE14763067A010357C90097
:107B240011C3D94703572900835649000326890006
:107B340003D52900EFF03FE92A8463198501232442
:107B44000900050A3109E3156AFD61B77DD9835738
:107B540009002390FA00F5B703D5290015BF0111D8
:107B640070879307E00F1306E1000147894606CEAC
:107B7400EFF07FE5F24005618280797122D42A8496
:107B84000A2526D2AE849305210106D64AD09790C1
:107B9400FA1FE78060EB79C51C252AC693F7070214
:107BA4009DC7A881EFF0BF97AA87B24511E91E24AB
:107BB40039459EA0B25022549254025945618280A4
:107BC4002A204946829701C51E249EA0E5B7035981
:107BD40024004A85EFF0DF8F01ED41657D15EFF05C
:107BE4003F8F09E51E2425459EA0E9B723102501F2
:107BF400130745008147BD46122339EE3147B38749
:107C0400E702130984003146CA8591073E9597809F
:107C1400FA1FE78000723146CA8548089780FA1F28
:107C2400E780207152242A2041478146DD45EFE058
:107C34000FD02ACE09E51E2445459EA0A5BF0C48B9
:107C440052249780FA1FE780C06E2A204C08EFA0C8
:107C54007FB22DD15945B9BF85073107E39ED7F8C7
:107C640025459DB705458DB7797122D42A840A2507
:107C740026D2AE849305E1014AD006D63289979084
:107C8400FA1FE78060DC2DC91C2593F7070295EFE6
:107C940018389307200511E35C20362450440E2441
:107CA4002A200147EFF03FD2AA8729E11C3891E747
:107CB4002A20EFA03FA8D94711E18147B2502254AE
:107CC400925402593E85456182802AC6A887EFF006
:107CD4001F85AA8705C5B2452A2049468297AA87E7
:107CE40045D91A249AA0183869FBC9BF5947E31A21
:107CF400E5FE23000900D1B78547E5B7B947D5B7F5
:107D0400397122DC4AD84ED652D406DE26DAAA8944
:107D14002E8A32C636899790FA1FE78020D009440C
:107D24000DC53C211307E00FAA845D44638FE7006F
:107D34001307F00F5944639AE700324605E2D285EF
:107D44004E85EFA09FAB2A841DCD2285F25062544C
:107D5400D2544259B259225A2161828003550A00F1
:107D64009305E101231F01009790FA1FE780C0CD1E
:107D7400A887EFF01F8DAA8505464E85EF20507722
:107D84002A8455DDD9B79307F00FE300F9FC377562
:107D94000500938624007946A6851305C51CEFE0EB
:107DA4006F85A381240155B73971B727002026DADE
:107DB40083A4475D52D45AD05ECE62CC06DE22DC68
:107DC4004AD84ED656D266CA2A8BAE8B328C368AA5
:107DD40099E08149A9A0804483DC44000149835A85
:107DE400A400631499018440E5B73E24A28963F892
:107DF400670105094209135909014104DDB7E3EAA2
:107E0400FBFE630B0A000C204840D28662863AC609
:107E1400EF905FE4324771DD19C323105701F2502C
:107E240062544E85D2544259B259225A925A025B34
:107E3400F24B624CD24C216182809A21B621854753
:107E440063E5E60439C34111D42126C237E50600AF
:107E54009384550022C426862E84130585338945D0
:107E640006C6EF903FDFC14719C954202E200A20CF
:107E740001472686EFF05FF3814711E1A947B2403D
:107E8400224492443E85410182803E8582802E8632
:107E94000A22AE21854763E1A50219CD542241117E
:107EA4000147150606C6EFF03FF0814711E1A947E7
:107EB400B2403E85410182803E8582802E860A2220
:107EC400AE21854763E1A50219CD54224111014732
:107ED400150606C6EFF05FED814711E1A947B240F0
:107EE4003E85410182803E85828039714ED6BE2115
:107EF40083D9050006DE22DC26DA4AD852D456D2CB
:107F04005AD05ECE62CC66CA6AC863EA3715854722
:107F140063880912416BAE8A2A8A2314010002C6BF
:107F2400014401497D1B894B054CC94C054D83D542
:107F34002A000147814601464E8523130100EFF0D4
:107F4400BFE6AA84630B050E09EC1307200293060F
:107F540061005A8695455285EFE06F9D2A8463023D
:107F6400051038849C2041CB18856305A707414739
:107F74006385E7022C005285EFA0CFCC09CD3400F5
:107F84001546D9455285EFE04F8011C5324597809B
:107F9400FA1FE780E017814765A0BE244146130518
:107FA40024001CA0BE24A1831CB0CC409780FA1FDF
:107FB400E780203849043C848507C207C1837C8458
:107FC40063FD2707BE24638A67078509C20993D91D
:107FD4000901B1BFE39077FBBE24094613052400D1
:107FE4001CA0BE24A1831CB0CC409780FA1FE7805C
:107FF40040341104C9B722C603596100B8241305DB
:108004002400638F7701335999032305710118A064
:10801400BE244146A1831CB0CC401379F90F79B733
:108024002305810118A0BE24135929001379F90FDF
:10803400A1831CB00946CC404DBF3C8485FFA947B1
:10804400F2506254D2544259B259225A925A025BA3
:10805400F24B624CD24C424D3E8521618280854771
:10806400C5B7C547F1BFB727002003C7E75E8547FB
:1080740063F4E706011122CC26CA4AC806CE2A8434
:108084003289AE849790FA1FE780409919C5382148
:108094009307E00F5D456308F700631C0900A6859C
:1080A4002285EFA02FF2F2406244D2444249056196
:1080B40082808A209305E100231701009790FA1F1C
:1080C400E78080982887EFF0CFD7AA8505462285D8
:1080D400EF20104269D5C1BF5945828013F70502CC
:1080E40001C7B2856FF02FD7411126C24AC006C618
:1080F40022C413F98500AA84631709001397850124
:108104006187635B070232853684EFF08FD3AA85DB
:1081140005466313090001462685EF20703D01E9F9
:108124000145B240224492440249410182801C34F8
:10813400EDDB1C24F5F7F5B793F72500F5F30D45B2
:10814400CDB77971AE8622D42A848A229305E101BF
:1081540006D636C69790FA1FE780008F11C90C2502
:10816400B246B08722859D3FB25022544561828039
:108174000545DDBF13F7050201C7B2856FF0AFCD2A
:10818400411122C426C206C693F485002A8491E4D0
:10819400139785016187635007023285EFF06FCA38
:1081A400AA85054691E0014622852244B2409244C4
:1081B40041016F20F03393F72500014591E30D450C
:1081C400B24022449244410182807971AE8622D425
:1081D4002A848A229305E10136C606D69790FA1FAF
:1081E400E7808086B24609C90C25B08722855937B5
:1081F400B2502254456182800545DDBF797126D293
:10820400AA842A25C16722D44AD04ECE06D6231783
:108214000100FD173284B6890149630CF500050598
:108224009420D04042051307E1004181EFF0DFB70D
:108234002A899420D04037E5060089451305853303
:10824400EF905FA115C5A2242285EFF04FBE09C5AA
:108254007D142A9442044180638409002390890098
:10826400B25022544A8592540259F249456182809F
:108274009420D04037E50600894513054534EF9036
:108284007F9D71F19420D04037E5060089451305A0
:108294004531EF903F9C11C9E30809FA3C87E39507
:1082A40087FA0354A9007D1475B7A22475B73971F0
:1082B40022DC26DA4AD84ED652D456D25AD062CCD0
:1082C40006DE5ECEBE899C252A8AAE84C18B328CA2
:1082D40036843A89C28A468B9DE783CB040089475A
:1082E400638BFB046285EFF0CFA11DC183280500D9
:1082F400638008025A88D6874E87CA862286A68556
:108304005285829839A03285EFF06FA1AA8711EDCA
:108314003945F2506254D2544259B259225A925AAF
:10832400025BF24B624C216182802946A68552850C
:10833400829745D5F9BFD8401C331823A207D98F9B
:10834400C2070D67C187930607906383D71E63CC6A
:10835400F60693062780638ED70A63C0F6021307D6
:108364000780E3C1E7F82D45E39509FADC4490233F
:10837400CC432310C9002285B9A213073780E393A5
:10838400E7F62D45E39709F885472310F900DC4407
:1083940081459C231CA0AA240505420541819780A0
:1083A400FA1FE780606A835709006310051091077C
:1083B4002310F90011468145130514009780FA1F14
:1083C400E780C0FDF1A8930627906386D71463C1A4
:1083D400D71093063790638DD71413074790E39310
:1083E400E7F02D45E39709F2DC441D472310E9002B
:1083F400982318A0983318B0BA2338A0BA2321833D
:1084040038B0D82358A0FA2358B0FE23A1837CA007
:1084140041A82D45E39F09EEDC446C0083C9170095
:108424009823A209B3E9E90011472310E9009C232A
:108434004E851CA0DC449C331CB09780FA1FE78057
:10844400A060AA8425C13086C1659306E100FD15AC
:108454008329C500EFF09FDA09ED9420D04037E579
:108464000600894513054534EF90CFFE19E1FD5709
:108474007C8703C7090089476310F70283A5490075
:108484000946130544009780FA1FE78080EA835762
:10849400090089072310F9003C873CA0A1833CB064
:1084A400014585BD23173101C5BF18218907BA9736
:1084B4002310F9003E251CB03E25A1833CA01021C9
:1084C4004C41130534009780FA1FE78080E6C9BF4A
:1084D400C8449780FA1FE78040EF93170501C183D2
:1084E4002A871D45E3E737E36399F9002310090060
:1084F400CC4403560900CE95BDBD4207B3863A016C
:10850400418363C7E600B38737412310F900CDB731
:1085140023105901F1BF2D45E39D09DECC4452855A
:10852400EFE07FDF2310790108A0218108B08DBF1F
:108534002D45E39009DEDC44231079019C231CA023
:10854400DC449C331CB0A9BF1D71CAC82A892A21E6
:10855400A2CCCEC6D2C4D6C2DAC05EDE62DC66DA93
:108564006ED686CEA6CA6AD8AE8AEF90DF82130C86
:10857400F5FF93170C01B72B0020C1832A8A814988
:1085840013840B793EC6372B0020B72C0020C16D15
:108594008357C90063F5F9001E2063CC8701035596
:1085A400290093850B79EFA0CF8D2A8D15CD594DD8
:1085B40025A883278900139719009305E101BA9729
:1085C40084339C23A204DD8C26859780FA1FE780E0
:1085D400A047AA8515E923909A004840054D09C58E
:1085E4009780FA1FE780C0B2F64066446A85D64495
:1085F4004649B649264A964A064BF25B625CD25C0F
:10860400425DB25D2561828032488348490083A679
:108614000C5DB08703552900814713076B5CEFF0AD
:108624001FC92A8D13880C5D09C523909A00484000
:108634007DB75C4085E70355290051478146138681
:10864400FDFFBD45EFD0BFAEB727002048C013885B
:10865400075D09E523909A00454D79B71E2003571D
:108664006B5C93046B5C3E976346470113C7F7FF4B
:1086740052979AA048409220832508003E95850988
:108684009780FA1FE780E0CA1E209A20C20993D976
:108694000901BA971EA0EDBD397122DC2A842A2172
:1086A40006DE26DA4AD84ED652D45AD05ECE62CCF2
:1086B40066CA2E8B56D26AC8EF90EFED2A8A5424EC
:1086C4002E240A2478001306D400130CBAFF651A6A
:1086D400EFF08FED420A37290020AA898144135A0A
:1086E4000A01B72B0020B72C0020130909796382F3
:1086F400090463D08405938A0C5D8348440083A6EF
:108704000A0030862A205288814713876B5CCE8505
:10871400138D6B5CEFF0BFB91DC1814A30862E24E6
:108724004E859306E100EFF07FADAA8963990A06AE
:108734005DFDF1E41E2429452310FB0035A8835771
:108744000D001228E31BF6FC83A50A004848978015
:10875400FA1FE78000CF71D18327490095EF2A20C3
:108764004166454781467D169D45EFD05F9C1DE1DE
:108774001E2445452310FB00F2506254D254425942
:10878400B259225A925A025BF24B624CD24C424D7D
:10879400216182802322A90083DAA90041B78327BB
:1087A4004900A69723805701938714001397070164
:1087B40083274900418393DA8A00BA9723805701BB
:1087C40013872400832649009387340042079104C9
:1087D4004183C207C204C183C180369711C934875B
:1087E40014A303274900BA973887218398A301B7B4
:1087F400FD5614A303274900BA9794A31DBF2A204A
:10880400B725002089802398957893850579EF9082
:10881400FFCE3DD159458DB7411122C406C693F709
:1088240005012A84328585C3EFE0BFE1AA850546A8
:108834002285EF20E04B95476305F500BD47631D96
:10884400F502214515A893F7450099CBEFE07FDFAA
:108854000546AA8522852244B24041016F20404941
:1088640093F7050489C7EFE0DFDD0146DDB713F5B3
:108874001500133515000605B240224441018280DB
:1088840079714AD04ECE52CC06D622D426D22A8A28
:10889400AE89014983D749006364F900014581A089
:1088A40083A7090013141900930414003387970055
:1088B4001823A297882322079305E100598D9780F6
:1088C400FA1FE780601805E583A7090005453E9473
:1088D400182098A383A70900BE94982098B3B25097
:1088E400225492540259F249624A456182800C250D
:1088F40030875285EFF05FF201CD83A709003E94E3
:10890400182098A383A70900BE94982098B3C1BFE8
:108914000509420913590901B5BF011122CC2A8462
:108924008A219305E10006CE9780FA1FE780C011E3
:1089340011C90C2530872285EFF01FEEF240624406
:10894400056182800545DDBF1D71CAC82A892A21B7
:1089540086CEA2CCA6CAD2C4D6C2DAC05EDE62DC9F
:1089640066DA2E8ACEC66AD86ED6EF90CFC22AC6F1
:108974008346C9008355A900035589007808130666
:10898400D900EFF06FC2B247B7240020416B938A3D
:10899400A7FFC20AAA8B014493DA0A01372C0020EC
:1089A400B72C0020938404797D1B63820B18B08656
:1089B40083C58B0003552900EFF01FE6AA8D6313CE
:1089C40005168348490083A60C5DB086035529002B
:1089D4005688814713076C5CDE85EFF05F8DAA8DA6
:1089E40093096C5C138D0C5D631E051215CC03D7C3
:1089F4000900BE2011076397E7003247A2976D175D
:108A040063C7E706B725002093870579BA23035582
:108A14002900938505793354E40282A3EF903FCA79
:108A2400AA8D15C1D94D05A0035529004947814692
:108A34005A86C545EFD0AFEFC8C015E583D7AB0064
:108A4400C54D2310FA00F64066446E85D644464967
:108A5400B649264A964A064BF25B625CD25C425D9A
:108A6400B25D2561828083D709009107BEA0DC40F6
:108A740003D7AB009306E101A29798A393071400D0
:108A840013970701DC4041835E85BA9703D7AB0097
:108A9400218398A3B0868355A900EFF02FF613071E
:108AA4002400D44093073400420711044183C207D1
:108AB4004204AA8BC1834180369715EDFD5614A359
:108AC400D84083250D00BA9794A3C84003D6090063
:108AD40022959780FA1FE780C08583D709003E94CA
:108AE4004204418005F0835789002310FA00E39C77
:108AF4000DF4A94D89BFB48783250D0014A3D84074
:108B0400BA97B887218398A3C84003D60900229551
:108B14009780FA1FE780E08183D709003E944204DE
:108B2400418061B583D7AB002310FA0065BF814D46
:108B340055BF5D71A6C2CAC0AA84035985002A2103
:108B4400A2C44EDE52DC5AD85ED662D466D286C641
:108B540056DA6AD06ECE2E8BEF90EFA3930BD5FF2F
:108B64007115131A0501B72900200144135A0A018B
:108B7400372C0020B72C002093890979635B741388
:108B8400D424AE241307E1001386D4004A85EFF001
:108B9400AFA12A8D630F05100359A5000C2530875A
:108BA400AA20EFF07FC7631B051083C8440083A687
:108BB4000C5D3087AA205288814713076C5CEA85D4
:108BC400EFF0EFEE930D6C5C13880C5D65E905C85E
:108BD40083D70D0003D7290089076308F706B72553
:108BE4000020138705793E23AA2093850579335401
:108BF400F40202A3EF905F990DC559451DA0AA2068
:108C040041664D4781467D16A545EFD04FD2B72723
:108C1400002023A2A9001388075D1DE123102B0166
:108C24004545B640264496440649F259625AD25AFA
:108C3400425BB25B225C925C025DF24D61618280B8
:108C440083D70D0089072391F90083D70D00A297DC
:108C540063D1770783A749000357AD00930A240023
:108C6400A29798A305049317040103A44900C183A0
:108C7400C20A3E948357AD008325080093DA0A01A3
:108C8400A1831CA003A5490003D60D005695977037
:108C9400FA1FE780006A03D40D00C167FD175694DC
:108CA40042044180E30CF9EC050942091359090116
:108CB400F1B529450DF423102B01A5B76DDC05B7DB
:108CC4001E2181E789473E858280411126C24441A5
:108CD40022C406C64AC09420D0402A8437E5060040
:108CE400894513058533EF80FFF611C93C202547DC
:108CF400E51793F7F70F6376F702E14721A894206D
:108D0400D04037E50600894513054534EF809FF4CC
:108D140071FD8947B2402244924402493E85410193
:108D240082803729002083564954854713094954C2
:108D3400F5D21A203697C166E3CEE6FC9165938599
:108D4400257031459770FA1FE780802FAA84CD479C
:108D540071D1314681459770FA1FE78020641E2047
:108D64008355090001460147B386E500C206C18266
:108D7400636BF702AE97C207C18319C22310F900CF
:108D840023A004002146A285138544009770FA1F8E
:108D9400E780205AB72700209387475D984309EF5F
:108DA40084C3814785BF50401315470005072A96A1
:108DB40036A6054655BF3E871C43F5FF04C399BF3D
:108DC400011106CE22CC26CA4AC809E98944F240D8
:108DD400624426854249D244056182802AC62A8497
:108DE400280036896C845085EFF09FEDAA8465F1E4
:108DF400E30F09FC3E24F9DB9165938555703145F9
:108E04009770FA1FE780C02305C53E242320050080
:108E1400232425015EA1B72700209387075E98438A
:108E240001E788C36DB73E871C43F5FF08C345B708
:108E3400CD4471BFB72700209387875C98230DE347
:108E4400054798A3058909CDB726002037250020BA
:108E540093860651414691451305054D6FF05FF623
:108E640001458280B7270020238CA7528280C167E6
:108E7400FD176315F5002E856FE04FB8411106C646
:108E8400EFE04FB209C5FD571EA123010500B24012
:108E94004101828001114AC806CE22CC26CA8547E8
:108EA4002A896392F5044A85EFE08FE231E9C164CF
:108EB40037E606009385F4FF1307E100894613069D
:108EC40086310545EFE05FEE2A84FD1405C44C4469
:108ED4004A85EFF0DFF9308722858146A685EFF0D9
:108EE400EFB12A84E5B789476396F5008545EF20FD
:108EF400200055D9F2406244D2444249056182803F
:108F0400EFE04FD86DB7011126CAB734002093841F
:108F1400C49C22CC8834372400201304845DB727F2
:108F240000203727002006CE4AC84EC6232004005E
:108F340023AE075C2326075C59C11389C75D9307D9
:108F4400200C3305F5029165938515709309C75C70
:108F54001905420541819770FA1FE780600E90342D
:108F64009307200C81453306F60208C01906977052
:108F7400FA1FE780A0421C40983481459386870BF2
:108F84007D5563E8E5069306800BB306D7020146D8
:108F9400FD550507B6972320F900BE868EA2ACB214
:108FA400ACA22382060005069906E369E6FEF9569B
:108FB40096A399463307D702BA9723A0F9003775C9
:108FC40005001305E57EEFD04F90378505001305A6
:108FD400259AEF803FCF3775050013052575EF10EF
:108FE4003068F2406244D2444249B24901450561C5
:108FF40082802394A6F41386C6F423100600232447
:1090040006003106E31BD6FE85059386860B95BFC5
:10901400411106C622C42A84EFC04FB3EFE02FA04B
:10902400B7270020A38B8752B727002003A5C75C6E
:10903400EFE0CF9CB7270020238387542244B2401B
:1090440037950500130585E941016F107061939709
:109054000501C18763D10730B727002003C57753C3
:10906400797122D45AC806D626D24AD04ECE52CCD2
:1090740056CA2E8B9770FA1FE78040212A8429C58F
:1090840018219307000B631EF702B72400208547BD
:109094009384045DDC849C4023150100B9E3EF0054
:1090A40080759165938535709770FA1FE78040F954
:1090B40088C005E99C8491C74C2013058400EFD037
:1090C4008FDC2285EF70EFF1B250225421653345D5
:1090D400AB0092540259F249624AD24A424B45616A
:1090E4008280372A00206146814513050A799770EA
:1090F400FA1FE780A02A03494400894793040A79A8
:10910400D289930A0A79631AF904F5258AA02A20D8
:1091140093050A79EF906FAF3A209E20162401ED53
:1091240063E3F6001EA40E243A85EFC0BFFA22853D
:10913400EFC0FFCF41B763E3F6001EA41E24D94558
:10914400938609790D463A852390FA00EFC0FFE330
:109154008D4571DD1385097965A899476319F9026D
:109164009305A1002285EFF02FD3AA8469D1D947B2
:10917400639EF40C05092A201379F90FD9459386C7
:1091840009794A86EFC07FE0CA8555D1E1B7A14786
:109194006318F9009305A1002285EFF09F99F1B7B8
:1091A400A947631AF9060A246C009780FA1FE7801E
:1091B400A0892A89630905122A2041669306E100E1
:1091C40055477D16AD45EFC09FF6C8C0AA8625CD8C
:1091D400834844000358E10030862A20814713075E
:1091E4000A79CA85EFF0AF8CAA84631F050C2A2084
:1091F40093050A79EF90EFBE1DD92A2093060A79C8
:109204002D46D945EFC07FD81DD1AD4513050A7948
:10921400EFD06FC729BFB147631BF90C0A246C0058
:109224009780FA1FE7804082AA8455CD2A204166A0
:109234009306E10059477D16B545EFC05FEF23A2C1
:10924400AA00AA8631E11E24C5447C851830D14782
:10925400E30FF7EC5C202A20938509792380FA0038
:109264003C8523829A002391FA00EF803FC9E300F2
:1092740005EC2A20938609790546D945EFC0FFD02D
:10928400E30705EA8545F9B5834844000358E1003E
:109294003E2430862A20A68513070A79EFF02F8111
:1092A400AA841DE12A2093050A79EF90CFB8E30040
:1092B40005E82A20D94593060A793546EFC0FFCC44
:1092C400B545E30605E679B5D9476393F4008144CF
:1092D40003A54A009770FA1FE78080E3E38904E45A
:1092E4001E247C85A5B71E2485447C8585B7B94793
:1092F4006318F9009305A1002285EFF0EFA4B5B53A
:10930400C1476318F9009305A1002285EFF0CFE36C
:10931400A9BDC947631AF900130691009305A1007A
:109324002285EFE07F9491B5D947631DF900930539
:10933400A1002285EFE07F84AA84E31A05E2A30456
:109344000100F5B3E147E314F9DE9305A10022859A
:10935400EFE0AFF119BD01458280F9CE011152C48D
:109364002E8A854522CC4EC656C206CE26CA4AC887
:10937400AA8AB6893284EF10B037D1471DC5B72702
:1093840000203727002083C7C75E8346D75E814409
:1093940019E0B684BE86372700200327475E9397DB
:1093A4004400BA9763EDD400D547F2406244D244F6
:1093B4004249B249224A924A3E85056182803E89E9
:1093C400C10703D727FF09C7850493F4F40FD9BF56
:1093D40031CC9565938525C0130500029770FA1F5B
:1093E400E78000C62326A90061D113060002814547
:1093F400938404049770FA1FE78040FA23119900BC
:1094040023000900231359010DC4373700201C34ED
:10941400032607932304F900118C8327C9001184C0
:109424001180C0AF23A02901814741B72326090039
:10943400C1BF23044901FDB785473E858280B72714
:10944400002083C5C75EB727002003A7475E814776
:109454006395F5008146368582803223BA8619C227
:10946400E30BA6FE850793F7F70F4107D5B7B72798
:10947400002003C6C75EB727002003A7475E8147C5
:109484006315F6008146368582802E23BA8681C50F
:109494004C23E38AA5FE850793F7F70F4107CDB761
:1094A400B727002083C5F75EB737002003A70793CB
:1094B40081476395F5008146368582801223BA86FA
:1094C40019C2E30BA6FE850793F7F70F4107D5B73B
:1094D400B727002003C8D75EB727002083A7475EBD
:1094E40001476315E800814636858280B223BE8633
:1094F40009CAF2236317A600D04701C63222E30546
:10950400B6FE05071377F70FC107E1BF411122C467
:10951400404526C206C6AA8415C0484409C59770AA
:10952400FA1FE780E0BE484809C59770FA1FE78034
:1095340020BE22859770FA1FE78080BD26854146AC
:1095440081459770FA1FE78060E5B2402244FD57D9
:109554009CB4924441018280011122CC2A842A21A4
:1095640006CE2EC6EF104067324622858145EF00B5
:10957400F05622856244F24005616FF03FF905C55B
:109584003A21411122C406C62A8411CBDD45EF00DD
:10959400F05722852244B24041016FF03FF7B240B8
:1095A4002244410182808280411126C2B146930443
:1095B400C5FFB386D402B73700201387079406C6C5
:1095C40022C4369736276397B602484305C51384E9
:1095D40007949307F00F6305F6001C21639CC700F2
:1095E4009770FA1FE780C0B2B147B387F402A2971D
:1095F40023A20700B24022449244410182804111D7
:1096040022C42E8426C24946AA848145228506C6E0
:109614009770FA1FE78080D895CCDC2C139747000D
:10962400B737002083A70793BA979A231AA0BA23BF
:10963400FE233AA0372700200357A75E5AA09A209A
:109644007AA0BA201AA4DA203AA4FA205AA49A24B6
:109654001EA87AA4B2402244924441018280B727D2
:10966400002083C5C75EB737002003A80793B72738
:10967400002003A6475E014781476394E5003E85C9
:109684008280142299CA544689CAD42E9206C2965C
:109694006315D500850793F7F70F05071377F70FC1
:1096A4004106E1BF130600643386C50293069500A4
:1096B400AA8537950500130525586F702FFE4111B3
:1096C40022C406C62A840835EF705F97FD571CB480
:1096D400B240224441018280011122CC4AC84EC6C4
:1096E40052C456C25AC006CE26CA2A89AE8901443B
:1096F400372A0020B72A00201D4B8347DA5E6365B2
:10970400F40463990902B7290020372A0020930A38
:10971400F00F83C7C95E6364F4061144A144228533
:10972400050442041306F00FCA854180EFF0DFE719
:10973400E31794FEF2406244D2444249B249224AB9
:10974400924A024B0561828083A74A5E93144400C7
:10975400BE949C208DC3FE20639F270163956901FD
:10976400AA20EF10604726854E868145EF0010370A
:109774002685EFF0BFD905041374F40FBDBF83270A
:109784004A5E93144400BE949C208DC39C34638F22
:109794005701FE20639C27012685EFF05FF22685A2
:1097A400D145EF00B0362685EFF05FD6050413747B
:1097B400F40F85B741677917630BE502411122C4A1
:1097C40006C685472A846399F50022852244B2405F
:1097D400814541016FF05FF089476396F500854547
:1097E400EF1000717DD1B240224441018280828019
:1097F4009D456FF07FEEB727002003D5A75E8280DA
:10980400B727002003C7875E011106CE68876C86E0
:1098140085476318F70070009305E1000545EF5094
:109824008032F24005618280A947631DF6029C31B3
:109834009821A207D98F1EA1BC31B821A207D98FC4
:109844003EA1DC31D821A207D98F5EA1FC31F821D9
:10985400A207D98F7EA19C359825A207D98F1EA572
:1098640001458280054582809147631EF6009C3144
:109874009821A207D98F1EA1BC31B821A207D98F84
:109884003EA101458280054582809387C5FF93965A
:109894000701C1820D47636ED7003147B387E702E2
:1098A4003737002013070794BA97A8A38EA301455E
:1098B4008280094582809306402037270020AA87AA
:1098C40063F4A60093074020F1172315F75EB7272A
:1098D40000202387B75EB72700202388B75E8280E5
:1098E4001905956542054111938535C0418106C628
:1098F4009760FA1FE780C07401C9B240E95541017D
:109904001773FA1F6700038EB24041018280B727A4
:1099140000202387075EB727002079710547238439
:10992400075EB7370020238EE7924ECEB72700207C
:10993400B729002022D426D24AD037240020B724C5
:109944000020A388075E37290020B72700209389C9
:10995400F95E06D652CC2AC62306045EA386045EAC
:109964002395075E2322095E23800900EF10402E11
:109974003245B737002013060003238AA7923735F0
:1099840000201305059481459770FA1FE78000A114
:10999400373A002003450A971304C45E9384D45EC7
:1099A4001309495E05CD9565938545C012059760F9
:1099B400FA1FE780E068373700202328A79219CDE3
:1099C40003460A9793070A979C332380C90081456D
:1099D40012069CA09770FA1FE780409CB7370020BE
:1099E40003C5479D9C209565938555C03E95137589
:1099F400F50F08A012059760FA1FE7806064232022
:109A0400A90051C11020814512069770FA1FE78002
:109A1400E098032709001420814725077D56639E9B
:109A2400F604EF104043B1473305F502956593857D
:109A340065C0420541819760FA1FE7806060B737CF
:109A4400002023ACA7922A8401CDEF10C0403146F8
:109A54003306C502814522859770FA1FE78000947A
:109A64002254B25092540259F249624A3795050081
:109A74001305857B45616F10A03E850710A393F7FE
:109A8400F70F410769BF230004002380040051BF7E
:109A940041119397050126C206C622C44AC0C18754
:109AA400AE8463DE07083739002003454993976085
:109AB400FA1FE780A07D2A8429C918219307000989
:109AC4006312F7041831CD476319F706B73600203F
:109AD4000348250003C57683372700208347E75EC4
:109AE40013066400814581461307E75EAA8863165E
:109AF400D80291C11CA31C2391C7034549938545F2
:109B0400EF702F872285EF60DFCD2165258DB24070
:109B1400224492440249410182800C22AE9793F57B
:109B2400F70F93F7F80F63F4A50093F7F50F850685
:109B340093F6F60F090685455DBF092BE1B793F748
:109B440015000145E9D7EF00305209CDB7270020B1
:109B540083C7E75E81CBB737002003C547938545AC
:109B6400EF702F8113C514005DB785462A8763FF04
:109B7400C6029C319021A207D18F1EA16399D70000
:109B8400BC31B421A207D58F3EA10145828089460C
:109B94000145639ED700BC31B421A207D58F3EA3F3
:109BA400DC31D421A207D58F5EA382800545828053
:109BB4009147631EF6009C319821A207D98F1EA1FC
:109BC400BC31B821A207D98F3EA101458280054549
:109BD40082809147631EF6009C319821A207D98F99
:109BE4001EA1BC31B821A207D98F3EA101458280B4
:109BF40005458280A1476318F6029C319821A2078B
:109C0400D98F1EA1BC31B821A207D98F3EA1DC3166
:109C1400D821A207D98F5EA1FC31F821A207D98FE0
:109C24007EA1014582800545828089476319F6003B
:109C34009C319821A207D98F1EA101458280054538
:109C440082803E2279714ECE06D622D426D24AD0C4
:109C54001307F007AE896371F70209473AC47C869B
:109C6400300093F5F50FEF001076B2502254925461
:109C74000259F249456182805A22D9462A8932849E
:109C840063F7E6007E2263F4F6006379F700231499
:109C94000100300093F5F90F4A85F1B70A2202C496
:109CA400EFF01F80AA8435C5EFF07F9B9C24636985
:109CB400F5001146A246CE854A85EF00906775B738
:109CC400340026869305F00F4A85EFF00FE975F10D
:109CD400A2471A24DC479AA33A20BAA35A20DAA34B
:109CE4007A20FAA3DA209AA7DC4495C793F4F90FF3
:109CF4002286A6854A858297C167FD172A86E31BBB
:109D0400F5FA22459947F9451CA144A1EFF09F9922
:109D1400A9BF094645B7014671BFA947631DF602AD
:109D24009C319821A207D98F1EA1BC31B821A2076A
:109D3400D98F3EA1DC31D821A207D98F5EA1FC3195
:109D4400F821A207D98F7EA19C359825A207D98F27
:109D54001EA501458280054582809C211CA19C3161
:109D64001CB1BC31B821A207D98F3EA18280232225
:109D74000500D82189476304F70005458280F62150
:109D84000D47E37CD7FE9C45011106CE22CC26CAA2
:109D94004AC84EC684339023A204D18C138644004F
:109DA4006311D604A033BC23AE8922045D8C9307CF
:109DB400C4FFC207C1832A896361F70203A589002E
:109DC4002311990023108900F1559760FA1FE78049
:109DD40060412322A900014531A02285EFF02FE63E
:109DE40071FD0545F2406244D2444249B2490561DD
:109DF4008280397122DC2E841C204AD806DE26DAC1
:109E04004ED619472A89B2856392E7063020280086
:109E1400EFF01FDAAA8405E92884EFF04FE2AA895B
:109E24000C3015C937B705002E861307E7B1340087
:109E34009D454A85EF00702F4E8509468145792955
:109E44004E85EFF0AFECF250625426854259D2545D
:109E5400B2592161828089477C803C840A867C8156
:109E64003C857C824A85EF001056F1BF49476398D0
:109E7400E70232202800EFF0FFD7AA8469F53735CE
:109E84000020130505945E2599E381446DBF1830C5
:109E9400142068253C000146CA85CD2C6DB7514776
:109EA400639EE70032202800EFF01F98AA8441FD4A
:109EB4000C3030004A85EFF0DFD871B75947639B07
:109EC400E70432202800EFF03F9AAA842DFD2C8469
:109ED4004A85EFF0EFDF05C9584534851E23B69750
:109EE400C207C1831EA3D5D35C47C5D3B7270020BF
:109EF40083C7E75ED9DBB737002003C547938545A1
:109F0400EF603FC789B789473EC03C840A860C305E
:109F14007C8289BF0C300A8623100100EF00B04A0E
:109F2400ADB75D71A6C256DA86C6A2C4CAC04EDEFB
:109F340052DCAA8A8831AE8432C6EFF04FD3B245E0
:109F440001ED8144B6402644268506499644F259DB
:109F5400625AD25A616182802302050023110500EE
:109F640083C9040085472A846399F900B02028082E
:109F7400EFF0BFBFAA8405491DA09D476391F90472
:109F840018218D47E31FF7FAB02028080549EFF0A0
:109F94005FC4AA8409E50546814522858126228578
:109FA400EFF0EFF108243C080147CE862686D685DB
:109FB400F12AE30909F82285EFF04FD561B7CD47BF
:109FC400639BF90018219147E31DF7F6B020280898
:109FD400EFF0BFC545B7D547E395F9F6034A050049
:109FE4008947E310FAF6B02028080549EFF0FFD2BC
:109FF400AA8455F583570102A1EBB8841306F00334
:10A004005C44930607FCC206C182636AD600B0852D
:10A01400D94663F6C600B486D94563EDD5002A2037
:10A02400BAA30549EF00503B03560102D2852285AD
:10A03400A92CB5B7AC87BAA3D2A38EA3F6A3854740
:10A044001CA0014A0149CDB7014AF9BF7971AA851B
:10A0540022D426D22221AA84280806D6EFF03FD1A2
:10A06400F24599E53DE185452285EFF06FF975A04C
:10A07400BC8415476395E706B8858D4763F7E70405
:10A084006800EFF09FCD3887DD4763FBE7008C86DF
:10A09400B70717008507100822853EC8EF00B032C5
:10A0A4003C87B88591076305F7002285EFF04FF4EC
:10A0B4001C8672466C00858B1106228591CFEFF0C9
:10A0C4005FE601C52285EFF0AFF2884449DD976071
:10A0D400FA1FE780E00341BFEFF0BFD1DDB71147BE
:10A0E4006389E7001387A7FF42074183854663EB33
:10A0F400E6023147F117B387E70237370020130729
:10A104000794BA979A2371D3A8233008A28505200F
:10A114004DFDB8849147E318F7F4B2502254925499
:10A12400456182802C082285FD2445F1FDB701118B
:10A134004AC82A89314526CA06CE22CC2EC6B28404
:10A144009760FA1FE780200F21C1B2459307000AE8
:10A154001EA12EA12A84214611058DC0A6859760D3
:10A16400FA1FE780001DA2854A85EF606FEC014568
:10A17400F2406244D244424905618280814597603D
:10A18400FA1FE780A021C5B70545DDB7797126D24E
:10A19400AA841305000206D622D42ECE32CC36CAA7
:10A1A4003AC83EC69760FA1FE780E00829C56246B0
:10A1B400F2454247D246B2472A84130520FA08A042
:10A1C40010B02EA058A054B013058400614691CF5E
:10A1D400BE859760FA1FE780C015A2852254B2504D
:10A1E4002685925445616F60AFE481459760FA1FFC
:10A1F400E780C01ADDB7B250225492544561828080
:10A204005845797122D406D62A84AE862DC73E23BA
:10A21400FC85930720066397F504B727002003D62F
:10A22400A75E7E236373F600B28713F6F70F2E2B17
:10A234001C2B8D8F93F7F70F81E5890793F7F70FA1
:10A24400B297FD17B3C7C702FC863E206E200824D0
:10A25400FC8401473C080146EFF05FF3B2502254FE
:10A2640045618280582FB737002083A707931207D0
:10A27400BA97FE23D1BF2EC6194681452808976098
:10A28400FA1FE780A011B246C9B7797122D406D665
:10A2940026D22A8499CD81470147930600062E864B
:10A2A4006E200824EFF09FEEB25022549254456180
:10A2B4008280B284280059469760FA1FE780000E16
:10A2C400648499E43E2048446C007C85EFF02FB30D
:10A2D4003C000147930600060146D9B7797106D6BA
:10A2E400814791E93E21584570867C843C0001C732
:10A2F4003E237C853C002E866E210825014793066B
:10A304000006EFF0BFE8B25045618280411122C4DB
:10A3140006C61C2111472A846392E7022E866E2109
:10A32400082581470147CD46EFF05FE649466E2098
:10A334002244B240154541016FF00FA713F7B70F40
:10A3440089466317D7000146EFF03FF45146C5B77D
:10A354000D476398E7002244B240014641016FF083
:10A36400FFF7B2402244410182809A21B146B737B7
:10A37400002071173307D70293870794BA97D843FD
:10A3840001EBD841AAA70145D8C3BA219AA7828074
:10A3940059458280797122D4404526D24AD006D6C6
:10A3A400AA842E8931C4484419C59760FA1FE780EE
:10A3B40020D6232604001E20EE2088247C853E20FF
:10A3C4000147930640067C861E244A867C871C48E7
:10A3D4003EC8BE207C843C00EFF05FDBA30E24016A
:10A3E40023280400B25022549254025945618280B9
:10A3F4002800314681459760FA1FE78020FABE2085
:10A40400EE2088247C8401473C00930640064A865B
:10A41400EFF0DFD7C1BF797152CC2A8A8A2126D2C4
:10A4240006D622D44AD04ECE56CAAE84EFF02F813F
:10A4340019E1854795A84045AA8965DC7E21E39A00
:10A4440047FF1E2463890710542CB73A002003A742
:10A454000A939206FD173697C2077A23C1831EA476
:10A464006316F70093053006EFF09FD95C48A5EF1B
:10A47400C840034915001C2122093369F900BE2094
:10A4840013072900631CF702F9559760FA1FE78048
:10A4940060D5C8C02391240103C589002686D285CE
:10A4A400EFF0FFC8814721E1B2502254925402597F
:10A4B400F249624AD24A3E85456182809565938518
:10A4C40015C04A859760FA1FE78080B748C8C8401E
:10A4D400231C2401F9559760FA1FE780A0D0BE2001
:10A4E400C8C0F917BEA0484825CDB220362C1E2C72
:10A4F4003308D60063C80707582C83A70A939545E9
:10A504001207BA97BE2363C90705CC4036959760F6
:10A51400FA1FE78000E23A2CBE20BA97C2071A2C31
:10A52400C1833EACE397E7F003D7290003C5890054
:10A53400300078845848D2857C853AC6EFF03FBF16
:10A5440011C548489760FA1FE78080BC232A04009D
:10A55400232C0400F9BD99454E85EFE0FFFFD1BDE2
:10A56400A545DDBF9145CDBFBA2171CBB7270020EA
:10A5740083D6A75EED4763E5E60C011122CC2E8459
:10A5840026CAAA844840914506CE9760FA1FE78000
:10A5940060C53E20AA861CA13E20A1831CB11E20BA
:10A5A4003CA11E20A1833CB13220C167F9171106DA
:10A5B400420641826394F4042AC4314532C697604A
:10A5C400FA1FE78040C7AA85CD471DC1930700F94C
:10A5D4001CA13246F957A2463EA189475CA1B73770
:10A5E400002072A114C503C54793EF606FA481478F
:10A5F400F2406244D2443E850561828081452685CD
:10A60400EF40C061AA8711E9B726002003C7E65EC0
:10A6140065D37D172387E65EE1BF09476304E5023E
:10A624001D476303E50249476302E5027D47E311E1
:10A63400E5FCB726002003C7E65E8147D1BFED479E
:10A644003E858280D1476DB791475DB789474DB745
:10A6540001114AC831471309C5FF3307E902B73767
:10A66400002026CA9384079406CE22CCBA94D840FC
:10A6740029C713840794B727002083C6E75E85475C
:10A6840095C668849E24AA242C003AC67C85EFF0E3
:10A69400BFED11C5C8409760FA1FE78060A7B147B6
:10A6A400B307F902A29723A207008547F240624448
:10A6B400D24442493E85056182808147C5BF797194
:10A6C40026D24445372700204AD0FE200359A75EEE
:10A6D40052CC06D622D44ECE56CA2A8A63F3270118
:10A6E4003E89BA284209135909019E2835CF998F0A
:10A6F4004A8463D527011394070141808945228543
:10A70400EFF00F9EAA89CD4A31C5BE202AC66085C6
:10A714007C84BE2899EB9E28930925001CA19E28C1
:10A72400A1831CB1637424058228BE28CC442286EC
:10A734004E85BE959760FA1FE780A0BF03556A0057
:10A744002C00EFF07FE2AA8A15C54E859760FA1FA8
:10A75400E780009CB2502254568592540259F24923
:10A76400624AD24A45618280890759B77914420402
:10A77400418065BFBA289E203A94FD17C20742045F
:10A784009A28C18341809EA0A2A86376E400F9F3CD
:10A79400FD57DCBCC1B781455285EFF0BFBF5DBF3B
:10A7A40079714AD03729002052CC034A195F22D448
:10A7B40056CA5AC85EC662C406D626D24ECE528443
:10A7C400B72A0020054B930BF00F372C002083A7EA
:10A7D4004A5E93144400BE9483C90400639B6907D2
:10A7E400DC44A5CBD84735C79A2329CBB72700200B
:10A7F40083C7E75E99CF2685EFF07FECAA8515E93C
:10A80400B727002083C7D75E05046351F402A30869
:10A81400895EB25022544E8592540259F249624ADA
:10A82400D24A424BB24B224C45618280A308095E56
:10A83400CDB72685EFF01FB68149E1BFDC3F639AAF
:10A844007701930520062685EFF09F9BDC44A38EB9
:10A8540007008347DC5E05041374F40F6363F4009C
:10A864000144E31644F7C9BF4111154506C6EFF08C
:10A874003FDE09C50545B240410182801945EFF02C
:10A884003FDD6DF91145EFF0BFDC6DF51D45EFF0CF
:10A894003FDC6DF1B727002083C7D75EE9DFB24004
:10A8A40041016FF0FFEF9E210D47F117C207C183ED
:10A8B4006363F706DC41A5C3411122C42E84854598
:10A8C40026C206C6AA842D2529C926853D2BC16723
:10A8D400F917638FF40009ED3E2099CB1620194730
:10A8E4006393E604372700200357A75E63FDE7025E
:10A8F400B727002083C7E75EA285268599C722442F
:10A90400B240924441016FF03FC62244B2409244A7
:10A9140041016FF09FA5094582805145B240224410
:10A924009244410182806D45D5BF397126DA4ED6F5
:10A93400AA84AE895D4589454AD806DE22DC32897F
:10A9440036C63AC4EFE0DFF935C122472A8401450F
:10A9540011C7B24613054400B68502979357850084
:10A9640023003401A30024013CB09547FC84B7279D
:10A97400002083C7E75E28A01105E88522CE2C08B5
:10A98400268595C3EFF05FBEAA8411C52285975032
:10A99400FA1FE780E077F250625426854259D25478
:10A9A400B25921618280EFF05F9CF9BFCD44E5B7D5
:10A9B400797126D24AD052CC56CA06D6BA8A22D443
:10A9C4004ECE19472E89B284368A6395E5062A222B
:10A9D4000944EFE0DFA62AC635C55C458359650006
:10A9E400BE239EA0B247B7360020154723805701E7
:10A9F40003C6C693BAA3130716001377F70F238E63
:10AA0400E692D0A301E70547238EE69251476317E8
:10AA1400E9001547BAA0DC479A249AA75287A6866C
:10AA2400CA854E85EFF07FF02A84324515C4EFE0E5
:10AA3400FFAD09A842867400BE85AA89EFE0FF91A4
:10AA44002A844DD12285B250225492540259F2499B
:10AA5400624AD24A45618280F945EFE0BFC4DDB75E
:10AA64009E211CA19E21A1831CB1BE213CA1BE211B
:10AA7400A1833CB1114582809E211CA19E21A1830A
:10AA84001CB1BE213CA1BE21A1833CB1DE215CA14D
:10AA9400DE21A1835CB1FE217CA1FE21A1837CB1D6
:10AAA400214582809E211CA19E21A1831CB1BE212F
:10AAB4003CA1BE21A1833CB1DE215CA1DE21A183A6
:10AAC4005CB1FE217CA1FE21A1837CB19E251CA545
:10AAD4009E25A1831CB5294582809A218546AA8793
:10AAE40018A19A21218318B19A216319D700BA2198
:10AAF40038A1BA21218338B1114582800945631DEB
:10AB0400A700BA211945B8A3BA212183B8B3DA2121
:10AB1400D8A3DA212183D8B382809E211CA19E214F
:10AB2400A1831CB1BE213CA1BE21A1833CB111452E
:10AB34008280797126D24AD04ECEB2842A89AE89D7
:10AB440029468145480022D406D636849760FA1FE8
:10AB5400E780C08464868DE43E207C82B727002091
:10AB640083D7A75E7C845C4481CFD42F3737002001
:10AB74000327079392069E2736973A237C8578838A
:10AB840037B705004A85130787AA540013F6F90F4F
:10AB9400D545EFF09FD92A8911C195E085471CA0BE
:10ABA40023020400014681452285EFF00FEEB250E6
:10ABB40022544A8592540259F24945618280228581
:10ABC400EFE0DF94EDB737B70500B2861307E7ADC2
:10ABD4002E8685456FF07FD501116887B7B60500CD
:10ABE4004165700001489307F00F0D47938646A610
:10ABF40099457D1506CEEFF0BFDBF24005618280FA
:10AC0400B7B60500B28701482E8611479386C6A7BA
:10AC1400C9456FF0FFD9011122CC37340020130449
:10AC2400849726CA4AC84EC606CE2A89AE8993049A
:10AC340004031C4081C7CE854A8582971104E31A18
:10AC440094FEF2406244D2444249B2490561828092
:10AC5400B737002003C5D783411122C437340020FD
:10AC6400937735001304C49C09811CB4AA9706C6C3
:10AC740026C21CA4ADCB1305C0033385A702A5656A
:10AC84008505B73400209750FA1FE780603B1024F5
:10AC94009307C00381453306F60223AAA49697506E
:10ACA400FA1FE780A06F83A74497142401478907FC
:10ACB4007D566341D7022244B24092443735002086
:10ACC4001306000381451305859741011753FA1FA5
:10ACD4006700C36C92A32381070023A5070205071D
:10ACE4009387C703F9B7B24022449244410182805A
:10ACF400011122CC2EC632C406CE2A849760FA1FD4
:10AD0400E78040D92246B24511E9C167F9176303C8
:10AD1400F4005145F24062440561828054555C213F
:10AD24008DC213F7270141456314A70015457DF231
:10AD3400C18B3D45E5D3BC2E0145E3FDB7FC314550
:10AD4400D1BFC18B0145F9F71545E9B7797126D211
:10AD54004AD0B7340020416922D44ECE52CC56CAD0
:10AD64005AC806D6AA8901449384C49C373A002061
:10AD7400930AC0037D19054B9C246364F4000145C8
:10AD840025A8B307540303274A97BA97BA2363162F
:10AD9400270105041374F40FC5B7C8333000938535
:10ADA4006700EF00B1671946CE8528009750FA1F57
:10ADB400E7802069E31F65FDB25022549254025982
:10ADC400F249624AD24A424B45618280B737002039
:10ADD40083C5479DC166B737002003A74797FD1673
:10ADE40081476395F5000146328582800358270028
:10ADF4003A866306D80003480700E307A8FE8507E0
:10AE040093F7F70F1307C703E9BF411106C697600D
:10AE1400FA1FE78020C809C54A29B240410182804F
:10AE24000145E5BFB737002083C6479DB7370020EB
:10AE340003A747970145814711076393F600828072
:10AE4400102301C605051375F50F850793F7F70F52
:10AE54001307C703DDB7B737002003C5479D8280BA
:10AE64003737002093068797814713078797314622
:10AE74008C4291E58A07BA9788C301458280850789
:10AE84009106E397C7FE4D458280411106C622C450
:10AE94009760FA1FE78000C00DCD2A842A218545DA
:10AEA400EFF07FD7485409C59750FA1FE780402632
:10AEB40022851306C00381459750FA1FE780004E90
:10AEC400FD573EA0230204000145B2402244410143
:10AED40082800945DDBF411106C69760FA1FE780ED
:10AEE40060BB09C54825B240410182800145E5BFE8
:10AEF400C167F9176305F502411122C406C62E8401
:10AF04009760FA1FE78000B9AA87014589C7C8235B
:10AF1400698C33358000B24022444101828005456A
:10AF24008280011106CE2EC69760FA1FE78080B694
:10AF3400854701C95A29B24585476304B7004EA91C
:10AF44008147F2403E850561828029CD01114AC8BE
:10AF54004EC637390020C16922CC26CA52C456C213
:10AF640006CE0144AA841309C99C373A0020930AE7
:10AF7400C003FD1983478900634BF400F240624427
:10AF8400D2444249B249224A924A05618280330539
:10AF9400540383274A973E953E2163833701829465
:10AFA4000504C9BF8280B737002003C6479DB73761
:10AFB400002083A74797C166014589070147FD160D
:10AFC40091456313E600828003D807006309D80023
:10AFD40003C8A7006315B80005051375F50F050729
:10AFE4001377F70F9387C703E9BFB737002003C66A
:10AFF400479DB737002083A64797014781479106AD
:10B004006310E602858393C7F7FFC207C183054532
:10B014006362E50285473395A7004205418182803A
:10B024008C2299C1CE36CD8F05071377F70F9386FF
:10B03400C603F9B793F61700F1FE0505858313756A
:10B04400F50FF9B7797156CAAA8A2E8526D24AD045
:10B054004ECE52CC5AC85EC662C406D622D4AE8442
:10B06400328B368CBA8B3E8AC28946899760FA1F26
:10B07400E78040A23DED41657D159760FA1FE780AA
:10B0840060A12A84554531C81946DE85130564003C
:10B09400A30284019750FA1FE780A0298357010374
:10B0A40026A0230264013EA88357410323005401D0
:10B0B400232604025EA8230644012317340123181F
:10B0C4002401EFF09FF20AB8232A04022685232CD8
:10B0D40004028145EFF03FB40145B250225492542A
:10B0E4000259F249624AD24A424BB24B224C456160
:10B0F40082804545DDB7B737002083C6479DB73703
:10B10400002003A7479781476395F60041657D15A5
:10B1140082803A861307C703835547FF6394A500CB
:10B124002A228280850793F7F70FF9BFB7370020EB
:10B1340003C8479DB737002083A647974166014758
:10B144007D16954811436314E80001458280BE22B0
:10B154003685638EC702CC5A9DC9BC31AC2189CDDA
:10B16400938597FD93F5F50FE372B3FE9387D7FAB2
:10B1740093F7D70F89EF82809385F7FD93F5F50F49
:10B18400E3F6B8FC9387D7FA93F7D70FE1D3050713
:10B194001377F70F9386C6037DB7B737002083C5AF
:10B1A400479D4166B737002003A747977D1681471F
:10B1B40025486394F5000145828036233A85638BE4
:10B1C400C600545B81CAB4329386E6FD93F6F60F4B
:10B1D400E374D8FE850793F7F70F1307C703D1BFAE
:10B1E400011122CC2A84494506CEEF80EFB21DC15D
:10B1F4002AC622859760FA1FE780C08901CD624480
:10B20400B737002032460E39F24003C5F79C05617A
:10B214006F501FB4F24062440561828039714ED68A
:10B2240052D4AE892A8A93053005414526DA4AD894
:10B2340056D206DE22DC32C63689BA8A9750FA1F05
:10B24400E78000E0CD4429C92A8489446381090444
:10B2540032468145F08241469750FA1FE780001438
:10B264005686CE8522859750FA1FE780800C2146AA
:10B27400630E0902CA8528089750FA1FE780600BFD
:10B28400A28650082C085285EF30700FAA842285BC
:10B294009750FA1FE780C0E7F2506254268542595E
:10B2A400D254B259225A925A216182808145280887
:10B2B4009750FA1FE780800EE1B7411122C440592C
:10B2C40026C206C6AA8429CC085409C59750FA1F79
:10B2D400E78000E4285809C59750FA1FE78040E347
:10B2E400685809C59750FA1FE78080E2285C09C5B1
:10B2F4009750FA1FE780C0E1685C09C59750FA1FB0
:10B30400E78000E10325040809C59750FA1FE78088
:10B3140020E022859750FA1FE78080DF23AA0402E9
:10B324002244B73700208E38B240924403C5F79CBC
:10B3340041016F50FFC9411126C206C622C4AE8422
:10B344009750FA1FE780007529C14C592A8495CD7E
:10B3540083A8C50703A88507FC59B859F42192218D
:10B36400AC212685EF804FA32285EFF01FF5EFF087
:10B37400DFE201CD2244B7370020B240924403C536
:10B38400F79C854541016F50CFFEB2402244924460
:10B3940041018280011122CC06CE2A842EC6975008
:10B3A400FA1FE780206F5C5989CF9E23B245639AC8
:10B3B400870085476397F5006244F24005616FF0AA
:10B3C400DFEFF240624405618280411106C622C467
:10B3D40026C2EFF0BFD529C14059AA8415CC3C2020
:10B3E4009DC7B737002083A7C79A89C7DC4399C391
:10B3F4002285829738309307F002631FF7002244B6
:10B40400AA20B2409244814541016FF0DFF2B73780
:10B41400002083A7879AD1BFB240224492444101BD
:10B424008280411126C24AC006C622C4AA842E893B
:10B434009750FA1FE780006605CD405955C41E2079
:10B444006394970A3C30130710026395E7083C2085
:10B45400ADCF7C5403270408DE2B15E313F7170044
:10B4640019CF18545A23058B19CB930720023CB0EB
:10B47400B24022449244024905454101828013F7B7
:10B48400270001CB18545A23098B01C793074002A4
:10B49400F9BF918B81CB1C54DE23918B81C7930719
:10B4A4006002F1B7B737002083A7C79AF1D3DC4312
:10B4B400E1D32285829738309307F0028145E3195E
:10B4C400F7FA2685EFF03FE765B7B737002083A783
:10B4D400879AE9BF1307A0026398E7006304090091
:10B4E40013092003CA85F1BF631C09002685975000
:10B4F400FA1FE780205A09C55C2193E707015CA184
:10B50400A6854A85EF705FA4A5B7797126D29947BD
:10B51400EC85AA842E858D4522D406D632C636C43F
:10B52400FC84EFE0EFBB2ACE4D441DC13246A24657
:10B53400AA85328582962A8419E52C082685EFF09F
:10B544008FB62A8411C572459750FA1FE78040BC14
:10B554002685EFF0FFC82285B250225492544561EB
:10B5640082804111B7D6050022C42E862E8493868C
:10B5740086CE894506C626C24AC02A89EFF0FFF85E
:10B584000C20AA844A85EFF01FDBB24022442685B2
:10B594000249924441018280B737002083A7879AE9
:10B5A40085CB9C4395C71D71A2CC86CE98411008CB
:10B5B4002A843AC8D84185453ACA829711C5488633
:10B5C4002A206C00EFF0FFF9F64066442561828082
:10B5D4008280AE8711CD785501CF142394A1143302
:10B5E40094B1342BB4A1142F584BB4B1D8C1828078
:10B5F400414681453E851753FA1F670023DAB73762
:10B60400002083A7C79A91C703A38700630303009D
:10B6140002830945828037370020032707BA1DC7F4
:10B624005843AA8705450DC703A50708411106C657
:10B63400930605021306050C930505061305050478
:10B644000297B2401375F50F41018280054582804F
:10B6540082804DC9357122CD2A840A2126CB4AC95C
:10B664004EC756C306CF52C55AC1DEDEB68AB2896A
:10B674002E899750FA1FE780E041AA8431C50C183F
:10B684002285EFF01FF53C20138A6400A9CBEF70EC
:10B694000FE62A8B014583CB5400EF704FE3AA8455
:10B6A4000C100818EF10A04708542C10EF10C047D6
:10B6B400D288268A56C05E88D2875A8714103010E2
:10B6C400CE854A85EF20606FFA406A44DA444A49DD
:10B6D400BA492A4A9A4A0A4BF65B0D618280EF7096
:10B6E4000FE1AA8B014503CB5400EF704FDE2ACE45
:10B6F40008540C10EF10A0422C100818EF10C04290
:10B70400F2484DBF8280C14719C91455C14781CA47
:10B71400785511C7BC32BD4663F3F6001C2F3E8535
:10B724008280894779C9F1C9411106C622C426C25B
:10B734001C312E849CA13C219CB13C31BCA15C21D8
:10B74400BCB15C31858B93968700DE2193F7F7EFCC
:10B75400D58FDEA1543193F7F7DFA20693F60620C6
:10B76400DD8ED6A1583193F6F6BF22071377074032
:10B77400558FDAA15C31FD769386F67F8D87858BB4
:10B78400758FAE07D98FDEA17421F99B858ADD8E72
:10B79400D6A178219377270013F7D6FF5D8FDAA11E
:10B7A4007C2193F647009377B7FFD58FDEA17821EC
:10B7B400DD9B4D45218BD98FDEA1EF70FFD5AA8487
:10B7C4005145EF707FD5383093F4F40FC947636067
:10B7D40097021375F50F636CE50014201147E147D8
:10B7E4006367D700143005476363D7008147B240CD
:10B7F400224492443E85410182803E85828015C167
:10B80400AA8709458DC141112E85414693851700AC
:10B8140006C69750FA1FE780C0B1B2400145410106
:10B82400828009458280828089470DC585C5411182
:10B8340006C61831AE87194698A1930525001385CD
:10B8440017009750FA1FE780C0AEB24081473E858B
:10B85400410182803E85828015C1AA8709458DC138
:10B8640041112E8541469385170006C69750FA1F4D
:10B87400E78020ACB24001454101828009458280C5
:10B884008280894705C99DC5411106C638211431F6
:10B89400AE872207558F9AA121469305350013855B
:10B8A40027009750FA1FE780C0A8B24081473E8521
:10B8B400410182803E85828015C1AA8709458DC1D8
:10B8C40041112E8541469385170006C69750FA1FED
:10B8D400E78020A6B240014541018280094582806B
:10B8E4008280894709C981C91831BD46E14763E4AB
:10B8F400E60098A181473E85828015C1AA87094543
:10B904008DC141112E8541469385170006C6975077
:10B91400FA1FE78000A2B240014541018280094537
:10B924008280828015C1AA8709458DC141112E8567
:10B9340041469385170006C69750FA1FE780609F1B
:10B94400B2400145410182800945828082801DC147
:10B95400AA87094595C141112E85130600049385D4
:10B96400170006C69750FA1FE780A09CB240014515
:10B974004101828009458280828015C1AA870945D8
:10B984008DC141112E8541469385170006C69750F7
:10B99400FA1FE780009AB2400145410182800945BF
:10B9A400828082801D71A2CC2A84084586CEA6CAD4
:10B9B40023060100042135479387F4FF93F7F70F1B
:10B9C4006364F70C37E706008A071307C7CFBA97F3
:10B9D4009C4382870C08EFF0DFD4C9476310F5025B
:10B9E40099475C862A206C00EFF0BFB7F6406644A6
:10B9F400D644256182800C08EFF01FEC31C51C860B
:10BA0400F5F32A20EFF0CFFDD5B70C08EFF0FFEEE9
:10BA1400F5B70C08EFF0FFECD5B70C08EFF03FDEFC
:10BA2400F1BF0C08EFF0FFE5D1BF0C08EFF0DFE247
:10BA3400F1B70C08EFF05FDFD1B70C08EFF09FEE21
:10BA440075BF1C312308F1002A209750FA1FE780A4
:10BA54006004A14705C15825631AF702B7370020CF
:10BA640003A7C79A9D4719C7184309C71008A68595
:10BA74000297AA875C8661B70C08EFF05FEDBDBF43
:10BA84000C08EFF09FEF9DBF9D47A1BFB737002083
:10BA940003A7879AC1BF011122CC06CE26CA4AC881
:10BAA4004EC61821930720092A846313F7121C3108
:10BAB40039476393E70A5621096761078147639110
:10BAC400E610B739002003A5C99BCE84630A050E8E
:10BAD4000C4403C90500631E09001C218505214689
:10BAE400A9CF29059750FA1FE780A08483A7C49B98
:10BAF400B5C349459740FA1FE780E0732A840DC512
:10BB0400930710FC1CA1A300250183A5C49B090570
:10BB1400414689059750FA1FE780A08183A7C49BFB
:10BB2400A2858833EF40DFD003A5C49B9740FA1F5A
:10BB3400E780005E23AE049A31A809059740FA1FF6
:10BB4400E780207FEF30600305494DF183A7C99B4F
:10BB5400238027018547ADA01307E0036398E70816
:10BB640038219547631CF7024A21EFF0CFB691477D
:10BB7400E312F5FEB737002083A7879AE1DF03A31A
:10BB84008700E30903FC72244A209305640062449D
:10BB9400F240D2444249B24905610283A147631C81
:10BBA400F7006C204A206244F240D2444249B24930
:10BBB40005616FF01F87930600038147E303D7FEF7
:10BBC400F2406244D2444249B2493E8505618280D2
:10BBD4009306000A8147E315D7FEEFF0BFDC084463
:10BBE40035D99740FA1FE780A052ADB78147C9BF46
:10BBF400011126CA06CE22CC89440DCD85CDAA8456
:10BC04002E8468008D45EF601FE01C872685228600
:10BC140093F7F70393E707046C005C87EF20E010C9
:10BC2400AA8409E90D466C00130534009740FA1FF5
:10BC3400E7802070F24062442685D2440561828008
:10BC44005D714EDE86C6A2C4A6C2CAC052DC56DAF4
:10BC54005AD85ED6894945CD5DCA138B4500420B3F
:10BC6400135B0B01AE8A2A8A930530055A85B28488
:10BC74009740FA1FE780C03C2A84CD4949C9EF7038
:10BC8400EF882A895686D285935A8900135A090166
:10BC9400937BF90F1305440093FAFA0F137AFA0F02
:10BCA400135989019740FA1FE780207EA30174018C
:10BCB40023015401A300440123002401EF706F8485
:10BCC400AA85414608089740FA1FE780007C21476F
:10BCD40034005A86A2850808EF20A02BAA891DE10A
:10BCE40021462C0023807401A38054012381440144
:10BCF400A3812401138544009740FA1FE780E0786C
:10BD0400EF708F8122859740FA1FE7806040B6402C
:10BD140026444E8596440649F259625AD25A425BE9
:10BD2400B25B6161828001114AC82A892E8506CEE0
:10BD340022CC26CA2EC69750FA1FE780A0D55DCD27
:10BD440040595DCC5C300947B24593F6B70F638721
:10BD5400E60011471305E00F639DE7061E20094521
:10BD64006399B706930484004146CA8526859740A3
:10BD7400FA1FE780005C4146CA8513058401974099
:10BD8400FA1FE780005B383085469307F7FE93F788
:10BD9400F70F63E6F6041306C4033285C14532C6C1
:10BDA400EF607FC632469306C402A6852285EFF073
:10BDB4005F8A3C2089CB22856244F240D2444249C6
:10BDC40005616F00707A3830C947E306F7FE3CB06E
:10BDD4000145F2406244D24442490561828093079E
:10BDE40010050145E317F7FE3C20E5D722856244A0
:10BDF400F240D244424905616F00507D0945D1BFEC
:10BE04004945C1BF39C9011126CA06CE22CCAA842C
:10BE140009459DCD0D4628002E848D059740FA1FB7
:10BE2400E78020511C8570002C0093F7F70393E7FB
:10BE3400070426855C85EF10506F19E90D46A2852D
:10BE440068009740FA1FE780C05F7D153335A00076
:10BE5400F2406244D2440561828009458280011126
:10BE640052C42A8A32854EC656C25AC006CE22CC45
:10BE740026CA4AC82E8BB28AB6899750FA1FE78021
:10BE840060C109ED8944F240624426854249D244A6
:10BE9400B249224A924A024B056182805C592A893E
:10BEA400C544F5F34D45EF702FE71374F50F514575
:10BEB400EF708FE6E38809FC83C78901E3E487FC1C
:10BEC4001375F50FE360F5FC930530051305400881
:10BED4009740FA1FE780C016232AA9022A84CD447A
:10BEE4005DD11306400881459740FA1FE780004B57
:10BEF400A30104002301440123026401231054011B
:10BF04002326340723240402A30204008144E30CFF
:10BF14000AF62285EF00905FAA8435D54A85EFF0B2
:10BF2400CFB995B7397122DC06DE26DA4AD84ED667
:10BF340052D456D25AD05ECE62CC66CA0944630D3E
:10BF44000610630B0710AA8B3A89368BB28A2E8CA3
:10BF54009750FA1FE78000B42A8A5144630E050EF5
:10BF64009305300541459740FA1FE780600DAA8983
:10BF74004D447DC18344190083472900A204C207AC
:10BF8400BE9483470900BE9483473900E207BE94F8
:10BF940083278A0263E697007D5709446399E70A79
:10BFA40063070C0083474A000544898BCDC3930C77
:10BFB4004B00214681450A85C20C9740FA1FE78051
:10BFC400E03D93DC0C019305300566859740FA1F2C
:10BFD400E78000072A8C4D443DC95A86D685110551
:10BFE4009740FA1FE780604A1146CA8562859740E8
:10BFF400FA1FE7808049414693058A014E859740A0
:10C00400FA1FE780804821478A866686E2854E8546
:10C01400EF1030782A841DE521468A852800974050
:10C02400FA1FE7808046214693054900280097407F
:10C03400FA1FE78000418547631EF502A6855E85E9
:10C04400EF705F8462859740FA1FE780600C4E852D
:10C054009740FA1FE780C00B2285F2506254D254F5
:10C064004259B259225A925A025BF24B624CD24C58
:10C07400216182800544F9B779719397050122D42F
:10C0840006D626D24AD04ECEC1872E8463D5070465
:10C09400B73400209384C49CA8309740FA1FE780EB
:10C0A400E01E2AC609CDEFF01F9FB24511E5A82076
:10C0B4009307F00F631EF5002E85EF408FF2216584
:10C0C400218DB250225492540259F2494561828022
:10C0D400EF400FF6EDB793F7150091C7EFF0EFAE11
:10C0E40013451400F9BFA1E10145E1BF850493F4B0
:10C0F400F40FEFE05FD6E3F9A4FE3395990013192A
:10C10400050113590901B3772401EDD34A85EFE002
:10C114009FFEC167FD176305F500DD45EFF0AFA194
:10C124003345240179BF85448549E1B7B7370020F9
:10C1340023AE079AB737002023A6079A37C705000E
:10C14400B73700201307876C23A4079AB73700205A
:10C1540023A0E79C37C705009387079C1307674113
:10C16400D8C337B705001307072298C737D7050088
:10C17400B73700201307E75423A8E79A37D70500F9
:10C184009387079B1307C70FD8C337D70500130737
:10C19400C73998C78280B737002083C7079D918B22
:10C1A40089C7B73700209387079B3737002023249C
:10C1B400F79A01458280011106CE2AC6EFF01FF7D7
:10C1C4003245B73700209945A387A79CEFD0EFEB02
:10C1D400F24037B505001305853905616FE05FC886
:10C1E4001C5581C7A1473E858280011122CC26CAF5
:10C1F4002A84AE84130500049305300506CE9740C7
:10C20400FA1FE780E0E308D475C113060004A6858D
:10C214009740FA1FE780E01178543C2B93F687008F
:10C22400F5CA1454B422A18AF5C683270408DDEFA5
:10C2340093053005130500109740FA1FE78040E08E
:10C244002320A4088D4745C5A302040078549C30DC
:10C25400143391EB91EABC20918BC5E33C2B918B79
:10C26400C9EF854701A881C6214758B089C75C300A
:10C2740093E707015CB06C54BC29858B99CB1C54A3
:10C284000547BC238D8B6396E7007C2093E717005A
:10C294007CA08327040889C77C2093E787007CA0BF
:10C2A4005C300547639EE70A930484004146814558
:10C2B40026859740FA1FE780600E414681451305A5
:10C2C40084019740FA1FE780600D1306C40332858A
:10C2D400C14532C6EF602FF3832704083246B9CF35
:10C2E4002285EF00B02E9307000525C5A147F24033
:10C2F4006244D2443E85056182809C201423154704
:10C30400B387E70237E70600130707D5BA97B6974E
:10C314009C238DB7943089C6143399C2E14799BFE1
:10C32400B420D58F918B95DF9C2014231547B387B8
:10C33400E70237E70600130747D3C9BF22859306F0
:10C34400C402A685EFF0EFB02285EF00F02159FD7D
:10C35400C1470A203CB08145EF70EFBC814741BF23
:10C3640013F7870135CFC18B930484004146B1C7CD
:10C37400890526859740FA1FE780A0FB4146814541
:10C38400130584019740FA1FE78040017C201306BF
:10C39400C403328593E747007CA0C14532C6EF60F1
:10C3A4008FE683270408324685C32285EF001022D6
:10C3B4009307200505FD3CB055B781452685974078
:10C3C400FA1FE780A0FD5DBF9306C402A6852285FF
:10C3D400EFF02FA82285EF003019CD4769DD39B77A
:10C3E400094785456388E70093F7D70F114763969C
:10C3F400E70089450A20EF700FB37C2093E74700DC
:10C404007CA08327040881C7930710056DB7C5472F
:10C414005DB73C21638B0722797122D406D626D2DC
:10C424004AD03C31130750052A84639DE70603492B
:10C4340075001306C503C14593573900AA97328581
:10C44400842732C6EF602FDCB737002083A707BAF2
:10C45400A1C79C47B1C30325040893767900B3D6DA
:10C46400D4403246858A93050504180893E60608E5
:10C474001305050882971375F50F19ED41460C084D
:10C484001305C4029740FA1FE780A0EA2285EF0053
:10C49400B00D930760053CB0B25022549254025937
:10C4A40045618280130710026392E7021C5503273B
:10C4B4000508DE2361E313F707104DCF78555A2B97
:10C4C4001377071045CB930770023CB03C30130739
:10C4D40070026397E70C3C5885E39305300571457A
:10C4E4009740FA1FE780C0B528D819C57146814521
:10C4F4009740FA1FE78080EA2458B1C4BC2C89E72E
:10C504002285EFF04FA0A8AC2858814541469740BA
:10C51400FA1FE780A0E828583D472C2D9387F5FFA4
:10C5240093F7F70F6364F700EF60EFCDEF404FCA66
:10C534003C58A1458AAB13852701EF60CFCC2C581A
:10C544000A20EF00B031930780020A203CB09740E4
:10C55400FA1FE7802054414609C57E2513D61700EB
:10C564003E96B737002003C5F79C06068545EF4085
:10C574002FFE1DB713F7072009CB78545A2B1377D6
:10C58400072001C79307900289B793F707409DDFFF
:10C594007C54DE2B93F7074095DB9307B00235B745
:10C5A400130780026397E7023C5899C78E2B0A2031
:10C5B40013862701EF00F02F1C54DE2313F7072006
:10C5C40029CF78545A2B1377072021CB9307900255
:10C5D400ADBF13079002639BE700EF60EFF1AA85FC
:10C5E4000A20EF00102C9307A00285B71307A002BE
:10C5F4006390E704EF60AFEFAA8585470145638444
:10C60400F500814505452EC6EF606FEC2A86B245DC
:10C614000A20EF00B0251C54DE2393F707409DC386
:10C624007C54DE2B93F7074091CF9307B00231BFC0
:10C634001307B0026398E700EF60AFECAA850A2005
:10C64400EF00902A9307F002B9B58280411122C409
:10C65400405926C206C67C54AA84DE2B13F7071061
:10C6640011C718545A23137707100DE313F7072043
:10C6740011C718545A231377072009EB93F707407F
:10C684008DCB1C54DE2393F7074085C79307100214
:10C694003CB02285EFF0FFD738309307F002631ED9
:10C6A400F7002244AA20B2409244814541016FE040
:10C6B4009FC89307F0023CB0EDB7B24022449244C5
:10C6C40041018280397122DC405926DA4AD84ED69B
:10C6D40006DEAA89AE8432896302043A2A211E2026
:10C6E4006384A700A14421A03C2091EB9D44F25017
:10C6F400625426854259D254B2592161828093876B
:10C70400E5FF93F7F70F2D47E362F7FE37E70600DF
:10C714008A071307C7D6BA979C438287B2852285B6
:10C72400EFF01FACAA84E1B74146CA851305C404DF
:10C734009740FA1FE780E0BF22858525AA8411C1AE
:10C74400A1443C30130740056396E7009307900526
:10C754003CB071BF130760056395E7009307A0051C
:10C76400C5BFD147F5B79309C4054E854146CA856F
:10C774009740FA1FE780E0BB0325040845C53C3019
:10C78400130790056398E70022854D259307E0057C
:10C794003CB079A01307A0056390E7087C3013D759
:10C7A4003700229714279D8BB3D6F640B737002065
:10C7B40083A707BA858A93E606F893F6F60F9DD306
:10C7C4009C478DD39305050818084E861305050468
:10C7D40082979374F50FE39704F041460C08130510
:10C7E400C4049740FA1FE780C0C57C304D478507D5
:10C7F40093F7F70F7CB06377F7002285052D930735
:10C80400E005B9B7B737002003C5F79C8545EF406D
:10C814004FB6930750052DBF1307C005E386E7F60F
:10C824008144F1B5130984004E86CA852285140813
:10C83400EFE03FE241469305C40408089740FA1F1D
:10C84400E78020C0E30505EA8A861306C403CE8583
:10C854004A85EF10A06A05E12285EFE0DFEAB737E9
:10C8640000202A8783A7879C0A20814601468A855F
:10C874008297AA8411C1A14493072002D1BD0C223E
:10C88400EFE07FAB71BF383093072002E310F7E687
:10C894007C5889EB9305300571459730FA1FE78082
:10C8A400207A68D86858E30305E44146CA8597406E
:10C8B400FA1FE78000A864582285EFE0DFE4A8AC03
:10C8C40093073002F1B5383093073002E310F7E2F2
:10C8D4001E2268582146930529001EA94905974040
:10C8E400FA1FE78000A57C54DE2B13F727002DC721
:10C8F40018545A23098B2DC39307400251BD383075
:10C9040093074002E314F7DE3C5C81EB85455D450B
:10C914009730FA1FE780C07228DC285CE30205F038
:10C92400834709004146CA857CA99740FA1FE780DE
:10C9340040A093075002A9BD383093075002E31773
:10C94400F7DA285C19469305190041059740FA1F48
:10C95400E780209E7C54DE2B918B95CF1C54DE23E4
:10C96400918B95CB9307600225B57C5C89EB93058D
:10C97400300551459730FA1FE780806C68DC685CAD
:10C98400E30205D64146CA859740FA1FE780609ABC
:10C994007C5C7D5798CB4E85EFF05FCB51B503257A
:10C9A400040813060004CA85130505049740FA1FFA
:10C9B400E78020982285EFE01FC63C30130700056E
:10C9C4006395E70093074005E1B313071005639CE3
:10C9D400E700B737002003C5F79C8545EF406F9902
:10C9E4009307500575B313072005E39BE7E2B737B8
:10C9F400002083A707BAE38707CE9C47E38407CECA
:10CA04008325040893048400180893850508814647
:10CA140026862E8582970A201008A685EF609FD966
:10CA24009307B005B5B338309307E005E310F7CCAE
:10CA34008325040841464A859740FA1FE78060A091
:10CA4400AD44E30605CA032504084146CA85974058
:10CA5400FA1FE780008E2285EFE0FFCAB737002077
:10CA64002A8783A7879C2C580A20814601468297EF
:10CA7400AA8411C1A14493071002D9B9AD47E39127
:10CA8400F5DA14222E21130665000821EF60AFDCCD
:10CA940041BB894759C2D1C108A29C211CB29C3117
:10CAA4003CA2BC213CB2BC31A30206005CA2DE2144
:10CAB400A183858B5CB2DA211377072001C793E742
:10CAC40027005CB2DE2193F7074089C75C3293E705
:10CAD40047005CB2DE2113974701635607005C32BE
:10CAE40093E787005CB223030600DC21858B7CA2DC
:10CAF400DA21098B01C793E727007CA2DE21918B01
:10CB040089C77C2293E747007CA2DA218147218BE5
:10CB140009C778221367870078A23E8582802E8613
:10CB2400AA8505456FF0FFF62E86AA8509456FF0A4
:10CB34005FF6894785C51DC1411106C6AE870D47FD
:10CB4400AA8598A31385170041469730FA1FE780FA
:10CB5400407EB24081473E85410182803E8582808D
:10CB6400894785C51DC1411106C6AE871147AA85EF
:10CB740098A31385170041469730FA1FE780607B1E
:10CB8400B24081473E85410182803E85828089474B
:10CB940085C51DC1411106C6AE871947AA8598A34C
:10CBA4001385170041469730FA1FE7808078B2401A
:10CBB40081473E85410182803E858280894795C9AF
:10CBC4000DC9411106C61D4798A11A21AE872146F9
:10CBD40098B11A212183B8A1930525001385370044
:10CBE4009730FA1FE780E074B24081473E854101E7
:10CBF40082803E858280894785C51DC1411106C654
:10CC0400AE872147AA8598A313851700414697301C
:10CC1400FA1FE7800072B24081473E85410182805D
:10CC24003E85828089479DC515C5411106C62547A5
:10CC340098A11821AE87194698B19305150013855C
:10CC440027009730FA1FE780C06EB24081473E85C7
:10CC5400410182803E858280894785C51DC141117D
:10CC640006C6AE872947AA8598A3138517004146AF
:10CC74009730FA1FE780E06BB24081473E8541015F
:10CC840082803E85828089478DC505C5411106C6CF
:10CC9400AE873147AA8598A31385170013060004AD
:10CCA4009730FA1FE780E068B24081473E85410132
:10CCB40082803E858280894785C51DC1411106C693
:10CCC400AE873547AA8598A3138517004146973048
:10CCD400FA1FE7800066B24081473E8541018280A9
:10CCE4003E858280894799C511C595479CA11C2121
:10CCF4009CB181473E858280894799C511C5AD475E
:10CD04009CA11C219CB181473E8582800DC55D712B
:10CD14008A8586C6A2C42A84EFE0BF8B0A20B7D6D0
:10CD240005000A86938626B29D45EFE00FFEB640C5
:10CD3400264461618280054582800DC55D718A85C6
:10CD440086C6A2C42A84EFE0DF880A20B7D605008D
:10CD54000A869386C6B29D45EFE02FFBB640264473
:10CD640061618280054582805D71A2C49305C5021C
:10CD74002A8441460A8586C69730FA1FE780605B9D
:10CD84000A20B7D605000A86938666B3C545EFE048
:10CD9400CFF7B6402644616182805D71A2C49305D9
:10CDA400C5032A8441460A8586C69730FA1FE78060
:10CDB40040580A20B7D605000A86938646B6C5456C
:10CDC400EFE0AFF4B640264461618280B7370020BB
:10CDD40083A707BAA9CB9C435D71A2C486C62A84E3
:10CDE4001305E00F8DCF032504089305050C1305E7
:10CDF4000508829783250408130600040A85938591
:10CE040005089730FA1FE780C0520A20B7D60500FC
:10CE14009386A6C80A8693051004EFE00FEFB64088
:10CE24002644616182801305E00F8280317122DD26
:10CE34002A840A2126DB06DF4AD94ED752D556D397
:10CE44005AD15ECF62CD9740FA1FE780A0C43C5808
:10CE5400AA8489EB9305300571459730FA1FE78062
:10CE6400201E28D82858CD4705C9714681459730DA
:10CE7400FA1FE780A052032904072285EFE0BF8848
:10CE8400230DA9003C203739002063810712832732
:10CE940009BA85E39307E00FFA506A54DA544A5901
:10CEA400BA592A5A9A5A0A5BFA4B6A4C3E85296146
:10CEB400828083AB0701E38F0BFC032B0408EF5044
:10CEC4001FE32A8C0145EF509FE0DC303858130BE8
:10CED4000B029309C403130AC405938A64003AC07D
:10CEE400B337F0002A87930801045688B3368001CB
:10CEF4005286CE855A85829B1C54B8232307E102AF
:10CF04009833A306E1029C232306F102832709BA7E
:10CF1400D1D303AB4701E30F0BF6DC30B337F0009A
:10CF24003ECEEF50DFDCAA8B0145EF505FDA0327DA
:10CF34000408F2472AC03AC2B33870015688781000
:10CF4400930684004E86D2858800029B7C54B82BBD
:10CF54002305E1029833A304E1029C232304F10294
:10CF6400832709BA03A94701EF507FD82A8B0145CB
:10CF7400EF50FFD583C854009C082A883EC2B338BA
:10CF84001001B33760013810930684015286CE85B0
:10CF940056C0880002990A20B7D605009386A6CB0E
:10CFA4009008C545EFE06FD6AA87FDB5D430832736
:10CFB40009BA032B0408B336D00083AB070136CE7D
:10CFC400EF50FFD22A8C0145EF507FD03C58F246F7
:10CFD400130B0B02130AC4059309C403938A640058
:10CFE4002A88930801044E86D2853EC05687B337FB
:10CFF40080015A85829B1C54130B0103B823230719
:10D00400E1029833A306E1029C232306F10283275D
:10D0140009BA83AB4701DC30B337F0003ECEEF50A2
:10D024001FCD2A8C0145EF509FCAF2472AC0B3385E
:10D03400800156887810930684004E86D2855AC2A1
:10D044008800829B8325040841465A859730FA1F3D
:10D05400E780203FAD47E31B05EE3DBDB7D6050095
:10D064002E86938626B9C5456FE02FCA5D71B287B7
:10D07400A2C44C802A84BE8513051100194686C6B5
:10D084009730FA1FE780E02AB7D605000A86228582
:10D09400938686C2A145EFE04FC7B640264461613E
:10D0A4008280B7D605002E869386A6BFC5456FE05D
:10D0B400CFC55D71B287A2C46C802A84BE85130576
:10D0C4002100214686C69730FA1FE7808026B7D60E
:10D0D40005000A862285938606BCAD45EFE0EFC2C3
:10D0E400B640264461618280B7D605002E869386B9
:10D0F400C6C5C5456FE06FC1797122D406D626D264
:10D104003C31130730052A846381E708130750056F
:10D114006392E7089307A0053CB17C31C14513D75E
:10D1240037002A9714279D8B1305C503B3D6F64001
:10D13400858A93E606F893F6F60F36C6EF50BF8C51
:10D14400B246B737002083A707BA9DCB9C478DCB47
:10D154000325040818081306C403930505041305DE
:10D16400050882971375F50F01ED1305C4024146B6
:10D174000C089730FA1FE780C01B2285EFF0DFBE52
:10D18400B2502254925445618280930790053CB179
:10D19400814645BF130710026391E7027C550327BC
:10D1A4000508DE2B61EF13F7170069CB18555A23D6
:10D1B400058B69C7930720023CB03C30130720025B
:10D1C4006394E70E3C5889EB93053005714597301D
:10D1D400FA1FE780E0E628D82458ADCC2285EFE09A
:10D1E4008FD2A8AC2858814541469730FA1FE78072
:10D1F400E01A28583D472C2D9387F5FF93F7F70F36
:10D20400636DF702B737002083C7B7BAD9CB41465D
:10D21400814508089730FA1FE7804018B735002089
:10D2240019469385C58908089730FA1FE78060106E
:10D2340030580C082E85EF80302AEF306FF93C58B7
:10D24400A1458AAB13852701EF50EFFB2C580A2028
:10D25400EFF0DFE0930730020A203CB09740FA1F5A
:10D26400E7804083414611C17225B737002003C5CA
:10D27400F79C06068545EF30BFAD19B713F72700B5
:10D2840001CB18545A23098B01C7930740022DB7C9
:10D29400918B85D71C54DE23918B85D39307600231
:10D2A40021BFEF504FF651BF130730026396E702D8
:10D2B4003C5899C78E2B0A2013862701EFF07FDF95
:10D2C4007C54DE2B13F7270021CB18545A23098BE7
:10D2D40021C79307400249B713074002639BE70045
:10D2E400EF509FA1AA850A20EFF0BFDB93075002FD
:10D2F400A5B713075002639DE702EF505F9F15E542
:10D30400814505452EC6EF509F9C2A86B2450A20CA
:10D31400EFF0DFD57C54DE2B918B8DC71C54DE23BC
:10D32400918B8DC39307600205BF85450145D9BF25
:10D33400130760026398E700EF50BF9CAA850A2098
:10D34400EFF09FDA7C5403270408DE2B09EF13F770
:10D35400071011CB18545A231377071009C79307E2
:10D3640070023CB031BD13F7072009CB18545A237F
:10D374001377072001C793079002E5B793F7074097
:10D3840089CB1C54DE2393F7074081C79307B0026F
:10D39400C9BF9307F002F1B7397122DC26DA4ED601
:10D3A40052D406DE4AD8AE89328AAA849730FA1F4C
:10D3B400E780406E4059414681450A859730FA1FFF
:10D3C400E780C0FD35C4035904006313990638305F
:10D3D40093071002631FF7028327040899CF2C5880
:10D3E400A1C94A85EF10607A0545F2506254D254BF
:10D3F4004259B259225A216182808A861306C40591
:10D404009305C40313058400EF00502F15E18A85AA
:10D41400C9BF2C5891CD9E29639C47012146C9055B
:10D424004E859730FA1FE780C00119C12C5855BFAB
:10D4340026859730FA1FE780E0652A84054555D490
:10D444004C54B1C59E29639447052146C9054E85B0
:10D454009730FA1FE780E0FE8547631AF502B72785
:10D46400002083C7F75489C74C54BC3D639AA70C6A
:10D47400BD452685EF10206CB737002083A7C785EC
:10D484000145A5D71D45894582970145B9BFB737E1
:10D49400002003C7C7BAB739002093898982058B56
:10D4A4003E8929C3B7370020583083C747BA631B66
:10D4B400F702B73500201946938555BA1305640061
:10D4C4009730FA1FE780E0F78547631DF50083A7CF
:10D4D400490381C791451D458297BD452685EF10B7
:10D4E400806519B7373700200347B7BA83A74903C4
:10D4F40031CB0347C9BA098B09CB81C795451D4573
:10D5040082972685EF10A068C5B581C78D451D4556
:10D5140082974146814508089730FA1FE78000E862
:10D52400B735002019469385C58908089730FA1F36
:10D53400E78020E00C082E850A86EF80E0798A8552
:10D5440026854DB58545C5FF6DBF797122D44059F7
:10D554004AD04ECE52CC06D626D2AA892E8A3289F9
:10D56400630A04622A211E20638CA700A144B250DE
:10D574002254268502599254F249624A45618280B6
:10D58400242099C09D44E5B79387F5FF93F7F70FDF
:10D594003147E369F7FE37E706008A071307C7D95F
:10D5A400BA979C4382871C54F1F393053005130505
:10D5B40000049730FA1FE780A0A808D445D9034790
:10D5C4000900914763F4E7008D4455B703471900F8
:10D5D4008547E3EBE7FE13060004CA859730FA1F7C
:10D5E400E78020D50C547054A3020400D4415C4A53
:10D5F400858AFD8E5E2AF99BD58F5EAAD841544A4E
:10D60400F59B0583058B8582F98E8606DD8E56AAE9
:10D61400DC41584AED9A8983858B09837D8F0A07FB
:10D62400558F5AAAD4415C4A5D9B8D82858A8D832D
:10D63400F58F8E07D98F5EAAD841544A93F7F7EF36
:10D644002183058BA182F98EA206DD8E56AADC41C8
:10D65400584AA583858B25837D8F9317970013F7ED
:10D66400F6DF5D8F5AAAD4415C4AA982858AA983D0
:10D67400F58F9396A7009377F7BFD58F5EAAD44111
:10D68400584AAD82858A2D83758FFD769386F67F01
:10D694002E07F58FD98F5EAA3C2A03250408A18B97
:10D6A400FDC3BC21A18BE5C3E31205EC9305300552
:10D6B400130500109730FA1FE78080982320A408F0
:10D6C40001D57C54A302040003471900943399E65E
:10D6D40041C75C3093E707015CB021A0A1475CB06F
:10D6E4006DFB2285EFF06FE56C54BC29858B89CBEB
:10D6F4001C54BC238D8B89C77C2093E717007CA026
:10D704008327040889C77C2093E787007CA05C30CA
:10D714000547639BE70A414681451305840097301A
:10D72400FA1FE780A0C7414681451305840197305D
:10D73400FA1FE780A0C6C1451305C403EF50AFAC80
:10D74400032704089307000511E3C1470A203CB0EE
:10D754008145EF505FFD21BDB82B118B19E70347BD
:10D764002900118B19E3854785BF9C231547834600
:10D774000900B387E70237E70600130707D5BA970E
:10D78400B6979C2391BF19C59730FA1FE78040983C
:10D79400232004087C54983311C70347190019C384
:10D7A400E1471DBFB82B118B09E703472900118BF3
:10D7B4005DDB9C23154783460900B387E70237E7FF
:10D7C4000600130747D365BF13F7870139CBC18B15
:10D7D40013058400414695CF89059730FA1FE780E9
:10D7E40040B541468145130584019730FA1FE7800F
:10D7F400E0BA7C20C1451305C40393E747007CA02D
:10D80400EF506FA08327040899CB930720053CB001
:10D81400B9BB81459730FA1FE78040B8D9B7CD47E7
:10D82400FDB7094789456386E70011476397E70019
:10D8340085450A20EF503FEF21A01947E38AE7FE10
:10D844007C2093E747007CA08327040881C79307C3
:10D85400100575BFC54765BF4146CA851305C40495
:10D864009730FA1FE780E0AC3C3013076005639CF7
:10D87400E700B737002003C5F79C8545EF306FAF4D
:10D884009307500569B745476383E7029306C402CB
:10D894001306C403930584002285EFD09FDB228501
:10D8A400EFF08FCCAA8411C1A144D1478DB7C947E9
:10D8B400B9BF9309C4054E854146CA859730FA1FFE
:10D8C400E78020A70325040869C53C3013079005A9
:10D8D4006398E7002285EFF04FCC9307E00505BF7E
:10D8E4001307A0056399E706B737002083A707BA93
:10D8F400E38A07C803A88700E30608C87C309305B9
:10D9040005084E8613D73700229714279D8B0A8764
:10D91400B3D6F640858A93E60608130505040298F3
:10D9240041468A851305C4049730FA1FE78060B125
:10D9340011E1D2842285EFF04FC67C30CD46130727
:10D94400E005850793F7F70F7CB063E4F60013074F
:10D95400600538B029B91307C005E39AE7C0B737A3
:10D96400002083A707BAE38F07C09C47E38C07C056
:10D9740093050508130984000A8781464A862E8583
:10D9840082970A200A86CA85EF50DFE29307B00522
:10D99400BDBD8A864E86930584002285EFD07FCB59
:10D9A40041469305C4040A859730FA1FE78060A9AD
:10D9B4008547D284E31DF5BA2285EFF00FBEAA8411
:10D9C400E31605BA9307100299B53830930770022D
:10D9D400E31AF7BA7C5889EB930530057145972013
:10D9E400FA1FE780E06568D86858E30D05B8CA8572
:10D9F40041469730FA1FE780C093032944072285E4
:10DA0400EFD07FD0230DA9009307800209B53830E9
:10DA140093078002E318F7B61E226858214693053F
:10DA240029001EA949059730FA1FE78080907C548D
:10DA3400DE2B13F7072035C718545A231377072012
:10DA44002DC393079002E1B3383093079002E31B90
:10DA5400F7B23C5C89EB930530055D459720FA1FCE
:10DA6400E780005E28DC285CE30E05B04146CA85E9
:10DA74009730FA1FE780E08B9307A00249BB383048
:10DA84009307A002E310F7B01C22285C1946930503
:10DA940019007CA941059730FA1FE78080897C54DE
:10DAA400DE2B93F70740A1C71C54DE2393F70740EE
:10DAB4009DCF9307B002A1BB38309307B002E313A4
:10DAC400F7AC7C5C89EB9305300551459720FA1F30
:10DAD400E780005768DC685CE30A05A84146CA850C
:10DAE4009730FA1FE780E0847C5C7D5798CB03D5A0
:10DAF40029008145EFD03F849DBC38309307F00462
:10DB0400E3F6E7A603250408E30205A613060004CA
:10DB1400CA85130505049730FA1FE78080812285A2
:10DB2400EFF0CFAAAA842285EFD0FFAE3C301307D2
:10DB34000005639FE700B737002003D6E90003C55B
:10DB4400F79C85450606EF30AFA093073005C1B1B9
:10DB5400130710056395E700930760054DB9130794
:10DB64002005E396E7A09307C00555B13830930725
:10DB7400E005E31DF79E032504084146CA85972066
:10DB8400FA1FE780007B2285EFF04FAAAA841DBD0F
:10DB94000C228DB785478144E39BF59C03284600FE
:10DBA4003C32382214322E2110220145EF502FC16D
:10DBB4007DBA8147C1463307F500B388F5001823C1
:10DBC40083C808003308F60085073347170123008C
:10DBD400E800E392D7FE82800147BD471308F00FA7
:10DBE4003306F5001422B388F500FD178606558F19
:10DBF4002380E800182293F7F70F1D83E39207FFB1
:10DC040082808147930800F8414893F6F70F3387E1
:10DC1400F50063FAC600B306F500942214A3850741
:10DC2400E39507FF82806395C60023001701C5BFF3
:10DC340023000700EDB701114AC856C22E89AA8AEB
:10DC440093053005414506CE22CC26CA4EC652C4A1
:10DC5400328A9720FA1FE780A03EAA8493053005F4
:10DC640041459720FA1FE780A03D2A84CD49A5C4E9
:10DC740031CD414681459720FA1FE78020722686E0
:10DC8400A2855685EF804005AA8929E1838704008F
:10DC940063D30706A2852685EFF01FF4B7E50600D7
:10DCA4004A86938505DD2285EFF0BFF083070900DE
:10DCB40063D80704A2854A85EFF01FF2B7E5060092
:10DCC4005286938505DD2285EFF0BFEE26859720E9
:10DCD400FA1FE780E04311C422859720FA1FE780EA
:10DCE4002043F24062444E85D2444249B249224A1A
:10DCF400924A05618280CA852685EFF0FFED7DB7E3
:10DD0400D2854A85EFF05FEDD1B781474146B3062E
:10DD1400F5003387F500182303C806008507334749
:10DD2400070198A2E395C7FE8280011126CA4EC658
:10DD3400AE84AA8993053005130500034AC806CEAC
:10DD440022CC32899720FA1FE780802F2DC5130635
:10DD5400000381452A849720FA1FE7802064414606
:10DD6400CE8522859720FA1FE7802072A6850D466E
:10DD74001305D4019720FA1FE780207113060402CB
:10DD8400930504012285EF703075AA840D4693052E
:10DD9400D4024A859720FA1FE780206F22859720B6
:10DDA400FA1FE780E036F240624426854249D244B5
:10DDB400B24905618280CD44FDB75D714EDE62D407
:10DDC400AE892A8C9305300513050003A6C2CAC088
:10DDD40052DC56DA5AD85ED686C6A2C4B28B368BCB
:10DDE400BA84BE8A4289468A9720FA1FE780402572
:10DDF400630405101306000381452A849720FA1F43
:10DE0400E780C0594146E28522859720FA1FE780C2
:10DE1400C067414681450A859720FA1FE78000586C
:10DE24001D46DE850A859720FA1FE78000661D4699
:10DE3400DA85130571009720FA1FE78000653339EE
:10DE44002001B3349000414681450808230721018D
:10DE5400C4879720FA1FE78060541946D68548087E
:10DE64009720FA1FE78060621946D2851305A10145
:10DE74009720FA1FE7806061930404014146CE8530
:10DE840026859720FA1FE78040608A852685EFF073
:10DE9400DFE7930904024E86A6852285EF70D063DE
:10DEA4002A890DE94146CE8526859720FA1FE78009
:10DEB40040480C082685EFF05FE54E86A68522854E
:10DEC400EF7090612A8946454146CE859720FA1F16
:10DED400E780A05B22859720FA1FE7806023B64085
:10DEE40026444A8596440649F259625AD25A425BFC
:10DEF400B25B225C616182804D49D5B7011126CAAB
:10DF040052C4AA842E8A13050003930530054AC817
:10DF14004EC606CE22CC3289B6899720FA1FE780F6
:10DF2400201235C52A84A68541469720FA1FE7802A
:10DF3400C055930404012146D28526859720FA1FF3
:10DF4400E780A054CA852146130584019720FA1F4F
:10DF5400E780A05313090402A6854A862285EF7040
:10DF6400B057AA844146CA854E859720FA1FE78098
:10DF7400C05122859720FA1FE7808019F24062443D
:10DF840026854249D244B249224A05618280CD4461
:10DF9400F5B739715AD05ECE2A8BAE8B41459305C5
:10DFA400300506DE26DA52D456D262CC66CA6AC876
:10DFB400368C328DBA8C22DC4AD84ED69720FA1F82
:10DFC400E7800008AA8A9305300541459720FA1F87
:10DFD400E78000072A8ACD44638E0A0859C52A8639
:10DFE400D6855A85EFF03FC5AA8441E193053005F3
:10DFF40041459720FA1FE780A0042A89930530053C
:10E0040041459720FA1FE780A003AA89630A090EF5
:10E014006306050E1304FD0011841376FD0049C048
:10E024007D144204418035EE131544004E86D68596
:10E034005E95EFF01FB8414681454A859720FA1F47
:10E04400E780C035014D93170D01C18363F4870840
:10E05400BDC04A859720FA1FE780800B63870900BB
:10E064004E859720FA1FE780A00A56859720FA1F4D
:10E07400E780000A63070A0052859720FA1FE780A9
:10E084002009F250625426854259D254B259225A78
:10E09400925A025BF24B624CD24C424D2161828017
:10E0A4000144131544008A855E95EFF09FB54E86B2
:10E0B400D2850A85BDBF93154D000A86DE954A8533
:10E0C400EFF03FAF4A868A855A85EF70F040AA8404
:10E0D400050D95BFBDFC0A86CE854A85EFF07FAD60
:10E0E4004A868A855A85EF70303FAA846686CA8537
:10E0F40062859720FA1FE780C023A1BFCD4491BF5A
:10E10400CD44A9BF397162CC2A8C594526DA4AD844
:10E114004ED652D456D25AD05ECE06DE22DCAE8B18
:10E12400328BB68A3AC63E8AC28946898344010440
:10E134009720FA1FE78020102DCD9167938717E968
:10E144001EA185473CA12A8432472105630A0C0499
:10E15400930710033CB0194681459720FA1FE780C6
:10E16400E02323036401A303540144A8231274018C
:10E17400231744012318340123192401A285B73736
:10E1840000206254F250D2544259B259225A925A3F
:10E19400025BF24B624C03C5C79C21616F204FE9BF
:10E1A400A30104001946BA859720FA1FE780601876
:10E1B4004DBFF2506254D2544259B259225A925A23
:10E1C400025BF24B624C21618280011122CC2A84D1
:10E1D400314506CE2EC632C436C23AC09720FA1F45
:10E1E400E780600515C99167938717E91EA1B245B9
:10E1F4002246924602478D473CA120B16244B7377C
:10E2040000204EA172A116A53AA5F240AA8503C525
:10E21400C79C05616F20CFE1F240624405618280B2
:10E2240001114AC82A89394526CA06CE22CC2EC6EF
:10E23400B2849720FA1FE78000001DCDB245916794
:10E24400938727E91EA191473CA1A30125014EA173
:10E254002A84A685190521469720FA1FE780600DB8
:10E26400A285B73700206244F240D244424903C534
:10E27400C79C05616F20CFDBF2406244D24442491F
:10E284000561828001114AC82A89414526CA06CE01
:10E2940022CC2EC6B2849720FA1FE780C0F915CD90
:10E2A4009167B245938727E91EA195472A843CA12B
:10E2B40023122501214619059720FA1FE7806007DC
:10E2C400A28566A4B73700206244F240D244424992
:10E2D40003C5F79C05616F20AFD5F2406244D24478
:10E2E400424905618280011122CC2A84394506CE37
:10E2F4002EC632C436C23AC09720FA1FE780A0F374
:10E3040015C99167938717E91EA1B2452246924623
:10E31400024799473CA142A1B737002062446EA14D
:10E3240012A536A55AA5F240AA8503C5C79C056166
:10E334006F200FD0F240624405618280797122D44B
:10E3440006D62A842EC632C436C23AC09720FA1F93
:10E35400E780407419CDB245224692460247EC84C8
:10E36400F0852C081306F00F2285F486F887EFC099
:10E374003F89B250225445618280011122CC2A8403
:10E38400394506CE2EC632C436C23AC09720FA1F8B
:10E39400E78060EA15C99167938717E91EA1B24522
:10E3A4002246924602479D473CA142A1B73700202E
:10E3B40062446EA112A536A55AA5F240AA8503C5EA
:10E3C400C79C05616F20CFC6F2406244056182801C
:10E3D4005D713EC2835701062AC6130540024EDE14
:10E3E40052DC56DA5AD85ED662D466D26AD06ECE81
:10E3F40086C6A2C4A6C2CAC02E8DB28C368C3AC4BC
:10E40400C28DC68B035B0105835A4105034A81050E
:10E414008349C1053EC09720FA1FE780C0E161CD62
:10E424001166130616E9324312A1130690022A89D3
:10E4340030A19304E90021051304490192472247BE
:10E444006302030893071003A301F90019468145E9
:10E454009720FA1FE78080F4194681452685972086
:10E46400FA1FE780A0F31946814522859720FA1FF9
:10E47400E780C0F2824723039901A30389012300A3
:10E484004903A30039032311F9022644B7370020B6
:10E494002312A901231D7901231E6901231F590198
:10E4A400B6409644F259625AD25A425BB25B225C3D
:10E4B400925C025DF24DCA8503C5C79C0649616141
:10E4C4006F200FB7BA85A301090019463EC29720F1
:10E4D400FA1FE78000E6924726851946BE859720F5
:10E4E400FA1FE78000E51946EE8522859720FA1F7A
:10E4F400E78020E441B7B640264496440649F259E1
:10E50400625AD25A425BB25B225C925C025DF24D6B
:10E5140061618280011122CC2A84214506CE2EC657
:10E5240032C436C29720FA1FE780E0D005C92246DC
:10E5340092469167938717E91EA1B245B1473CA162
:10E5440020B170A174B16244B73700204EA1F240EB
:10E55400AA8503C5C79C05616F208FADF240624454
:10E564000561828041110D4506C69720FA1FE78098
:10E5740080CC15C1930710F91CA19307E0031CB1CB
:10E58400C5473CA1B7370020B240AA8503C5C79C44
:10E5940041016F20EFA9B24041018280011122CCD8
:10E5A4002A84294506CE2EC632C436C29720FA1FC5
:10E5B400E78060C805C9B24592469167938717E919
:10E5C4001EA12246C9473CA14CA120B114A5624416
:10E5D400B737002072A1F240AA8503C5C79C056124
:10E5E4006F200FA5F24062440561828001114AC880
:10E5F4002A892D4526CA06CE22CC2EC6B28497205F
:10E60400FA1FE78040C329C1B245930710F91CA142
:10E614009307E0031CB1CD473CA1A30125014CA104
:10E624002A84A685150519469720FA1FE78060D02D
:10E63400A285B73700206244F240D244424903C560
:10E64400C79C05616F20CF9EF2406244D244424988
:10E6540005618280011122CC2A84214506CE2EC672
:10E664009720FA1FE78020BD05C5B24591679387BF
:10E6740017E91EA1D1473CA16CA142A1B7370020E4
:10E684006244F240AA8503C5C79C05616F204F9A76
:10E69400F240624405618280011122CC2A84214522
:10E6A40006CE2EC632C49720FA1FE780C0B81DC11B
:10E6B4002246B245930710591EA120A170A16244BD
:10E6C400B73700204EA1F240AA8503C5C79C056157
:10E6D4006F200F96F240624405618280011122CCC2
:10E6E4002A84214506CE2EC632C49720FA1FE7801D
:10E6F40080B415C522469167938727E91EA1B245C8
:10E70400A1473CA160A170B16244B73700204EA17B
:10E71400F240AA8503C5F79C05616F206F91F24012
:10E72400624405618280011122CC2A84314506CEDF
:10E734002EC632C436C23AC09720FA1FE780A0AF73
:10E7440005C922468567B24592460247938717C991
:10E754001EA120A170A16244B73700204EA116A5C6
:10E764003AA5F240AA8503C5C79C05616F204F8C6A
:10E77400F240624405618280011126CAAE844AC80F
:10E784002A891385C40006CE22CC32C69720FA1FEC
:10E79400E78060AA0DCD8567938717E9B2451EA16E
:10E7A40024A1231225012A84310508C42686972032
:10E7B400FA1FE78000B8A285B73700206244F24010
:10E7C400D244424903C5C79C05616F206F86F2405D
:10E7D4006244D244424905618280011122CC2A84D8
:10E7E400194506CE2EC69720FA1FE780C0A405C59A
:10E7F4008567938717F91EA1B24585473CB120A1CF
:10E804006244B73700204EA1F240AA8503C5C79CD5
:10E8140005616F20EF81F2406244056182804111FD
:10E8240022C42A840D4506C69720FA1FE780A0A0BB
:10E834000DC1930710F91CA1E9471CB120A1224482
:10E84400B7370020B240AA8503C5C79C41016F10A9
:10E854003FFEB240224441018280011122CC2A842D
:10E86400214506CE2EC69720FA1FE780C09C0DC511
:10E874009167938727E91EA1B245930700033CA142
:10E8840060A16244B73700204EA1F240AA8503C5B7
:10E89400F79C05616F10DFF9F240624405618280E4
:10E8A4000111214506CE2EC632C49720FA1FE780F7
:10E8B400809805C58567B2452246938707391EA10E
:10E8C40085473CA1B73700204EA172A1F240AA852A
:10E8D40003C5479305616F10BFF5F240056182805F
:10E8E400397122DC1304F5FF4AD852D456D25ECED5
:10E8F400420406DE26DA4ED65AD0894B2A8A328959
:10E90400B68A418063937515B72B002083C70B5FCC
:10E914005E8B894495CF83C916009C229144A20939
:10E92400B3E9F900B737002083D78783F51763D19C
:10E93400F9029307C6FF639DF90831452EC6972057
:10E94400FA1FE780408F2A84B24519ED9304F00F33
:10E95400F250625426854259D254B259225A925ADC
:10E96400025BF24B216182804209135909014CA1D7
:10E9740023132501930700F91509A1651EA123118D
:10E98400450185054A859710FA1FE780606B08C426
:10E9940015C983C70B5F9385EAFF13562900FD173A
:10E9A4002388FB5E9720FA1FE780409C1C44A285C5
:10E9B40089071CC4B737002003C54793EF105FE7EE
:10E9C400814479B722859710FA1FE7806074BDBF30
:10E9D4009307D6FFE3CCF9F6B1473304F402B73416
:10E9E400002083A78493A297B82719C7884309C531
:10E9F4009710FA1FE780C07113854900A16542058D
:10EA04008505418103AA84939710FA1FE780406328
:10EA140083A78493229A2320AA00A29788431DD512
:10EA24000547B8A783470B5F4A86D685FD17230899
:10EA3400FB5E9720FA1FE780C08F83A784933E94E0
:10EA44002313240123123401A5BF8547E390F5F075
:10EA5400B1473304F402373B002083278B93DA89D0
:10EA6400A297FA2388435DC3DE23B306C700910748
:10EA740063CED7083A95D6859720FA1FE780608B36
:10EA840003278B93814422977E23CA97C207C183AD
:10EA94007EA35A231107E39DE7EA31459710FA1F35
:10EAA400E7806079AA850DCD930700F91EA183271D
:10EAB4008B932302750123114501A297FA239C43EA
:10EAC4007AA11CC5B737002003C54793EF105FD662
:10EAD40083278B933E9423130400230504008DBDE8
:10EAE40083278B93A297884311C99710FA1FE78055
:10EAF400206283278B93A29723A0070083A789937F
:10EB04003E9423130400230504005DBD11C997102E
:10EB1400FA1FE780E05F83A78993A29723A00700E9
:10EB240083A7899385443E9423130400230504009A
:10EB340005B56FA060206FA080216FA040450545FA
:10EB4400828005458280411106C6EFA08020B24034
:10EB54000145410182806FA0A0226FA060246FA0B4
:10EB640000276FA0C0286FA0602A6FA0202C6FA080
:10EB7400E02D6FA0A02F6FA040316FA000331C3296
:10EB84001022A2075D8E6FA060346FA0A0356FA025
:10EB940000386FA0603A6FA0C03C6FA000426FA025
:10EBA400E0436FA0C0456FA0A0476FA080496FA04D
:10EBB400604B411122C60344C10226C483440103AD
:10EBC40003430101030E4101834E8101034FC1013F
:10EBD400834F0102834241028343810222D632449D
:10EBE40026D8A2441ED416D27ED07ACE76CC72CA4F
:10EBF4001AC841016FA0604F6FA0C0486FA0A04A1F
:10EC04006FA0804C05458280054582800545828041
:10EC14006FB0504005458280054582806FB0B04595
:10EC2400B7E606008147938606DE1308F00F3387A4
:10EC3400F60010231317060141836364E500631390
:10EC44000601828092216364C7009AA182808507AD
:10EC540093F7F70FE9BF41119397050122C406C644
:10EC640026C2C1872E8463D607029710FA1FE78055
:10EC7400E061AA8401CD1C21054793C7070863649A
:10EC8400F700EF5090042685EF10BFB52165218D64
:10EC940021A893F7150091CFB737002083A7C7A306
:10ECA40091C3829713451400B24022449244410117
:10ECB400828093F7250091CBB737002083A707A460
:10ECC40091C3829713452400C5B793F7850099CB68
:10ECD400B737002083A7C7A4FC5791C38297134575
:10ECE4008400D9B793F7450099CBB737002083A7A1
:10ECF400C7A4BC5791C382971345440075B793F7D3
:10ED0400050281CFB737002083A707A683A7070989
:10ED140091C382971345040241BF93F7050181CF44
:10ED2400B737002083A707A683A7C70891C3829794
:10ED34001345040195BF939725010145E3D607F6D2
:10ED4400B73700209387879DF433F023CC33C8234F
:10ED5400EFA00049096525BF411126C2B734002040
:10ED6400B737002013060012814522C42A84138574
:10ED7400849D06C623AE07AE4AC09710FA1FE780EB
:10ED8400E0610145EF10D05A0145EF10B061B7279B
:10ED94000020A38D877CB707D7071384849DB5070C
:10EDA4005CC8B7B70D0D938707141CCCB7B7D7074A
:10EDB400938707145CCCED77938707147D471EB0C7
:10EDC400232CE40C81470327840C232EF40CE167E5
:10EDD4009387F79F5D8F8327C40C8966938606B05B
:10EDE40037390020D58F130989822326F40C232A6E
:10EDF400F40C8347E9002324E40C2328E40CA30A3D
:10EE0400F40AA30EF40AF977FD17231FF40E231056
:10EE1400F410FD472301F41085679387F7F03EBC97
:10EE24005EBCA30C0402EF206FE29307C01C2319FD
:10EE3400F4068547A30FF4028357490003570901D9
:10EE440028B0A983A30EF4068D472311F4042322CA
:10EE540004049306B00F9387849D63F4E6001307BC
:10EE6400B00F93150701BAB7FAB703C7C703C18137
:10EE74001386E500118B35CB1387A5080E0783C6CF
:10EE8400D70342074183DAB7918ABDC29386A508A6
:10EE94008E06C206C18296BB6D459384849DAE8660
:10EEA40063F3A500ED46B6B093058014BA86637487
:10EEB400B700930680141307C01C2390E704370798
:10EEC40016000E0613070790D6B3F2B396B7D8DB35
:10EED400EF70605FEF30A044EF6050472244B240CF
:10EEE4009244024941016F50F02A1317360041BF82
:10EEF4009316360079BF397122DC3704400026DAD4
:10EF04004ED6AE84AA899305E4FF054506DE4AD8A9
:10EF1400EF20AFDC498C131704014183218393173D
:10EF2400840013590401D98F231601001379F90FB2
:10EF340010088A854E857C87A306210102C002C27F
:10EF440002C402C802CA02CC02CEEF60F058834762
:10EF5400E1010347D101A0B0A2074207BA970347D2
:10EF6400F1012180C0A0BA97F25062549CA013D73B
:10EF74008700C183A382240198B0BCA04259D25413
:10EF8400B25921618280B735002037350020011144
:10EF9400194693850584130585AB06CE22CC26CA73
:10EFA4004AC891644EC69710FA1FE780803893854B
:10EFB400F4FF0145EF202FD02A84FD550145EF20B1
:10EFC400CFD1A287FD147D5933F79700B366E500CE
:10EFD400D5CA631425016307970A37340020130741
:10EFE400849D2308F70EA18393E707FC9169C1640C
:10EFF4002326A70EA308F70E1304849DFD19FD1400
:10F00400CE850145EF202FCB2A89FD550145EF2000
:10F01400CFCCB3672501EDD7FD576314F500E301A9
:10F0240039FF93570501230AF40E93578501A30A68
:10F03400F40E8317040E2319A40E230B240F420588
:10F04400135989001379F9034185A30B240F658DA6
:10F05400E58F6312F5020317440F8317240E658F9F
:10F06400E58F631AF7000317640F8317440E658F47
:10F07400E58FE307F7F8F2406244D2444249B249CB
:10F0840005618280A6850145EF20EFC22A84FD55E3
:10F094000145EF208FC4A28705BF411126C2B734B2
:10F0A400002006C622C44AC09387849D03C7E70391
:10F0B40083C7F703636AF70001442285B240224400
:10F0C40092440249410182802A8993051024130540
:10F0D40080079710FA1FE780A0F62A8471DD1306D3
:10F0E400800781459384849D9710FA1FE780002B45
:10F0F40063140900C1575CA0BC48B1E3E0C4A0C8D4
:10F10400E0C8232004008547238FF40285475CB0C0
:10F11400930700F97CB0B73700209387C7B19853A1
:10F12400DC5338C47CC4FD573CA8B737002003C562
:10F13400C7832302A406EF60904708B8BDBFFC480C
:10F1440080C3E0C82320040083C7E40385076DBFA0
:10F154003C2D411122C406C699075CB53C451147B4
:10F1640058A598A33C4558352A8498B3834715037A
:10F17400858B91E70347050389476317F7003844F4
:10F184001C2393E707041CA328449305240319466E
:10F1940009059710FA1FE780C0192844322C0C5433
:10F1A40021059710FA1FE780C018930730F97CB047
:10F1B400B24022444101828041114AC037390020C3
:10F1C4009307899D83A7C70A06C622C426C299E36A
:10F1D400054531AAAA841309899DEF60D06A832763
:10F1E400C90A8297EF20106C2A847DD19C50EC448C
:10F1F4002324F508F8309307A0096310F710854716
:10F204002300F51483C7F4052303F514A303F514AD
:10F21400FC3598290148A2074207BA97F8251546F4
:10F22400F905BA9703C735FF130584136207BA9724
:10F23400232CF40883C755FF03C765FFA2074207C1
:10F24400BA9703C745FFBA97232EF40883C775FFFF
:10F25400A30BF40283C795FF03C785FFA207D98FC9
:10F264001EBC83C7B5FF03C7A5FFA207D98F3EBC49
:10F2740083C7D5FF03C7C5FFA207D98F5EBC83C769
:10F28400F5FF03C7E5FF232E0413A207D98F7EBC25
:10F294008147232CF4129710FA1FE7808009F84461
:10F2A40083473702FD8BA30AF40203473702ED17A5
:10F2B40093F7F70F15832308E4022D476365F702DC
:10F2C4003E3C05679306A7C7E917C207C18363ECF1
:10F2D400F600563C9307301F63E7D7007E3C1307C4
:10F2E40007C8637BF7020A24EF20D07B0145B240B4
:10F2F400224492440249410182808327090D1397D5
:10F304001701E35707F0BC4498239C21F98F958398
:10F31400858B2300F514EDBD8327090B2285829785
:10F324008327890D0A24294693F7072091E305468C
:10F3340093050008EF50E0308327090D1397170158
:10F34400635807000A24514693050008EF50602FC4
:10F354008327C904BC4B13974700E35B07E6C82027
:10F36400A3890400494693050008EF50802D8DB50C
:10F37400B737002083C7979D411122C406C626C211
:10F384004AC02A8485EB582485476314F70E8347C3
:10F39400940303471404858B631BF70C19469305E8
:10F3A40024041305A4039710FA1FE7808009B334DB
:10F3B400A00099A883471504C5C78347750413079C
:10F3C400000493F7070C639DE708485529C5130902
:10F3D4002404CA851305A5029720FA1FE780A03EDE
:10F3E4008547AA846319F502485489472300F40425
:10F3F4003C311946CA8593E72700A300F40451055C
:10F404009710FA1FE780E0F2B240224426850249B1
:10F41400924441018280582485476303F70483475B
:10F42400C405918B95EF834784039DEB1305040476
:10F434009720FA1FE780604348D41DC18947230001
:10F44400F4043C3119469305240493E72700A300F0
:10F45400F40451059710FA1FE780A0ED85446DB7B9
:10F4640083478403898B85D35C549C3389FF81440F
:10F4740061BF8347C405918B99FB1C3413F71700B4
:10F4840005C374340D47639DE60028406C40224454
:10F49400B2409244024941011723FA1F6700E34333
:10F4A400898BCDDF78349547E31AF7FAF9BF411118
:10F4B400B737002022C406C69387879D2388070692
:10F4C400930710F97CB1B737002003A487AF0DC0B0
:10F4D400B727002003C5B77D8545EF10BFBD93074F
:10F4E40010273305F50222832244B24041010283EE
:10F4F400B2402244410182807C2991C7782163145F
:10F50400F7006FF0DFFA583901CF7421638FE600FA
:10F5140078A1B727002003C5B77D89456F106FE533
:10F52400EDD3782179FF7CA1EDB7E1DFEDBF6C4528
:10F5340031479C3193F7F7037CA56386E700930773
:10F5440000083E8582809C210D47BD8B7CB5E398E5
:10F55400E7FE41114AC01309250322C419462A842F
:10F56400A1054A8506C626C29710FA1FE78060EDFA
:10F574009147630505146C441946130524049C2122
:10F5840089059987858BA300F4049710FA1FE780F7
:10F5940040DA2285EFF0DFDDA14763010512130590
:10F5A400200483040401EF303FF76205618593076B
:10F5B400000863C5A41024449D475CA49CA085470F
:10F5C400BCA0BCB01946CA85138544009710FA1F25
:10F5D400E78020D6BC20B830990793F7F70F13675C
:10F5E4008700BCA0B8B03844BA9703578406B8B3B0
:10F5F400BC2038448346D4053E978357840692063C
:10F60400A183BD8BD58F5CA3B820814709071377ED
:10F61400F70FB8A0322C8346C40501CA93F7060439
:10F62400CDE7F957998F93F7F70F93F6060481CE38
:10F63400B030344413660604B0B03697143834B38B
:10F64400B8200507B8A0322C014709CE63ECC700E7
:10F65400BC2028440C548D073E959710FA1FE78070
:10F6640040CD382CB42093F7F60385073E9758B461
:10F67400B4A083471403858B91E7034704038947A8
:10F684006317F70038441C2393E707041CA33C4486
:10F694004C348CB3930790F97CB00345F40583474D
:10F6A40074065D8DEF60007D014681450D45972010
:10F6B400FA1FE780C066EF60101D8147B240224404
:10F6C400924402493E8541018280F557A1BF6C45B1
:10F6D400130720029C3193F7F7037CA5639CE71082
:10F6E400411122C406C626C29C2115472A84BD8B1B
:10F6F4007CB5639AE7021946A10513052503971003
:10F70400FA1FE78000D4914765C16C44194613057C
:10F7140024049C2189059987858BA300F404971000
:10F72400FA1FE78000C12285EFF09FC4A1474DCDA9
:10F73400B737002083A7C78182972444A14708D004
:10F744005CA49CA08547BCA0BCB0194693052403C7
:10F75400138544009710FA1FE780A0BDBC209907C9
:10F76400BCA0BC3093E72700BCB08347140491C706
:10F7740038441C2393E707F81CA319469305240473
:10F784001385A4009710FA1FE780A0BABC2099073C
:10F7940093F7F70F13F7F703050758B4BCA0834793
:10F7A4001403858B91E70347040389476317F70024
:10F7B40038441C2393E707041CA33C444C348CB307
:10F7C4009307A0F97CB00345F405834774065D8D67
:10F7D400EF60406A014681450D459720FA1FE78096
:10F7E4000054EF60500A8147B240224492443E855F
:10F7F40041018280930700083E85828041114AC0FE
:10F8040037390020832649B422C426C206C693078A
:10F81400000AFCD2B737002083A707B1B70533002D
:10F824002A84D857719B13671700D8D79843137746
:10F83400F7E798C398431377F7E71367071098C35C
:10F8440037370020032787B910474D8E10C713069A
:10F85400A005B0CA5057759A50D70347E5051376EB
:10F86400F7079843137707F8518F98C3DC420D4785
:10F8740093E71700DCC224459D475CA585469CA000
:10F88400A3810400B4A08347B5056385E700194745
:10F89400639EE7188547BCB0194693052403138576
:10F8A40044009710FA1FE780C0A8BC209907BCA0A9
:10F8B4000347B4059947631FF702BC301385A400BE
:10F8C40093E72700BCB083471403898B6381071235
:10F8D4004C54BC29638D07101946D1059710FA1FA3
:10F8E400E78020A538441C2393E707F81CA3BC2019
:10F8F4009907BCA0BC30B82093E78700BCB03C4457
:10F90400BA9703578406B8B3BC2038448346D40559
:10F914003E97835784069206A183BD8BD58F5CA343
:10F92400B820814709071377F70FB8A0122C834634
:10F93400C40501CA93F70604F9EBF957998F93F7B5
:10F94400F70F93F6060481CEB030344413660604F0
:10F95400B0B03697143834B3B8200507B8A0122CC9
:10F964004DEA0147B0208347A4059376F603850644
:10F9740036979A07D18F58B4BCA083471403858B5C
:10F9840091E70347040389476317F70038441C23AE
:10F9940093E707041CA33C44583498B3930760F9D5
:10F9A4007CB03844832749B4B8DBB737002083C719
:10F9B400C78781EB3705060081451305054CEF1019
:10F9C4002FF9B73700209387C7B1A3810700834578
:10F9D400F4058347740650342244B24092440249E9
:10F9E400DD8D014541011723FA1F67004333834727
:10F9F400940391C738441C2393E707F81CA31946C2
:10FA04009305A4039710FA1FE780A092CDB5F5578C
:10FA140035B7E3E8C7F4BC2028444C508D073E9525
:10FA24009710FA1FE780E090182C2DBF1387E7FF8B
:10FA34001377D70F79EF93052503B4B019461385CF
:10FA440044009710FA1FE780C08EBC20B8301146DE
:10FA5400990793F7F70F13678700BCA0B8B0384431
:10FA6400BA9703578406B8B3BC2038448346D405F8
:10FA74003E97835784069206A183BD8BD58F5CA3E2
:10FA8400B820814709071377F70FB8A08345B40559
:10FA94008346C4056399C50093F70604ADEBF95793
:10FAA400998F93F7F70F93F6060481CEB43093E65B
:10FAB4000604B4B034443697143834B3B820050778
:10FAC400B8A00346B405914601476310D602122C30
:10FAD40009CE63ECC700BC2028444C508D073E95EA
:10FAE4009710FA1FE780E084182C0346B40591466A
:10FAF400B73700209387879D6315D61483C60707FD
:10FB040093F6060F93E656002388D706A1BDF55752
:10FB140041BF93F7B70F0547E395E7E4BCB09305FE
:10FB240025031946138544009710FA1FE780608067
:10FB3400BC209907BCA0BC3093E72700BCB0834726
:10FB4400940391C738441C2393E707F81CA3834705
:10FB540014031385A400898BF9C34C54BC29E1C355
:10FB64001946D1059700FA1FE780A07C38441C236E
:10FB740093E707F81CA3BC20B8300546990793F710
:10FB8400F70F13678700BCA0B8B03844BA9703577F
:10FB94008406B8B3BC2038448346D4053E978357C3
:10FBA40084069206A183BD8BD58F5CA3B8208147C0
:10FBB40009071377F70FB8A08345B4058346C40536
:10FBC4006399C50093F70604BDEBF957998F93F732
:10FBD400F70F93F6060481CEB43093E60604B4B06E
:10FBE40034443697143834B3B8200507B8A0034614
:10FBF400B405854601476310D602122C09CE63EC86
